:100000000C9443510C9474510C9474510C9474518D
:100010000C9474510C9474510C9474510C9474514C
:100020000C9474510C9474510C9474510C9474513C
:100030000C944B750C9474510D942B150D946F12F8
:100040000C9474510D94C8220C9474510C947451F6
:100050000C9474510C9474510C9474510C94C46DA0
:100060000C9474510D94A59A0C9474510C94745181
:100070000C9474510C94F27D0C9474510C94745142
:100080000D9479170C9474510C9474510C94745110
:100090000D94619A0C9474510C9474510C94745195
:1000A0000C9474510C9474510D94B70D0C947451BC
:1000B0000C9474510D94990D0C9474510C947451CA
:1000C0000C9474510C9474510C9474510D94590DFA
:1000D0000C9474510C9474510C9474510C9474518C
:1000E0000C947451000000000000000000000000AB
:1000F0000000000000000000000000000000000000
:10010000A55AB44B2C2C8201B2056F6ECE80CEDE88
:100110001503400366038603B303FB032804760438
:10012000A504EF0423054B055F05710583059405C0
:10013000A205AF05C005EE050D0621063B065606D5
:10014000650676068A06D106FC06430750075B075C
:1001500063076A0714036F07770782078C079707FF
:10016000A107B107BC07C707D207E507F6070608CE
:100170001708260831083E084708500860086A0832
:100180008A089408A108B008B508C008CC08DB08A4
:10019000EA08F50801091309230934094309530939
:1001A0006309750985099709A109B009BB09C20945
:1001B000D009DD09E809EE09F609FA09FF090B0A79
:1001C000190A1E0A280A350A380A450A4F0A5D0A22
:1001D000600A640A740A800AA70AB20ABC0ADF0A23
:1001E000EE0AFA0A0B0B120B270B2C0B370B400BEA
:1001F000550B1403600B6D0B7A0B860B950BA60B3E
:10020000B60BC50BD40BE00BEE0BFE0B0E0C1A0C51
:100210002B0C3A0C470C570C670C770C8C0C990C78
:10022000A10CAC0CB30CB90CC40CCB0CD40CDA0C78
:10023000180D4D0D5D0D660D7A0D880DA40DD90DAF
:10024000440E6D0E9A0E020F490F910FDA0F131024
:10025000341056105C106910711085109810A2109F
:10026000DF1005114411871144118711C411F811D1
:1002700031125312E61262138013AB13CE13D8134C
:10028000E913F6132608091415142314361441141F
:10029000481454145D146B147A148D149D14A9140D
:1002A000B714C414D614E414F61407150E151C154F
:1002B000221532154315541567157C158F15A21597
:1002C000AD15D515DC1526163616471656166016CA
:1002D0006F167516891691169716A516B316C116C0
:1002E000D516E016EE16FD160C171B172C17521715
:1002F000A817FC17181882188C1894189C18A418A2
:10030000DA18FD18051968198B19CC191A1ABC1AB4
:10031000E91A181B5E1B851BAC1BC91B271C401C44
:100320007D1CD21CFA1C4E1D7D1D911DB41DD31DBC
:10033000F81D241E5F1EA01E051F1403921F9C1F84
:10034000A21FAE1FB71FBE1FCD1FD21FDD1FE41F90
:10035000E91FFB1F0A2010202520372047205920A5
:100360006620762086209720AA20B920CC20D8208D
:10037000EB2000210F211E2132214221562169212B
:100380007E21140393219F21B321C521D521E5218D
:10039000FA210222122227223A224A2257226B22D3
:1003A00080229522AA22BA22CC2214031403E0222E
:1003B000F32208231B232C233F234F236023742382
:1003C00086239823A623B523C523EC23F9233F24B2
:1003D00048244B244E246B24B024E3244225852555
:1003E000DB2511269026DB26112740275627A1273B
:1003F000CB27172882281229A029E229542ACD2A9E
:100400004A2BAF2B1403B82BBD2B14031403C52B9D
:10041000182C252C0050726F626C656D206DB174C4
:10042000742E205A20616B736A65706C616E657200
:10043000696E67207476756E676574202E2E2E00A7
:1004400053656E6765706C616E6572696E67206674
:1004500065696C65742E205072696E7420617662D5
:10046000727574742E005661726D6520736B7275AF
:100470006464206176207067612E2073696B6B6500
:10048000726865742E00472D636F646520736C6914
:1004900063656420666F7220656E20616E6E656EA6
:1004A0002068B17964652E20466F72747365747428
:1004B000653F00472D636F646520736C69636564F5
:1004C00020666F7220656E20616E6E656E2068B169
:1004D0007964652E2056656E6E6C6967737420733F
:1004E0006C6963652069676A656E2E205072696E5B
:1004F0007420617662727574742E00472D636F6488
:100500006520736C6963656420666F72206E79651F
:1005100072652066617374766172652E20466F7213
:100520007473657474653F00472D636F6465207351
:100530006C6963656420666F72206E7965726520F0
:1005400066617374766172652E2056656E6E6C6995
:10055000677374206F70706461746572207379734F
:1005600074656D65742E205072696E7420617662B8
:10057000727574742E00472D636F646520736C6907
:1005800063656420666F7220656E20616E6E656EB5
:10059000207072696E7465722E20466F7274736576
:1005A0007474653F00472D636F646520736C6963E5
:1005B000656420666F7220656E20616E6E656E20C8
:1005C0007072696E7465722E2056656E6E6C696706
:1005D000737420736C6963652069676A656E2E2089
:1005E0005072696E7420617662727574742E005454
:1005F00072796B6B2076616C67686A756C657420C4
:10060000666F72208F20666F727661726D652064EE
:100610007973656E206F6720666F7274736574748A
:10062000652E005472796B6B2076616C67686A7511
:100630006C657420666F72208F2074612075742041
:1006400066696C616D656E746574006F67207472A5
:10065000796B6B20708F206B6E617070656E0053CC
:1006600065747420696E6E2066696C616D656E7468
:1006700000466172676520696B6B652072696B74F7
:1006800069670046696C2E20696B6B65206C61732D
:10069000746574004279747465742072696B74694E
:1006A00067004C6173746572206661726765004211
:1006B000797474652076656C6C796B6B6574210058
:1006C00090706E652074616C6A6564B172656E20AD
:1006D0006F6720666A65726E2066696C616D656E13
:1006E00074657420666F7220688F6E642E00426C91
:1006F000652066696C616D656E746574206C6173EC
:100700007465742068656C742075743F0056656E5E
:100710006E6C69677374206F707064617465722E9B
:10072000004E792066617374766172652074696C1D
:10073000676A656E67656C69673A0056656E7465D1
:100740007220708F2050494E4441206E65646B6A60
:10075000B16C696E670056656E6E6C696773742064
:1007600076656E7400496E67656E206265766567B2
:10077000656C73652E0056656E74657220708F20EF
:100780006272756B65722E2E2E00456E2073746139
:1007900062696C20726F6D2D2074656D7065726179
:1007A00074757220708F2032312D323643206F677E
:1007B00020657420736F6C696420756E6465726C5B
:1007C0006167206572206EB16476656E6469672E1C
:1007D0000056656E6E6C696773742066756C6C6626
:1007E000B1722058595A206B616C696272657269E6
:1007F0006E67656E2066B17273742E0056656E6EFC
:100800006C69677374206C617374207574206669F9
:100810006C616D656E7465742066B17273742C20A2
:100820006465726574746572207265706574657252
:100830002064656E6E652068616E646C696E6765C4
:100840006E2E00472D636F646520736A656B6B00C5
:1008500044797365206469616D2E00416C66616244
:10086000657400536F72746572004461746F005355
:10087000442D6B6F72740056656C67207370728FB5
:100880006B00447973656279747465004757206F13
:10089000707073657474004C6173746574657374FF
:1008A00000467269676AB172206D6F746F7265720B
:1008B00000426576656720616B73650054656D70F5
:1008C0006572617475720050494E4441206B616CD1
:1008D0002E004E756C6C7374696C6C2058595A20DC
:1008E0006B616C2E0056697320656E646573656E6E
:1008F000736F72657200504944206B616C6962725B
:100900006572696E6700506C616E6B6F7272656BB9
:10091000742073656E670053656E6765706C616EF9
:100920006572696E67004B616C6962726572205A0C
:10093000004B616C69627265722058595A005365A8
:100940006C7674657374005665696C6564657200D5
:100950005465737465722066696C616D656E7400B0
:100960004C61737420416C6C65005472656B6B2034
:1009700075742066696C616D656E746564206D6563
:100980006420656E2067616E67004E756C6C7374D1
:10099000696C6C004769206E797474206E61766EA4
:1009A0000046B1727374656C6167736B616C2E0085
:1009B00056656C670053748F6C20706C61746500B1
:1009C00053797374656D20696E666F004665696C56
:1009D00020737461742E204D4D55004665696C730B
:1009E000746174697374696B6B00537461746973B7
:1009F00074696B6B004B616C6962726572696E67DA
:100A0000004175746F4C6173742066696C616D652B
:100A10006E74004C61737420696E6E2066696C613F
:100A20006D2E004C6173742075742066696C616D65
:100A3000656E74004C6173742074696C2064797302
:100A4000656E00466F726C6173742074696C204D22
:100A50004D550053442D6B6F7274206D616E676C41
:100A60006572005072696E74206672612053442D65
:100A70006B6F727400476A656E6F7070746120707E
:100A800072696E74005061757365207072696E745E
:100A90006A6F6262656E00476AB172206B6C617248
:100AA000005365747420696B6B65206B6C61720018
:100AB000466F727661726D696E67004A7573746510
:100AC00072004A7573746572204C6976652D5A0000
:100AD000476A656E7461207072696E7400496E6653
:100AE0006F736B6A65726D00486A656C7000456E65
:100AF0002067616E67004C79640048B179740046E4
:100B0000696C2E2053656E736F7200427974742085
:100B100066696C616D656E7400466C79740048613D
:100B200073746967686574004D61676E6574206BE6
:100B30006F6D702E00202D005A2D73656E736F72CD
:100B4000206E722E00506C616E2D6E6574740049BB
:100B50006E6E7374696C6C696E676572004A6100D1
:100B60004E65690053746F7070207072696E746A9C
:100B70006F626200536A656B6B65722066696C0018
:100B800046696C20657220756B6F6D706C6574744E
:100B90002E20466F7274736574746520616C6C6985
:100BA0006B6576656C3F0084466F72667269736B25
:100BB0006500486F7665646D656E790056656E7484
:100BC000657220708F20647973652D206F672070A7
:100BD0006C6174656E65646B6AB16C696E670056B2
:100BE000656C672066696C616D656E743A0053656B
:100BF0006C7674657374204F4B0053656C76746526
:100C000073742073746172746572004279747465D0
:100C100074004672656D72652F76656E73747265C9
:100C200020766966746500416B736500416B73657E
:100C30006C656E676465004CB173207265696D0008
:100C4000547261666620696B6B6520656E646573BE
:100C5000656E732E00456E646573656E736F72000A
:100C6000456E646573656E736F726572004B6F627B
:100C70006C696E67736665696C0053656E672F56A5
:100C800061726D657200496B6B652074696C6B6F86
:100C9000626C6574005661726D65722F5465726D79
:100CA0006973746F720056656E6C69677374207334
:100CB0006A656B6B3A0053656C7674657374206675
:100CC00065696C210046696C616D656E7473656E53
:100CD000736F72005072696E7476696674653A005B
:100CE000486F74656E642D76696674653A004B6171
:100CF0006C6962726572657220686A656D00536521
:100D00006C7674657374206665696C657400416CFB
:100D100074206B6F7272656B7400536A656B6B65E0
:100D2000722073656E736F72657200536A656B6BC8
:100D3000657220686F74656E6400536A656B6B65DD
:100D4000722073656E6700536A656B6B6572205A1B
:100D500020616B73656E00536A656B6B6572205919
:100D600020616B73656E00536A656B6B657220580A
:100D700020616B73656E00536A656B6B65722065ED
:100D80006E646573656E736F726572004B6F72741B
:100D900020666A65726E65740054696C62616B6589
:100DA000004175746F737479726B65004C79646C73
:100DB000B173004D6F6475730048B1792073747915
:100DC000726B6500537472656E6700416476617280
:100DD00073656C00496E67656E00486F74656E647C
:100DE00020708F203238304321204479736520628F
:100DF0007974746574206F6720737472616D6D65AA
:100E0000742074696C20737065736966696B6173B3
:100E10006A6F6E656E653F00466F72208F20627943
:100E200074746520647973652C2076656E6E6C69C8
:100E3000677374206C65730A70727573612E696FC5
:100E40002F6E6F7A7A6C652D6D6B33730050494449
:100E5000206B616C2E20666572646967005049449E
:100E6000206B616C2E005072696E74207361747413
:100E700020708F207061757365005072696E7420E8
:100E800061766272757474004B6F7069657265206B
:100E90006465742076616C677465207370728F6B03
:100EA00065743F00447973656469616D657465724A
:100EB000656E20657220666F72736B6A656C6C6913
:100EC000672066726120472D436F64652E20466F50
:100ED000727473657474653F005072696E746572E4
:100EE000656E7320647973656469616D657465729C
:100EF00020657220666F72736B6A656C6C6967201F
:100F000066726120472D436F64652E20536A656BBE
:100F10006B20496E6E7374696C6C696E67657220C4
:100F2000666F722068766120736F6D206572207322
:100F30006174742E205072696E74206176627275CD
:100F400074742E0044657420657220696E67656E46
:100F50002066696C616D656E74206C617374657474
:100F60002E20466F727473657474653F0044657417
:100F700020657220696E67656E2066696C616D65BB
:100F80006E74206C61737465742E205072696E7477
:100F900020617662727574742E00446574207472D8
:100FA000656E677320666F727473617474206B6111
:100FB0006C6962726572696E67206176205A206181
:100FC0006B73656E2E2044752066696E6E657220A7
:100FD0004B616C6962726572696E6720756E6465DB
:100FE0007220686F7665646D656E79656E206F67D7
:100FF0002066B16C67205665696C65646572656EC4
:101000002E005072696E746572656E20657220697B
:101010006B6B65206B616C6962726572742E205611
:10102000656E6E6C69677374207365206D616E7593
:10103000616C656E2C20756E6465722046697273F2
:10104000742053746570732E0053656C76746573E9
:10105000742076696C20626C69206B6AB1727420AE
:10106000666F72208F206B616C6962726572652099
:101070006EB179616B7469672073656E736F726CA2
:10108000B17320686A656D706F7369736A6F6E2ED5
:101090000047616D6C6520766572646965722066D3
:1010A000756E6E6574205374616E646172696E6EE4
:1010B0007374696C6C696E67657220666F7220501C
:1010C00049442C204573746567206574632E206243
:1010D0006C697220736174742E004164766172735E
:1010E000656C3A20428F6465207072696E74657217
:1010F00074797065206F6720686F7665646B6F72B6
:101100007479706520657220666F72616E647265B5
:10111000742E00416476617273656C3A2050726976
:101120006E7465727479706520666F72616E647238
:1011300065742E00416476617273656C3A20486F65
:101140007665646B6F727479706520666F72616E1C
:10115000647265742E00506C617465005370696E22
:101160006E657220696B6B65005370696E6E657297
:101170000056656E73742E20686F74656E647669B0
:101180006674653F004672656D7265207072696EA7
:101190007476696674653F00566966746574657334
:1011A000740058595A206B616C6962726572696E7D
:1011B00067656E20657220677265692E20536B6AC1
:1011C000657668657420626C6972206A75737465EF
:1011D0007274206175746F6D617469736B2E005841
:1011E000595A206B616C6962726572696E67656ECF
:1011F00020657220676F642E20476F6474206A6FC9
:10120000626261210058595A206B616C6962726593
:1012100072696E67204F4B2E0A58206F6720592045
:10122000616B73656E2065722070657270656E64A7
:10123000696B756C91722E2047726174756C657262
:101240006572210058595A206B616C69627265722F
:10125000696E67656E206665696C65742E2048B19D
:101260007972652066726F6E74206B616C69627250
:101270006572696E677370756E6B7420696B6B65F0
:10128000206E8F64642E0058595A206B616C69621D
:10129000726572696E67656E206665696C65742E2D
:1012A0002046726F6E74206B616C69627265726940
:1012B0006E677370756E6B7420696B6B65206E8FD3
:1012C00064642E0058595A206B616C2E206D69732E
:1012D0006C796B7465732E2056656E6E6C696773DE
:1012E0007420728F6466B172206D656420688F6EA1
:1012F00064626F6B656E2E0058595A206B616C6981
:1013000062726572696E67656E206665696C657488
:101310002E204B616C6962726572696E67737075BD
:101320006E6B7420696B6B652066756E6E65742ECE
:1013300000506C61737365722073748F6C706C6194
:1013400074656E20708F207661726D6573656E674F
:10135000612E0041767374616E64206D656C6C6FF4
:101360006D2074757070656E206176206479736588
:101370006E206F672073656E676120657220696BF0
:101380006B65206B616C6962726572742E205665A4
:101390006E6E6C69677374207365206D616E756124
:1013A0006C656E2C20756E6465722046697273746C
:1013B0002053746570732C20666F722068766F728C
:1013C00064616E206465742066B172737465206C0C
:1013D0006167657420736B616C206B616C6962720C
:1013E000657265732E00506C61737365722065744D
:1013F0002061726B20756E64657220647973656E0E
:10140000206D656E73206A6567206B616C6962721E
:101410006572657220646520342066B172737465EC
:101420002070756E6B74656E652E2048766973202A
:10143000647973656E207461722070617069726581
:10144000742C20736B727520756D696464656C62B1
:10145000617274206176207072696E746572656E57
:101460002E0053B16B6572206574746572206B61D8
:101470006C6962726572696E677370756E6B740009
:101480004D8F6C6572207265666572616E736568FA
:10149000B179646520666F72206B616C69627265F8
:1014A00072696E677370756E6B740052656E676AF1
:1014B000B17220647973656E206F67207472796BE6
:1014C0006B2076616C67686A756C65742E00417577
:1014D000746F20686A656D00476A656E6F7070741E
:1014E0006172207072696E740050494E44412076DA
:1014F00061726D6573004B616C6962726572696ED1
:1015000067206665726469670053656E672066656B
:10151000726469670053656E67656E207661726DEF
:101520006573004F70707661726D696E67206665D5
:10153000726469672E005661726D6572206F7070FB
:1015400000546F74616C7400536973746520707219
:10155000696E74004D4D55206665696C004D4D55A2
:10156000206C617374656665696C004D4D55207320
:101570007472B16D206665696C004D617465726945
:10158000616C757476656B736C696E670053697313
:101590007465207072696E746665696C0046656971
:1015A0006C20746F74616C7400546F6D7420666984
:1015B0006C616D656E740054656D706572617475F3
:1015C0007265720053656E736F72696E666F726DCD
:1015D00061736A6F6E00456B7374727564657269CE
:1015E0006E666F0058595A2063616C2E20646574D2
:1015F000616C6A6572005072696E74657220495040
:10160000206164722E3A00756B6A656E74004D4DF0
:10161000552074696C6B6F626C6574004461746F03
:101620003A00666F722066696C616D656E74207534
:101630007400666F722066696C616D656E746C61B2
:101640007374005472796B6B2076616C67686A758D
:101650006C657400466F727661726D657220666F9C
:1016600072206B75747400466F727661726D65726C
:1016700020666F722075746D61742E00466F7276ED
:1016800061726D657220666F722066696C2E00460D
:101690006F727661726D657220666F72206C617315
:1016A00074004E65646B6AB16C696E67004B6F6D58
:1016B0006D65722046696C616D656E74207574206D
:1016C0006F67206861722072696B74696720666158
:1016D0007267653F004CB173207574004175746F7B
:1016E0006C617374696E672061762066696C2E2068
:1016F000657220616B7469766572742E20547279FC
:101700006B6B20708F206B6E617070656E206F67E1
:10171000207365747420696E6E2066696C616D65F6
:101720006E742E2E2E0046696C616D656E74207489
:101730006F74616C74005072696E746574696420B2
:10174000746F74616C74004272756B742066696C9E
:10175000616D656E74005072696E746574696400C1
:10176000466F727661726D20647973656E210046F2
:1017700045494C3A00592064697374616E73652061
:10178000667261206D696E2E0056656E73747265A7
:101790000048B1797265004D8F6C7420736B6A6577
:1017A00076686574004C65747420736B6A6576683E
:1017B00065740053746F7220736B6A657668657424
:1017C000005B303B305D2070756E6B74666F7273BA
:1017D0006B79762E004A75737465726572205A00B3
:1017E00042616B736964656E205BE46D5D004672F7
:1017F000656D736964656E205BE46D5D0048B17969
:10180000726520736964655BE46D5D0056656E7397
:101810002E20736964655BE46D5D00536174742010
:1018200074656D706572617475723A0045722076E8
:10183000656E73747265206F672068B17972652078
:101840005A2D766F676E2068656C74206F707065B6
:101850003F004B616C69627265722058595A2E20A4
:10186000526F7465722076616C67686A756C657416
:1018700020666F72208F20626576656765205A2D1D
:10188000616B73656E2074696C20746F7070737413
:101890006F7070656E652E20446572657474657234
:1018A000207472796B6B2E004B616C696272657289
:1018B000205A2E20526F7465722076616C67686AB8
:1018C000756C657420666F72208F2062657665671F
:1018D00065205A2D616B73656E2074696C20746F7E
:1018E000707073746F7070656E652E2044657265DC
:1018F00074746572207472796B6B2E0050494E447B
:1019000041206B616C6962726572696E67206D69F6
:10191000736C796B7465730050494E4441206B6160
:101920006C6962726572696E672065722066756C9B
:101930006C66B17274206F6720616B7469762E20BB
:10194000446572206B616E20626C692020736B723B
:101950007564642061762069206D656E79656E20FE
:10196000756E64657220496E6E7374696C6C696E15
:10197000676572202D3E2050494E4441206B616CBA
:101980002E00456B737472756465720042657665EE
:1019900067205A0042657665672059004265766582
:1019A00067205800506C61746520252E37730A5AE1
:1019B000206F66667365743A20252B312E33666D71
:1019C0006D0A2563466F727473657474650A2563C6
:1019D0004E756C6C7374696C6C0056656E6E6C69D8
:1019E000677374207365747420696E6E2066696C09
:1019F000616D656E742066B17273742E003E41761F
:101A00006272797400566564208F206B6AB17265CA
:101A1000205665696C65646572656E20736C6574CB
:101A200074657320616C6C206E8F769172656E6444
:101A300065206B616C6962726572696E677364615F
:101A40007461206F67206475206D8F2062656779EF
:101A50006E6E6520708F206E7974742E20466F72C2
:101A60007473657474653F00466F727661726D655C
:101A70007220647973656E2E2056656E6E6C696790
:101A800073742076656E742E2E2E00536574742048
:101A9000696E6E2066696C616D656E7420492065A3
:101AA0006B73747275646572656E206F67207472F3
:101AB000796B6B2076616C67686A756C65742066FB
:101AC0006F72208F206C617374652E00536574747F
:101AD00020696E6E2066696C616D656E7420692088
:101AE0006465742066B1727374652072B172657436
:101AF0002062616B204D4D55206F67207472796BA9
:101B00006B2076616C67686A756C657420666F72AD
:101B1000208F206C617374652E005072696E74653D
:101B200072656E2076696C206E8F207072696E749B
:101B30006520656E2073696B6B73616B6B206C69DC
:101B40006E6A652E20526F7465722076616C6768CC
:101B50006A756C65742074696C20647520668F7278
:101B60002064656E206F7074696D616C652068B16A
:101B70007964656E2E2053652062696C64656E65BC
:101B8000206920688F6E64626F6B612C20756E64B3
:101B90006572204B616C6962726572696E672C2098
:101BA000666F722068766F7264616E20646574205F
:101BB000736B616C2073652075742E0056656C67BD
:101BC0002074656D70657261747572656E20736FD7
:101BD0006D207061737365722064697474206D6127
:101BE00074657269616C652E0056656C6720666964
:101BF0006C616D656E747479706520666F722046D5
:101C0000B1727374656C6167732D206B616C69626E
:101C1000726572696E672E004A65672076696C206E
:101C20006E8F206B616C696272657265206176737C
:101C300074616E64656E206D656C6C6F6D2074757B
:101C40007070656E20617620647973656E206F67B1
:101C5000207661726D65706C6174656E2E005A2D10
:101C60006B616C6962726572696E6720616E626534
:101C700066616C65732E204B6AB172652064657471
:101C8000206E8F3F0056656E6E6C696773742074AA
:101C9000612073748F6C706C6174656E2061762046
:101CA0007661726D6573656E67612E004572207393
:101CB000748F6C706C6174656E20708F20766172A9
:101CC0006D6573656E67613F0056656E6E6C696722
:101CD000737420736A656B6B20688F6E64626F6BC0
:101CE000656E206F672066696B732070726F626C1F
:101CF000656D65742E20466F7274736574742073FD
:101D00008F205665696C65646572656E20766564C2
:101D1000208F206F6D737461727465207072696EAC
:101D2000746572656E2E00416C74206B6C61727408
:101D30002E20476F64207072696E74696E6721008F
:101D40004475206B616E20616C6C746964207374DF
:101D500061727465205665696C65646572656E2094
:101D6000667261204B616C6962726572696E672090
:101D70002D3E205665696C656465722E0048766953
:101D8000732064752068617220616E6472652073CF
:101D9000748F6C706C617465722C206B616C6962FD
:101DA000726572206465206920496E6E7374696C77
:101DB0006C696E676572202D3E204857205365740C
:101DC0007570202D3E2053748F6C706C6174657239
:101DD0002E0052656E676AB1722073748F6C706CDE
:101DE0006174656E206F67207472796B6B20766109
:101DF0006C67686A756C65742E0056696C20647532
:101E000020726570657465726520646574207369FD
:101E1000737465207472696E6E657420666F7220CB
:101E20008F206F6D6A757374657265206176737447
:101E3000616E64656E206D656C6C6F6D2064797386
:101E4000656E206F6720706C6174656E3F0056652B
:101E50006C67206479736574656D70657261747503
:101E60007220736F6D207061737365722064697482
:101E700074206D6174657269616C652E0045722015
:101E800066696C616D656E74206C61737465743F16
:101E9000004A65672076696C206E8F20666F7276C7
:101EA00061726D6520647973656E20666F72205073
:101EB0004C412E004E8F206B6AB1726572206A65AC
:101EC00067205A2D6B616C6962726572696E676515
:101ED0006E2E00466A65726E206E8F207465737474
:101EE0007072696E746574206672612073748F6C91
:101EF000706C6174656E2E0056656E6E6C696773EA
:101F00007420666A65726E2073656E64696E6773AD
:101F10006265736B797474656C73656E2066B172FB
:101F200073742E004E8F20736B616C206A6567207E
:101F30006B6AB17265206B616C6962726572696E01
:101F400067656E2E20446574206B616E207461207D
:101F50006F707074696C203234206D696E2E00468B
:101F6000B172737420736B616C206A6567206B6A51
:101F7000B1726520656E2073656C7674657374202C
:101F8000666F72208F20736A656B6B652076616E59
:101F90006C6967652062796767656665696C2E00A4
:101FA0004865692C206A65672065722064696E2027
:101FB0004F726967696E616C65205072757361203C
:101FC0006933207072696E7465722E2056696C20B8
:101FD0006475206174206A656720736B616C20767C
:101FE00065696C6564652064656720676A656E6E07
:101FF0006F6D206F70707365747470726F7365733A
:1020000073656E3F004865692C206A6567206572BC
:102010002064696E204F726967696E616C6520503B
:1020200072757361206933207072696E7465722EE7
:10203000204A6567206C6564657220646567206965
:10204000676A656E6E6F6D206574206B6F727420A9
:102050006F7070736574742C2068766F72205A20CC
:10206000616B73656E20626C6972206B616C696272
:10207000726572742E204475206572206461206B35
:102080006C61722074696C208F207072696E746547
:102090002E00465320616B736A6F6E00466F727438
:1020A0002E00462E206175746F6C61737400462E8D
:1020B000204CB1707574004B75747465720056696C
:1020C0006674656861737469676865740053656EEA
:1020D00067005669667465736A656B6B004D6F6463
:1020E000656C6C0044797365004D61746572207491
:1020F000696C204653656E736F7200466C79747418
:1021000065722076656C6765720053B16B6572000D
:1021100074612074696C62616B652066726120462F
:10212000494E4441004D61746572207574206669A2
:102130006C616D656E74005061726B6572657220C2
:1021400076656C6765720052657475726E6572654E
:10215000722076656C67657200557466B17265723F
:10216000206B757474004479747465722066696CB0
:10217000616D656E7400466F72626572656465724A
:1021800020626C61640056656C6765722066696CDC
:102190002E2073706F72004C6173746572207574B9
:1021A0002066696C616D656E740045525220544D15
:1021B00043206665696C65740045525220486A6523
:1021C0006C702066696C616D656E740045525220BA
:1021D000496E7465726E74004552522056656E7475
:1021E00020708F204272756B6572004176736C753A
:1021F00074746572206265766567656C73657200DC
:10220000556E6E678F7220736C6970696E67004DD2
:10221000617465722074696C2064797365004D6126
:102220007465722074696C20656B73747275646573
:1022300072004D617465722074696C2046494E4489
:10224000410055746C61737465722074696C2074FC
:1022500072696E73650055746C6173746572207475
:10226000696C2046494E444100467269676AB17202
:1022700020746F6D67616E6773686A756C00416B7F
:102280007469766572657220746F6D67616E6773CD
:10229000682E00554B4A454E54204645494C004552
:1022A0004E4452494E472041562046494C414D45E7
:1022B0004E540046494C414D454E542055545345CB
:1022C00054544554004C415354205554204D414ED4
:1022D00055454C540046572052554E54494D4520C3
:1022E0004645494C004D4D55204656204F505044D0
:1022F00041542E204EB24456450046554C4C204B7E
:10230000B2005547594C444947205645524B54B2A8
:10231000590046494C414D454E5420414C4C455284
:10232000454445204C41004B4F4D4D554E494B4186
:10233000534A4F4E534645494C004D4D5520535638
:102340004152455220494B4B45004D4D55204D4380
:1023500055204645494C004D4D552053454C56544B
:10236000455354204645494C455400544D43204460
:102370005249564552204B4F5254534C55545400D9
:10238000544D43204C41565350454E4E494E4720E4
:102390004645494C00544D4320445249564552202D
:1023A0004E554C4C5354494C4C00544D43204452D0
:1023B00049564552204645494C00544D43204F56FE
:1023C00045524F5050484554494E4700564152538C
:1023D000454C20544D4320464F52205641524D000B
:1023E00053454C454B544F52205354905220464134
:1023F00053540056454C474552204B414E20494BC3
:102400004B4520484F4D45004D49534C554B5420AA
:102410004C41535420455854522E004B4F4E545269
:102420004F4C4C45522046494E4441004653454E80
:10243000534F5220464F52205449444C4947005272
:1024400045494D20554245564547454C494700466C
:1024500053454E534F522046494C20464153540059
:102460004653454E534F5220494B4B4520544952F9
:1024700047472E0046494E44412046494C414D2E87
:1024800020464153540046494E444120494B4B4558
:102490002055544CB25354004B7574742066696CCB
:1024A000616D656E74004CB1732075742066726145
:1024B000204D4D55004C61737465722066696C61E6
:1024C0006D656E74004D4D552052657472793A20D9
:1024D000676A656E6F70707265747465722074657A
:1024E0006D706572617475722E2E2E00536F72744A
:1024F00065722066696C6572004E6F656E20666954
:102500006C65722076696C20696B6B6520626C6902
:1025100020736F72746572742E204D616B7320612D
:102520006E74616C6C2066696C6572206920656EE2
:10253000206D61707065206572203130302E00533F
:10254000544F505045542E00417600508F00446542
:1025500074206F707073746F6420656E207576657B
:102560006E746574206665696C2E004D36303020BF
:1025700066696C616D656E74736B696674652E2037
:102580005365747420696E6E20656E206E792066C6
:10259000696C616D656E7420656C6C6572206CB1E0
:1025A000732075742064656E2067616D6C652E0004
:1025B000466A65726E206465742075746B6173740D
:1025C0006564652066696C616D656E74657420660E
:1025D00072612066726F6E74656E206176204D4D5B
:1025E000552E0046696C616D656E74206F70706465
:1025F00061676574207576656E7465742E20506110
:10260000737320708F20617420696E67656E206619
:10261000696C616D656E74206572206C61737465A0
:10262000742E20536A656B6B2073656E736F7265D1
:102630006E65206F67206C65646E696E67656E6598
:102640002E00496E7465726E2072756E74696D65C8
:10265000206665696C2E205072B176206F6D7374A0
:10266000617274206176204D4D5520656C6C6572E9
:10267000206F707064617465722066617374766136
:1026800072656E2E004D4D552066617374766172D1
:1026900065766572736A6F6E20657220696E6B6F06
:1026A0006D7061746962656C206D656420736B7216
:1026B00069766572656E732046572E204F70706480
:1026C00061746572696E672074696C2076657273D7
:1026D0006A6F6E20332E302E332E004D4D552066FE
:1026E0006173747661726520696E7465726E2066BE
:1026F00065696C2C2076656E6E6C69677374206EEC
:10270000756C6C7374696C6C204D4D552D656E2E17
:1027100000466F726573707572742066696C616DC6
:10272000656E747665726B74B17920657220696B21
:102730006B652074696C676A656E67656C69672094
:10274000708F2064656E6E65206D61736B696E7647
:102750006172656E2E20536A656B6B20672D636F07
:10276000646520666F72207665726B74B179732D23
:10277000696E74656B732075742061762072656B69
:102780006B657669646465202854302D54342900C3
:102790004B616E20696B6B6520757466B172652044
:1027A00068616E646C696E672C2066696C616D652A
:1027B0006E74657420657220616C6C657265646509
:1027C000206C61737465642E2041766C6573732090
:1027D0006465742066B17273742E004D4D5520737C
:1027E000766172657220696B6B652072696B7469C2
:1027F000672E20536A656B6B206C65646E696E672B
:102800006572206F67206B6F626C696E6765722EF0
:10281000004D4D552073766172657220696B6B6552
:102820002E20536A656B6B206C65646E696E6765FC
:1028300072206F67206B6F626C696E6765722E0025
:10284000466C65726520646574616C6A6572206FA0
:102850006E6C696E650049646C6572656E206B61B3
:102860006E20696B6B6520678F20686A656D2072CA
:10287000696B7469672E20736A656B6B206F6D20BE
:102880006E6F652073748F72206920766569656E3E
:1028900020666F72206265766567656C73656E2E63
:1028A000004B616E20696B6B6520666C7974746592
:1028B0002076656C67657220656C6C657220746F3C
:1028C0006D67616E6773686A756C0056656C6765E5
:1028D00072656E206B616E20696B6B6520678F205F
:1028E000686A656D2072696B7469672E20736A650A
:1028F0006B6B206F6D206E6F652073748F72206913
:1029000020766569656E20666F7220626576656700
:10291000656C73656E2E004C617374696E6720740C
:10292000696C20656B73747275646572206D697370
:102930006C796B7465732E20496E73706973657260
:102940002066696C616D656E747370697373656E12
:102950007320666F726D2E2041766772656E7320EC
:1029600073656E736F726B616C6962726572696EAA
:1029700067656E206F6D206EB16476656E64696701
:102980002E0056656C676572656E206B616E2069FE
:102990006B6B65206265766567652073656720707F
:1029A0008F206772756E6E206176206174204649B3
:1029B0004E4441206F7070646167657220656E20BF
:1029C00066696C616D656E742E2053B17267206606
:1029D0006F7220617420696E67656E2066696C2E67
:1029E00020657220692076656C676572656E206F60
:1029F000672061742046494E44412066756E6765C4
:102A000072657220736F6D2064656E20736B616CEC
:102A10002E0046696C616D656E742073656E736F10
:102A20007220626C652075746CB1737420666F726D
:102A3000207469646C6967206D656E7320656B73C3
:102A4000747275646572656E20626C65206C61736A
:102A50007465742E20536A656B6B20617420696EF7
:102A600067656E74696E672073748F722066617318
:102A700074206920505446452072B17265742E202E
:102A8000536A656B6B2061742073656E736F72653A
:102A90006E206C657365722072696B7469672E00B5
:102AA0005265696D6D6F746F72207374616E7365BA
:102AB000742E20536A656B6B206174205265696DBA
:102AC000656E206B616E2062657665676573206F49
:102AD0006720736A656B6B206B6F626C696E6765EC
:102AE000720046696C616D656E742073656E736FFC
:102AF0007220736B727564646520696B6B6520610D
:102B00007620696D656E732066696C616D656E74A3
:102B10006574206C61737465742075742E2053691C
:102B20006B72652061742066696C616D656E746599
:102B300074206B616E2062657665676573206F67D0
:102B40002073656E736F72656E2066756E67657251
:102B500065722E0046696C616D656E742073656EDA
:102B6000736F7220626C6520696B6B652075746C85
:102B7000B1737420696D656E732066696C616D65F3
:102B80006E74657420626C65206C61737465742E5C
:102B90002053696B72652061742066696C616D6594
:102BA0006E7465742072656B6B6572206673656EFA
:102BB000736F72206F672061742073656E736F721C
:102BC000656E2066756E67657265722E0046494EA9
:102BD000444120626C6520696B6B6520736C617485
:102BE0007420617620756E6465722066696C616D13
:102BF000656E742075746C617374696E672E2050F5
:102C000072B176208F206C617374207574206D61B1
:102C10006E75656C742E2053696B7265206174202B
:102C200066696C616D656E746574206B616E20629F
:102C3000657665676573206F672046494E4441207D
:102C400066756E67657265722E0046494E44412076
:102C5000626C6520696B6B65207472696767657269
:102C600020756E646572206C617374696E67206193
:102C7000762066696C616D656E742E2053696B7287
:102C8000652061742066696C616D656E7465742081
:102C90006B616E2062657665676573206F6720469D
:102CA000494E44412066756E67657265722E004418
:102CB00065616B7469762E004C617374004C6173AE
:102CC000742075740053656E6765706C616E657213
:102CD000696E67206665696C65742E2053656E7336
:102CE0006F72656E2075746CB17374657320696B57
:102CF0006B652E2052657374657220708F20647925
:102D000073656E3F2056656E74657220708F206FFC
:102D10006D73746172742E0053656E736974697695
:102D2000697465740046657264696700000000009C
:102D30000000000000000000000000000000000093
:102D40000000000000000000000000000000000083
:102D50000000000000000000000000000000000073
:102D60000000000000000000000000000000000063
:103600000000536F6D652070726F626C656D206590
:103610006E636F756E74657265642C205A2D6C65CF
:1036200076656C696E6720656E666F72636564208F
:103630002E2E2E0001004D65736820626564206C9B
:103640006576656C696E67206661696C65642E20BD
:103650005072696E742063616E63656C65642E00E0
:10366000020048656174696E672064697361626C09
:103670006564206279207361666574792074696D70
:1036800065722E000300472D636F646520736C69BB
:1036900063656420666F7220612064696666657286
:1036A000656E74206C6576656C2E20436F6E746950
:1036B0006E75653F000400472D636F646520736C71
:1036C0006963656420666F7220612064696666655F
:1036D00072656E74206C6576656C2E20506C656129
:1036E00073652072652D736C69636520746865204D
:1036F0006D6F64656C20616761696E2E2050726920
:103700006E742063616E63656C6C65642E000500E9
:10371000472D636F646520736C6963656420666F11
:10372000722061206E65776572206669726D7761BF
:1037300072652E20436F6E74696E75653F000600DA
:10374000472D636F646520736C6963656420666FE1
:10375000722061206E65776572206669726D77618F
:1037600072652E20506C656173652075706461749C
:103770006520746865206669726D776172652E20B8
:103780005072696E742063616E63656C6C65642E43
:10379000000700472D636F646520736C696365647F
:1037A00020666F72206120646966666572656E745A
:1037B000207072696E74657220747970652E204372
:1037C0006F6E74696E75653F000800472D636F6406
:1037D0006520736C6963656420666F722061206484
:1037E0006966666572656E74207072696E74657262
:1037F00020747970652E20506C6561736520726548
:103800002D736C69636520746865206D6F64656CE9
:1038100020616761696E2E205072696E7420636149
:103820006E63656C6C65642E00090050726573737D
:1038300020746865206B6E6F6220746F20707265F3
:1038400068656174206E6F7A7A6C6520616E6420A1
:10385000636F6E74696E75652E000A00506C656149
:10386000736520707265737320746865206B6E6F6A
:103870006220746F20756E6C6F61642066696C6184
:103880006D656E74000B00616E64207072657373F9
:1038900020746865206B6E6F62000C00496E736562
:1038A00072742066696C616D656E74000D00436F03
:1038B0006C6F72206E6F7420636F72726563740038
:1038C0000E0046696C616D656E74206E6F74206CBD
:1038D0006F61646564000F004368616E6765642012
:1038E000636F72726563746C790010004C6F616471
:1038F000696E6720636F6C6F720011004368616EC0
:103900006765207375636365737321001200506CE3
:1039100065617365206F70656E2069646C657220E7
:10392000616E642072656D6F76652066696C616D8D
:10393000656E74206D616E75616C6C792E0013007C
:103940005761732066696C616D656E7420756E6C6D
:103950006F6164207375636365737366756C3F0094
:103960001400506C656173652075706772616465E1
:103970002E0015004E6577206669726D776172655D
:103980002076657273696F6E20617661696C616221
:103990006C653A00160057616974696E6720666F3E
:1039A000722050494E44412070726F626520636FEF
:1039B0006F6C696E67001700506C656173652077E6
:1039C0006169740018004E6F206D6F76652E0019C6
:1039D000005761697420666F7220757365722E2EB0
:1039E0002E001A00537461626C6520616D62696516
:1039F0006E742074656D70657261747572652032C5
:103A0000312D323643206973206E6565646564200C
:103A100061207269676964207374616E64206973E0
:103A20002072657175697265642E001B00506C65AB
:103A30006173652072756E2058595A2063616C69F4
:103A400062726174696F6E2066697273742E001CF5
:103A500000506C6561736520756E6C6F61642074D5
:103A600068652066696C616D656E74206669727345
:103A7000742C207468656E207265706561742074A2
:103A800068697320616374696F6E2E001D0043685E
:103A900065636B73001E004E6F7A7A6C6520642E2E
:103AA000001F00416C706861626574002000536FF4
:103AB000727400210054696D650022004E6F726DB2
:103AC000616C00230053442063617264002400533E
:103AD000656C656374206C616E6775616765002550
:103AE000004E6F7A7A6C65206368616E67650026A8
:103AF0000048572053657475700027004C6F61644F
:103B0000696E6720546573740028004469736162AC
:103B10006C652073746570706572730029004D6F59
:103B200076652061786973002A0054656D7065724E
:103B30006174757265002B0050494E4441206361E9
:103B40006C2E002C0052657365742058595A2063FE
:103B5000616C6962722E002D0053686F7720656E6C
:103B6000642073746F7073002E00504944206361A9
:103B70006C6962726174696F6E002F004265642027
:103B80006C6576656C20636F7272656374003000DB
:103B90004D65736820426564204C6576656C696E7E
:103BA0006700310043616C696272617465205A007C
:103BB000320043616C6962726174652058595A0021
:103BC000330053656C667465737400340057697A0A
:103BD00061726400350054657374696E67206669AC
:103BE0006C616D656E740036004C6F616420416CD1
:103BF0006C003700506C656173652070756C6C20CB
:103C00006F75742066696C616D656E7420696D6D89
:103C10006564696174656C79003800526573657418
:103C200000390052656E616D65003A004669727335
:103C300074206C617965722063616C2E003B0053C7
:103C4000656C656374003C00537465656C20736833
:103C500065657473003D00537570706F7274003E3B
:103C6000004661696C207374617473204D4D55007A
:103C70003F004661696C20737461747300400053A7
:103C800074617469737469637300410043616C69A2
:103C900062726174696F6E0042004175746F4C6F9F
:103CA00061642066696C616D656E740043004C6FE1
:103CB00061642066696C616D656E74004400556EC8
:103CC0006C6F61642066696C616D656E740045009F
:103CD0004C6F616420746F206E6F7A7A6C65004659
:103CE000005072656C6F616420746F204D4D5500FB
:103CF00047004E6F205344206361726400480050B7
:103D000072696E742066726F6D20534400490052D0
:103D10006573756D65207072696E74004A0050613C
:103D2000757365207072696E74004B005365742062
:103D30005265616479004C00536574206E6F742085
:103D40005265616479004D00507265686561740068
:103D50004E0054756E65004F004C697665206164B5
:103D60006A757374205A00500052657072696E74DF
:103D7000005100496E666F2073637265656E005274
:103D8000004173736973740053004F6E6365005490
:103D900000536F756E640055004C6F7564005600DB
:103DA00046696C2E2073656E736F7200570043680E
:103DB000616E67652066696C616D656E74005800A0
:103DC000466C6F770059005370656564005A004D6A
:103DD00061676E65747320636F6D702E005B004EBB
:103DE0002F41005C005A2D70726F6265206E722E3A
:103DF000005D004D657368005E0053657474696E04
:103E00006773005F005965730060004E6F006100CA
:103E100053746F70207072696E740062004368653D
:103E2000636B696E672066696C6500630046696C48
:103E30006520696E636F6D706C6574652E20436FCD
:103E40006E74696E756520616E797761793F006483
:103E50000084526566726573680065004D61696E25
:103E600000660057616974696E6720666F72206E24
:103E70006F7A7A6C6520616E642062656420636F7E
:103E80006F6C696E6700670053656C6563742066CC
:103E9000696C616D656E743A00680053656C667498
:103EA000657374204F4B00690053656C66746573CD
:103EB00074207374617274006A0053776170706566
:103EC00064006B0046726F6E742F6C6566742066BA
:103ED000616E73006C0041786973006D0041786910
:103EE00073206C656E677468006E004C6F6F73654D
:103EF0002070756C6C6579006F00456E6473746F2B
:103F000070206E6F7420686974007000456E647371
:103F1000746F700071004D6F746F72007200456EA7
:103F20006473746F7073007300576972696E6720F1
:103F30006572726F720074004265642F4865617427
:103F400065720075004E6F7420636F6E6E656374EA
:103F500065640076004865617465722F5468657207
:103F60006D6973746F72007700506C6561736520C2
:103F7000636865636B3A00780053656C66746573BB
:103F800074206572726F722100790046696C616DF0
:103F9000656E742073656E736F72007A005072697B
:103FA0006E742066616E3A007B00486F74656E64C3
:103FB0002066616E3A007C0043616C6962726174D4
:103FC000696E6720686F6D65007D0053656C66746F
:103FD000657374206661696C6564007E00416C6C79
:103FE00020636F7272656374007F00436865636B62
:103FF000696E672073656E736F727300800043682B
:1040000065636B696E6720686F74656E640081001C
:10401000436865636B696E67206265640082004374
:104020006865636B696E67205A20617869730083E5
:1040300000436865636B696E672059206178697316
:10404000008400436865636B696E6720582061785F
:104050006973008500436865636B696E6720656EF0
:104060006473746F707300860043617264207265BC
:104070006D6F7665640087004261636B0088004164
:1040800075746F20706F77657200890053696C6575
:104090006E74008A004D6F6465008B004869676824
:1040A00020706F776572008C0053747269637400BE
:1040B0008D005761726E008E004E6F6E65008F002E
:1040C000486F74656E64206174203238304321205B
:1040D0004E6F7A7A6C65206368616E6765642061F3
:1040E0006E64207469676874656E656420746F20FF
:1040F00073706563733F009000466F722061204EBD
:104100006F7A7A6C65206368616E676520706C6594
:1041100061736520726561640A70727573612E69DE
:104120006F2F6E6F7A7A6C652D6D6B337300910013
:104130005049442063616C2E2066696E697368651E
:10414000640092005049442063616C2E009300503B
:1041500072696E74207061757365640094005072AA
:10416000696E742061626F72746564009500436FBC
:1041700070792073656C6563746564206C616E672B
:10418000756167653F0096004E6F7A7A6C652064B2
:1041900069616D6574657220646966666572732015
:1041A00066726F6D2074686520472D636F64652E9D
:1041B00020436F6E74696E75653F0097004E6F7A8D
:1041C0007A6C65206469616D6574657220646966E6
:1041D000666572732066726F6D2074686520472D66
:1041E000636F64652E20506C65617365206368653C
:1041F000636B207468652076616C756520696E203C
:1042000073657474696E67732E205072696E7420C2
:1042100063616E63656C6C65642E0098005468651C
:104220007265206973206E6F2066696C616D656EC2
:1042300074206C6F616465642E20436F6E74696EC8
:1042400075653F0099005468657265206973206E3A
:104250006F2066696C616D656E74206C6F6164655A
:10426000642E205072696E742063616E63656C6C9D
:1042700065642E009A005468657265206973207326
:1042800074696C6C2061206E65656420746F206DAC
:10429000616B65205A2063616C6962726174696F39
:1042A0006E2E20506C6561736520666F6C6C6F7745
:1042B00020746865206D616E75616C2C2063686187
:1042C00070746572204669727374207374657073BC
:1042D0002C2073656374696F6E2043616C69627230
:1042E0006174696F6E20666C6F772E009B00507250
:1042F000696E74657220686173206E6F74206265E8
:10430000656E2063616C69627261746564207965B1
:10431000742E20506C6561736520666F6C6C6F77CE
:1043200020746865206D616E75616C2C2063686116
:10433000707465722046697273742073746570734B
:104340002C2073656374696F6E2043616C696272BF
:104350006174696F6E20666C6F772E009C005365E8
:104360006C66746573742077696C6C20626520726A
:10437000756E20746F2063616C6962726174652070
:1043800061636375726174652073656E736F726CBF
:10439000657373207265686F6D696E672E009D008E
:1043A0004F6C642073657474696E677320666F75F3
:1043B0006E642E2044656661756C74205049442CEF
:1043C00020457374657073206574632E2077696C63
:1043D0006C206265207365742E009E005761726EBA
:1043E000696E673A20626F7468207072696E7465D6
:1043F00072207479706520616E64206D6F746865D9
:1044000072626F6172642074797065206368616E96
:104410006765642E009F005761726E696E673A206F
:104420007072696E7465722074797065206368615A
:104430006E6765642E00A0005761726E696E673A00
:10444000206D6F74686572626F6172642074797038
:1044500065206368616E6765642E00A1005368651E
:10446000657400A2004E6F74207370696E6E696E81
:104470006700A3005370696E6E696E6700A4004CFC
:1044800065667420686F74656E642066616E3F00B7
:10449000A50046726F6E74207072696E742066613A
:1044A0006E3F00A60046616E207465737400A7001D
:1044B00058595A2063616C6962726174696F6E2029
:1044C000616C6C2072696768742E20536B6577206D
:1044D00077696C6C20626520636F727265637465C6
:1044E00064206175746F6D61746963616C6C792EA1
:1044F00000A80058595A2063616C6962726174693E
:104500006F6E20616C6C2072696768742E20582F62
:104510005920617865732061726520736C696768E2
:10452000746C7920736B657765642E20476F6F64B8
:10453000206A6F622100A90058595A2063616C6992
:1045400062726174696F6E206F6B2E20582F592034
:1045500061786573206172652070657270656E6444
:104560006963756C61722E20436F6E67726174753A
:104570006C6174696F6E732100AA0058595A2063E8
:10458000616C6962726174696F6E20636F6D7072C5
:104590006F6D697365642E20526967687420667256
:1045A0006F6E742063616C6962726174696F6E20F2
:1045B000706F696E74206E6F7420726561636861DC
:1045C000626C652E00AB0058595A2063616C6962B9
:1045D000726174696F6E20636F6D70726F6D697355
:1045E00065642E2046726F6E742063616C6962721E
:1045F0006174696F6E20706F696E7473206E6F7472
:1046000020726561636861626C652E00AC00585968
:104610005A2063616C6962726174696F6E206661B1
:10462000696C65642E2052696768742066726F6ECB
:10463000742063616C6962726174696F6E20706F5F
:10464000696E74206E6F7420726561636861626C5C
:10465000652E00AD0058595A2063616C6962726121
:1046600074696F6E206661696C65642E2046726F96
:104670006E742063616C6962726174696F6E207020
:104680006F696E7473206E6F742072656163686108
:10469000626C652E00AE0058595A2063616C6962E5
:1046A000726174696F6E206661696C65642E20505A
:1046B0006C6561736520636F6E73756C74207468CC
:1046C00065206D616E75616C2E00AF0058595A20DF
:1046D00063616C6962726174696F6E206661696C96
:1046E00065642E204265642063616C696272617446
:1046F000696F6E20706F696E7420776173206E6FC2
:104700007420666F756E642E00B000506C65617326
:104710006520706C61636520737465656C207368D7
:10472000656574206F6E20686561746265642E0033
:10473000B10044697374616E636520626574776566
:10474000656E20746970206F6620746865206E6FD6
:104750007A7A6C6520616E64207468652062656495
:10476000207375726661636520686173206E6F7473
:10477000206265656E20736574207965742E205003
:104780006C6561736520666F6C6C6F77207468650B
:10479000206D616E75616C2C206368617074657248
:1047A0002046697273742073746570732C2073656E
:1047B0006374696F6E204669727374206C617965E9
:1047C000722063616C6962726174696F6E2E00B2EF
:1047D00000506C6163652061207368656574206FAB
:1047E0006620706170657220756E646572207468F1
:1047F00065206E6F7A7A6C6520647572696E6720C9
:104800007468652063616C6962726174696F6E209F
:104810006F66206669727374203420706F696E74DD
:10482000732E20496620746865206E6F7A7A6C65F5
:1048300020636174636865732074686520706170BB
:1048400065722C20706F776572206F6666207468C1
:1048500065207072696E74657220696D6D6564693A
:104860006174656C792E00B3005365617263686989
:104870006E67206265642063616C6962726174694D
:104880006F6E20706F696E7400B4004D6561737552
:1048900072696E67207265666572656E6365206811
:1048A0006569676874206F662063616C6962726114
:1048B00074696F6E20706F696E7400B500506C651E
:1048C00061736520636C65616E20746865206E6F2E
:1048D0007A7A6C6520666F722063616C69627261BE
:1048E00074696F6E2E20436C69636B207768656E08
:1048F00020646F6E652E00B6004175746F20686F7E
:104900006D6500B700526573756D696E67207072D2
:10491000696E7400B80050494E4441204865617486
:10492000696E6700B90043616C6962726174696F96
:104930006E20646F6E6500BA0043616C69627261DB
:1049400074696E67205A00BB0042656420646F6E14
:104950006500BC004265642048656174696E67004B
:10496000BD0048656174696E6720646F6E652E00D6
:10497000BE0048656174696E6700BF00546F746162
:104980006C00C0004C617374207072696E7400C159
:10499000004D4D55206661696C7300C2004D4D5548
:1049A000206C6F6164206661696C7300C3004D4DBB
:1049B0005520706F776572206661696C7300C40062
:1049C0004D6174657269616C206368616E676573BF
:1049D00000C5004C617374207072696E742066614A
:1049E000696C7572657300C600546F74616C2066E3
:1049F00061696C7572657300C70046696C2E207220
:104A0000756E6F75747300C80054656D7065726162
:104A1000747572657300C90053656E736F72206997
:104A20006E666F00CA00457874727564657220699D
:104A30006E666F00CB0058595A2063616C2E20645B
:104A4000657461696C7300CC005072696E74657234
:104A500020495020416464723A00CD00756E6B6E3F
:104A60006F776E00CE004D4D5520636F6E6E65639F
:104A700074656400CF00446174653A00D000746FBF
:104A800020756E6C6F61642066696C616D656E7413
:104A900000D100746F206C6F61642066696C616D79
:104AA000656E7400D200507265737320746865205F
:104AB0006B6E6F6200D30050726568656174696ED9
:104AC0006720746F2063757400D400507265686548
:104AD0006174696E6720746F20656A65637400D5C0
:104AE0000050726568656174696E6720746F207527
:104AF0006E6C6F616400D6005072656865617469A0
:104B00006E6720746F206C6F616400D700436F6F15
:104B10006C646F776E00D80046696C616D656E7469
:104B200020657874727564696E67202620776974D1
:104B30006820636F727265637420636F6C6F723F7D
:104B400000D900456A65637400DA004175746F6CC2
:104B50006F6164696E672066696C616D656E742053
:104B60006973206163746976652C206A757374209B
:104B7000707265737320746865206B6E6F6220615C
:104B80006E6420696E736572742066696C616D6510
:104B90006E742E2E2E00DB00546F74616C206669DB
:104BA0006C616D656E7400DC00546F74616C207014
:104BB00072696E742074696D6500DD0046696C6110
:104BC0006D656E74207573656400DE005072696EE9
:104BD000742074696D6500DF0050726568656174EA
:104BE00020746865206E6F7A7A6C652100E000455C
:104BF00052524F523A00E100592064697374616E59
:104C000063652066726F6D206D696E00E2004C6511
:104C1000667400E300526967687400E4004D6561E2
:104C2000737572656420736B657700E500536C697A
:104C300067687420736B657700E60053657665726C
:104C40006520736B657700E7005B303B305D20705B
:104C50006F696E74206F666673657400E800416466
:104C60006A757374696E67205A00E9005265617253
:104C70002073696465205BE46D5D00EA0046726F35
:104C80006E7420736964655BE46D5D00EB005269CE
:104C900067687420736964655BE46D5D00EC004CCB
:104CA0006566742073696465205BE46D5D00ED00EA
:104CB0005365742074656D70657261747572653AC0
:104CC00000EE00417265206C65667420616E6420A0
:104CD0007269676874205A2D6361727269616765D1
:104CE0007320616C6C2075703F00EF0043616C694C
:104CF00062726174696E672058595A2E20526F741F
:104D000061746520746865206B6E6F6220746F201B
:104D10006D6F766520746865205A206361727269D0
:104D200061676520757020746F2074686520656EFA
:104D3000642073746F70706572732E20436C6963A6
:104D40006B207768656E20646F6E652E00F00043FF
:104D5000616C6962726174696E67205A2E20526FAD
:104D60007461746520746865206B6E6F6220746F67
:104D7000206D6F766520746865205A2063617272B9
:104D80006961676520757020746F2074686520659F
:104D90006E642073746F70706572732E20436C693B
:104DA000636B207768656E20646F6E652E00F1007E
:104DB00050494E44412063616C6962726174696F4D
:104DC0006E206661696C656400F20050494E444192
:104DD0002063616C6962726174696F6E206973200F
:104DE00066696E697368656420616E6420616374CE
:104DF0006976652E2049742063616E2062652064A7
:104E0000697361626C656420696E206D656E7520E2
:104E100053657474696E67732D3E50494E4441204A
:104E200063616C2E00F300457874727564657200DE
:104E3000F4004D6F7665205A00F5004D6F766520C1
:104E40005900F6004D6F7665205800F700536865ED
:104E5000657420252E37730A5A206F666673657451
:104E60003A20252B312E33666D6D0A2563436F6E14
:104E700074696E75650A2563526573657400F80080
:104E8000506C65617365206C6F61642066696C614C
:104E90006D656E742066697273742E00F9003E436E
:104EA000616E63656C00FA0052756E6E696E672004
:104EB00057697A6172642077696C6C2064656C65EF
:104EC00074652063757272656E742063616C6962CB
:104ED000726174696F6E20726573756C7473206192
:104EE0006E642073746172742066726F6D207468D2
:104EF0006520626567696E6E696E672E20436F6E0E
:104F000074696E75653F00FB005072656865617479
:104F1000696E67206E6F7A7A6C652E20506C6561C1
:104F2000736520776169742E00FC00506C656173B5
:104F30006520696E736572742066696C616D656E5B
:104F40007420696E746F207468652065787472755A
:104F50006465722C207468656E20707265737320AE
:104F6000746865206B6E6F6220746F206C6F616473
:104F70002069742E00FD00506C6561736520696EB8
:104F8000736572742066696C616D656E7420696EFC
:104F9000746F20746865206669727374207475621A
:104FA00065206F6620746865204D4D552C2074680F
:104FB000656E20707265737320746865206B6E6F08
:104FC0006220746F206C6F61642069742E00FE0093
:104FD000546865207072696E7465722077696C6CB4
:104FE000207374617274207072696E74696E6720C8
:104FF00061207A69672D7A6167206C696E652E2061
:10500000526F7461746520746865206B6E6F6220E6
:10501000756E74696C20796F7520726561636820A4
:10502000746865206F7074696D616C20686569676C
:1050300068742E20436865636B207468652070690E
:1050400063747572657320696E2074686520686189
:105050006E64626F6F6B202843616C696272617469
:10506000696F6E2063686170746572292E00FF009D
:1050700053656C6563742074656D706572617475D9
:105080007265207768696368206D61746368657311
:1050900020796F7572206D6174657269616C2E0084
:1050A000000153656C65637420612066696C616DF5
:1050B000656E7420666F722074686520466972732D
:1050C00074204C617965722043616C69627261740D
:1050D000696F6E20616E642073656C65637420690E
:1050E0007420696E20746865206F6E2D736372651D
:1050F000656E206D656E752E0001014E6F7720493B
:105100002077696C6C2063616C69627261746520E0
:1051100064697374616E6365206265747765656E3A
:1051200020746970206F6620746865206E6F7A7ACB
:105130006C6520616E6420686561746265642073CB
:105140007572666163652E0002015A2063616C69A5
:1051500062726174696F6E207265636F6D6D656EEA
:105160006465642E2052756E206974206E6F773FDF
:10517000000301506C656173652072656D6F766523
:1051800020737465656C2073686565742066726F42
:105190006D20686561746265642E000401497320A6
:1051A000737465656C207368656574206F6E206824
:1051B0006561746265643F000501506C65617365EB
:1051C00020636865636B206F75722068616E64622E
:1051D0006F6F6B20616E642066697820746865204B
:1051E00070726F626C656D2E205468656E207265FA
:1051F00073756D65207468652057697A61726420E3
:105200006279207265626F6F74696E672074686579
:10521000207072696E7465722E000601416C6C20FC
:10522000697320646F6E652E2048617070792070FC
:1052300072696E74696E6721000701596F7520638A
:10524000616E20616C7761797320726573756D652D
:10525000207468652057697A6172642066726F6D88
:105260002043616C6962726174696F6E202D3E200B
:1052700057697A6172642E000801496620796F755A
:105280002068617665206164646974696F6E616C21
:1052900020737465656C207368656574732C206376
:1052A000616C6962726174652074686569722070EE
:1052B00072657365747320696E2053657474696ECA
:1052C0006773202D204857205365747570202D205A
:1052D000537465656C207368656574732E000901ED
:1052E000506C6561736520636C65616E20686561F3
:1052F0007462656420616E64207468656E207072EB
:1053000065737320746865206B6E6F622E000A01EE
:10531000446F20796F752077616E7420746F2072EE
:105320006570656174206C6173742073746570209E
:10533000746F20726561646A757374206469737434
:10534000616E6365206265747765656E206E6F7A45
:105350007A6C6520616E6420686561746265643F83
:10536000000B0153656C656374206E6F7A7A6C650F
:1053700020707265686561742074656D7065726116
:1053800074757265207768696368206D61746368FD
:10539000657320796F7572206D6174657269616CD7
:1053A0002E000C0149732066696C616D656E742076
:1053B0006C6F616465643F000D014E6F772049207A
:1053C00077696C6C2070726568656174206E6F7AA5
:1053D0007A6C6520666F7220504C412E000E014998
:1053E0002077696C6C2072756E207A2063616C691D
:1053F00062726174696F6E206E6F772E000F014EBE
:105400006F772072656D6F766520746865207465AE
:105410007374207072696E742066726F6D2073747D
:1054200065656C2073686565742E001001506C65AD
:105430006173652072656D6F766520736869707041
:10544000696E672068656C70657273206669727337
:10545000742E001101492077696C6C2072756E20E2
:1054600078797A2063616C6962726174696F6E2009
:105470006E6F772E2049742077696C6C2074616B95
:105480006520757020746F203234206D696E732E24
:1054900000120146697273742C20492077696C6C84
:1054A0002072756E207468652073656C6674657310
:1054B0007420746F20636865636B206D6F73742054
:1054C000636F6D6D6F6E20617373656D626C7920B3
:1054D00070726F626C656D732E00130148692C2029
:1054E0004920616D20796F7572204F726967696E0E
:1054F000616C205072757361206933207072696E1F
:105500007465722E20576F756C6420796F75206CEE
:10551000696B65206D6520746F206775696465200F
:10552000796F75207468726F75676820746865207C
:1055300073657475702070726F636573733F0014C8
:105540000148692C204920616D20796F7572204FC8
:10555000726967696E616C2050727573612069337E
:10556000207072696E7465722E20492077696C6CA8
:1055700020677569646520796F75207468726F752E
:10558000676820612073686F72742073657475702A
:105590002070726F636573732C20696E2077686961
:1055A000636820746865205A2D6178697320776973
:1055B0006C6C2062652063616C6962726174656401
:1055C0002E205468656E2C20796F752077696C6C7D
:1055D00020626520726561647920746F2070726941
:1055E0006E742E00150150617573650016014653E7
:1055F00020416374696F6E001701436F6E742E0053
:105600001801462E206175746F6C6F61640019017A
:10561000462E2072756E6F7574001A01437574748E
:105620006572001B0146616E207370656564001C25
:1056300001426564001D0146616E73206368656305
:105640006B001E014D6F64656C001F014E6F7A7A0E
:105650006C6500200146656564696E6720746F2083
:105660004653656E736F720021014D6F76696E67E8
:105670002073656C6563746F72002201486F6D69F9
:105680006E67002301526574726163742066726FE5
:105690006D2046494E4441002401456A65637469A2
:1056A0006E672066696C616D656E740025015061DE
:1056B000726B696E672073656C6563746F72002628
:1056C0000152657475726E696E672073656C6563EF
:1056D000746F72002701506572666F726D696E6734
:1056E0002063757400280150757368696E672066C1
:1056F000696C616D656E740029015072657061722C
:10570000696E6720626C616465002A0153656C658F
:105710006374696E672066696C2E20736C6F740009
:105720002B01556E6C6F6164696E672066696C61F0
:105730006D656E74002C0145525220544D43206615
:1057400061696C6564002D014552522048656C709A
:105750002066696C616D656E74002E0145525220A1
:10576000496E7465726E616C002F0145525220576C
:1057700061697420666F722055736572003001464E
:10578000696E697368696E67206D6F76656D656EA9
:10579000747300310141766F6964696E67206772C6
:1057A000696E6400320146656564696E6720746FD6
:1057B000206E6F7A7A6C6500330146656564696EA8
:1057C0006720746F206578747275646572003401A7
:1057D00046656564696E6720746F2046494E444192
:1057E000003501556E6C6F6164696E6720746F20BF
:1057F00070756C6C6579003601556E6C6F6164690B
:105800006E6720746F2046494E4441003701446959
:1058100073656E676167696E672069646C657200A5
:105820003801456E676167696E672069646C6572EF
:105830000039014F4B003A01554E4B4E4F574E2009
:105840004552524F52003B0146494C414D454E5442
:10585000204348414E4745003C0146494C414D4597
:105860004E5420454A4543544544003D01554E4C55
:105870004F4144204D414E55414C4C59003E01464C
:10588000572052554E54494D45204552524F5200D3
:105890003F014D4D55204657205550444154452019
:1058A0004E45454445440040015155455545204627
:1058B000554C4C004101494E56414C494420544FEF
:1058C0004F4C00420146494C2E20414C5245414428
:1058D00059204C4F41444544004301434F4D4D55E1
:1058E0004E49434154494F4E204552524F52004475
:1058F000014D4D55204E4F5420524553504F4E446C
:10590000494E470045014D4D55204D4355204552C8
:10591000524F520046014D4D552053454C4654457B
:105920005354204641494C4544004701544D4320BF
:105930004452495645522053484F5254454400481A
:1059400001544D4320554E444552564F4C54414707
:105950004520455252004901544D43204452495676
:105960004552205245534554004A01544D4320446A
:105970005249564552204552524F52004B01544D08
:1059800043204F56455248454154204552524F52AC
:10599000004C015741524E494E4720544D4320542C
:1059A0004F4F20484F54004D0149444C455220432D
:1059B000414E4E4F54204D4F5645004E0149444CE8
:1059C00045522043414E4E4F5420484F4D45004FC5
:1059D0000153454C4543544F522043414E4E4F5482
:1059E000204D4F564500500153454C4543544F52AE
:1059F0002043414E4E4F5420484F4D450051014CDD
:105A00004F414420544F20455854522E204641497E
:105A10004C4544005201494E535045435420464999
:105A20004E44410053014653454E534F5220544F6C
:105A30004F204541524C5900540150554C4C45594A
:105A40002043414E4E4F54204D4F56450055014680
:105A500053454E534F522046494C2E2053545543E4
:105A60004B0056014653454E534F52204449444E35
:105A7000542054524947472E00570146494E44414D
:105A80002046494C414D2E20535455434B0058015C
:105A900046494E4441204449444E542054524947BB
:105AA0004745520059014375742066696C616D6504
:105AB0006E74005A01456A6563742066726F6D20CA
:105AC0004D4D55005B014C6F6164696E67206669DE
:105AD0006C616D656E74005C014D4D5520526574AE
:105AE00072793A20526573746F72696E67207465BB
:105AF0006D70657261747572652E2E2E005D015396
:105B00006F7274696E672066696C6573005E01531D
:105B10006F6D652066696C65732077696C6C206EAB
:105B20006F7420626520736F727465642E204D61FE
:105B3000782E204E6F2E206F662066696C6573206C
:105B4000696E203120666F6C64657220666F72200A
:105B5000736F7274696E67206973203130302E0064
:105B60005F0153544F505045442E0060014F66660C
:105B70000061014F6E006201556E65787065637457
:105B80006564206572726F72206F636375727265EF
:105B9000642E0063014D3630302046696C616D65BE
:105BA0006E74204368616E67652E204C6F616420BF
:105BB00061206E65772066696C616D656E74206F1B
:105BC0007220656A65637420746865206F6C642058
:105BD0006F6E652E00640152656D6F766520746886
:105BE0006520656A65637465642066696C616D65CE
:105BF0006E742066726F6D207468652066726F6EB9
:105C000074206F6620746865204D4D552E00650127
:105C100046696C616D656E74206465746563746556
:105C20006420756E65787065637465646C792E2088
:105C3000456E73757265206E6F2066696C616D6567
:105C40006E74206973206C6F616465642E204368F4
:105C500065636B207468652073656E736F72732063
:105C6000616E6420776972696E672E006601496E05
:105C70007465726E616C2072756E74696D652065F5
:105C800072726F722E20547279207265736574740B
:105C9000696E6720746865204D4D55206F722075C0
:105CA00070646174696E6720746865206669726DDE
:105CB000776172652E0067014D4D5520465720765D
:105CC000657273696F6E20697320696E636F6D70A2
:105CD000617469626C652077697468207072696E9E
:105CE0007465722046572E55706461746520746F18
:105CF0002076657273696F6E20332E302E332E003E
:105D000068014D4D55204669726D77617265206955
:105D10006E7465726E616C206572726F722C207089
:105D20006C656173652072657365742074686520A5
:105D30004D4D552E0069015265717565737465642A
:105D40002066696C616D656E7420746F6F6C20697C
:105D500073206E6F7420617661696C61626C65207E
:105D60006F6E207468697320686172647761726510
:105D70002E20436865636B2074686520472D636F30
:105D8000646520666F7220746F6F6C20696E646545
:105D900078206F7574206F662072616E67652028A9
:105DA00054302D5434292E006A0143616E6E6F7495
:105DB00020706572666F726D20746865206163740F
:105DC000696F6E2C2066696C616D656E74206973F5
:105DD00020616C7265616479206C6F616465642E0A
:105DE00020556E6C6F6164206974206669727374EB
:105DF0002E006B014D4D55206E6F742072657370CF
:105E00006F6E64696E6720636F72726563746C791C
:105E10002E20436865636B2074686520776972691A
:105E20006E6720616E6420636F6E6E6563746F725F
:105E3000732E006C014D4D55206E6F74207265738A
:105E4000706F6E64696E672E20436865636B2074A3
:105E5000686520776972696E6720616E6420636F80
:105E60006E6E6563746F72732E006D014D6F726597
:105E70002064657461696C73206F6E6C696E652E49
:105E8000006E015468652049646C65722063616E20
:105E90006E6F7420686F6D652070726F7065726CC4
:105EA000792E20436865636B20666F7220616E797E
:105EB0007468696E6720626C6F636B696E672069D6
:105EC0007473206D6F76656D656E742E006F01437F
:105ED000616E2774206D6F76652053656C65637401
:105EE0006F72206F722049646C65722E00700154CD
:105EF00068652053656C6563746F722063616E6EB4
:105F00006F7420686F6D652070726F7065726C7948
:105F10002E20436865636B20666F7220616E797412
:105F200068696E6720626C6F636B696E6720697465
:105F300073206D6F76656D656E742E0071014C6F08
:105F40006164696E6720746F20657874727564652A
:105F500072206661696C65642E20496E737065639A
:105F600074207468652066696C616D656E74207458
:105F700069702073686170652E20526566696E6570
:105F8000207468652073656E736F722063616C693D
:105F900062726174696F6E2C206966206E6565643B
:105FA00065642E00720153656C6563746F722063C3
:105FB000616E2774206D6F76652064756520746F3F
:105FC0002046494E444120646574656374696E6778
:105FD00020612066696C616D656E742E204D616B69
:105FE000652073757265206E6F2066696C616D65E2
:105FF0006E7420697320696E2053656C6563746FDD
:106000007220616E642046494E444120776F726B66
:10601000732070726F7065726C792E00730146691F
:106020006C616D656E742073656E736F722074722F
:106030006967676572656420746F6F206561726C53
:1060400079207768696C65206C6F6164696E672080
:10605000746F2065787472756465722E204368656C
:10606000636B2074686572652069736E27742061A4
:106070006E797468696E6720737475636B20696EDE
:10608000205054464520747562652E204368656330
:106090006B20746861742073656E736F7220726513
:1060A0006164732070726F7065726C792E00740178
:1060B00050756C6C6579206D6F746F7220737461AC
:1060C0006C6C65642E20456E73757265207468650E
:1060D0002070756C6C65792063616E206D6F7665DC
:1060E00020616E6420636865636B20746865207747
:1060F0006972696E672E00750146696C616D656E27
:10610000742073656E736F72206469646E277420E7
:10611000737769746368206F6666207768696C6559
:1061200020756E6C6F6164696E672066696C616D65
:10613000656E742E20456E737572652066696C619C
:106140006D656E742063616E206D6F766520616E83
:1061500064207468652073656E736F7220776F7248
:106160006B732E00760146696C616D656E742073E9
:10617000656E736F72206469646E2774207472692F
:1061800067676572207768696C65206C6F61646908
:106190006E67207468652066696C616D656E742E2B
:1061A00020456E73757265207468652073656E7323
:1061B0006F722069732063616C69627261746564D7
:1061C00020616E64207468652066696C616D656E1F
:1061D0007420726561636865642069742E007701BC
:1061E00046494E4441206469646E27742073776980
:1061F000746368206F6666207768696C6520756EC9
:106200006C6F6164696E672066696C616D656E7440
:106210002E2054727920756E6C6F6164696E6720F0
:106220006D616E75616C6C792E20456E737572654B
:106230002066696C616D656E742063616E206D6FA0
:10624000766520616E642046494E444120776F7226
:106250006B732E00780146494E4441206469646E98
:1062600027742074726967676572207768696C6546
:10627000206C6F6164696E67207468652066696C64
:10628000616D656E742E20456E737572652074683D
:10629000652066696C616D656E742063616E206D4A
:1062A0006F766520616E642046494E444120776FC9
:1062B000726B732E00790144697361626C65007AB8
:1062C0000153746F70007B014C6F6164007C015559
:1062D0006E6C6F6164007D0152657365744D4D5540
:1062E000007E015265747279007F01426564206C02
:1062F0006576656C696E67206661696C65642E20E1
:1063000053656E736F72206469646E2774207472B3
:1063100069676765722E20446562726973206F6ECB
:10632000206E6F7A7A6C653F2057616974696E6779
:1063300020666F722072657365742E00800153654C
:106340006E7369746976697479008101446F6E6552
:1063500000656E717565696E67202200446F6E6519
:10636000207072696E74696E672066696C65004E94
:106370006F204C696E65204E756D6265722077697D
:10638000746820636865636B73756D2C204C617352
:1063900074204C696E653A20004E6F204368656337
:1063A0006B73756D2077697468206C696E65206EFB
:1063B000756D6265722C204C617374204C696E653A
:1063C0003A2000636865636B73756D206D69736D4A
:1063D000617463682C204C617374204C696E653A5B
:1063E00020004C696E65204E756D62657220697380
:1063F000206E6F74204C617374204C696E65204E62
:10640000756D6265722B312C204C617374204C6960
:106410006E653A2000257520627974657320777265
:10642000697474656E20746F202553206174206137
:10643000646472657373203078253038780A0044BC
:106440002564202D20526561642F57726974652080
:1064500025530A003F3F00526F6D616E6100487224
:10646000766174736B69004D616779617200536C7A
:106470006F76656E63696E61004E6F72736B005369
:1064800076656E736B61004E656465726C616E64F7
:106490007300506F6C736B69004974616C69616E55
:1064A0006F004672616E6361697300457370616E5F
:1064B0006F6C004465757473636800436573746939
:1064C0006E6100456E676C6973680020436F756E7E
:1064D0007420583A200045303A25642052504D200F
:1064E00050524E313A25642052504D204530403AAA
:1064F00025752050524E31403A25750A0052657379
:10650000656E640025533A20256C640A25530A0001
:106510002F2F616374696F6E3A6E6F746966696379
:106520006174696F6E2025530A0046696C616D6560
:106530006E742072756E6F75742064657465637413
:106540006564210064697361626C656400656E61F5
:10655000626C656400454550524F4D005352414DA9
:1065600000442D31202D20456E646C657373206CC2
:106570006F6F700A004163746976652045787472A4
:10658000756465723A203000496E76616C696420EA
:106590006578747275646572004D3232302053250F
:1065A00064005344207072696E74696E672062796A
:1065B00074652000257500556E6B6E6F776E2063D5
:1065C0006F6D6D616E643A2022004D32303020498B
:1065D0006E76616C6964206578747275646572208A
:1065E000007A5F6D61783A20007A5F6D696E3A20BB
:1065F00000795F6D696E3A20005452494747455211
:106600004544006F70656E00785F6D696E3A2000DA
:106610005265706F7274696E6720656E6473746F13
:106620007020737461747573004D31313220636171
:106630006C6C65642E20456D657267656E637920AC
:1066400053746F702E002F2F616374696F6E3A75EB
:10665000766C6F5F7265636F766572795F72656184
:1066600064790053494C454E54004E4F524D414CB5
:10667000002553204D4F44453A2050657263656EA6
:106680007420646F6E653A20256868643B207072E0
:10669000696E742074696D652072656D61696E69DB
:1066A0006E6720696E206D696E733A2025643B2009
:1066B0004368616E676520696E206D696E733A206C
:1066C00025640A005072696E746572537461746552
:1066D0003A2025640A00456E642066696C65206C6A
:1066E00069737400426567696E2066696C65206C29
:1066F00069737400556E6B6E6F776E20256320632F
:106700006F64653A2025730A000A50494E444120BF
:1067100074656D70657261747572653A20252E31ED
:1067200066205A20736869667420286D6D293A20A6
:10673000252E3366000A537465703A2025642F367F
:106740000A000A537465703A2025642F3620287396
:106750006B6970706564290A50494E444120746524
:106760006D70657261747572653A202564205A20D7
:10677000736869667420286D6D293A300A000A5AD8
:1067800045524F3A20252E33660A007374617274A5
:106790002074656D70657261747572653A20252E7E
:1067A00031660A0025642020252E326600255320FC
:1067B000583A20252E356620593A20252E35662058
:1067C0005A3A20252E35660A00536C6565702E2EC8
:1067D0002E0045303A25642052504D0A50524E301A
:1067E0003A25642052504D0A004D31303700537520
:1067F00070657250494E44410048426564206F6E96
:10680000206C6F616400466C617368416972004579
:1068100072723A484F54454E442046414E204552EC
:10682000524F52002F2F616374696F6E3A72657315
:10683000756D6564002F2F616374696F6E3A7265C0
:1068400073756D65002F2F616374696F6E3A7265A1
:10685000616479002F2F616374696F6E3A6E6F7493
:106860005F7265616479002F2F616374696F6E3A9E
:1068700063616E63656C004F4B004C43442073743E
:1068800061747573206368616E67656400534420AA
:10689000636172642072656C6561736564002F2F9B
:1068A000616374696F6E3A7374617274004D383449
:1068B000004D373032004732382057004D353030E8
:1068C0000042616420696E7465727275707400575D
:1068D00061746368646F672074696D656F757400B7
:1068E000537461746963206D656D6F72792068619E
:1068F000730A6265656E206F76657277726974746B
:10690000656E004649524D5741524520435241530E
:1069100048210A437261736820726561736F6E3A31
:106920000A002020506C616E6E6572427566666565
:106930007242797465733A20002046726565204D75
:10694000656D6F72793A2000207C20417574686F04
:10695000723A2000204C6173742055706461746534
:10696000643A200020536F66747761726520526527
:1069700073657400205761746368646F67205265A3
:10698000736574002042726F776E206F75742052A9
:1069900065736574002045787465726E616C205271
:1069A0006573657400506F7765725570006572721B
:1069B0006F722077726974696E6720746F206669E0
:1069C0006C6500446F6E6520736176696E67206642
:1069D000696C652E006F6B0046696C616D656E7445
:1069E000004D6561737572656420736B6577733AEA
:1069F0002025662025660A0046697474696E672042
:106A00006661696C6564203D3E2063616C696272F9
:106A10006174696F6E206661696C65642E0A00435B
:106A2000616C6962726174696F6E2073756363650E
:106A300073732E0A00416C6C20342063616C6962B0
:106A4000726174696F6E20706F696E747320666F07
:106A5000756E642E0A00312F3400312F3400312F2F
:106A600039004572723A5052494E542046414E20E8
:106A70004552524F520025632533642F256481000F
:106A80005A25362E32662563005A2020202D2D2DC2
:106A90002000862533642525002D2D2D2525002554
:106AA0003364252500205344002020200020484F37
:106AB000002046524D2000872D2D3A2D2D202000FC
:106AC0008725337568202563256300872530327557
:106AD0003A2530327525632563002F2F6163746971
:106AE0006F6E3A706175736564002F2F616374690E
:106AF0006F6E3A70617573650044756D7020746FC8
:106B00002073657269616C0068656C702E707275B7
:106B1000736133642E636F6D00666F72756D2E70D6
:106B20007275736133642E636F6D0070727573617B
:106B300033642E636F6D004D3730310025533A0AB0
:106B40002531382E32666D200A25533A0A25313018
:106B50006C646420253032646820253032646D0016
:106B600025533A0A2531382E32666D200A25533ACC
:106B70000A2531306C646820253032646D20253060
:106B80003264730025362E32666D6D0025530A255A
:106B9000530A25533A0A25533A0025332E3266818B
:106BA00000252D31342E3134533A0A25530A252D30
:106BB00031342E3134533A25332E3266810A252D55
:106BC00031342E3134533A25332E32668100202061
:106BD00030002020310046494E44410050494E4487
:106BE000410057697A61726420656E642073746134
:106BF00074653A2025640A0053706F6F6C4A6F69A0
:106C00006E004669726D77617265005072757361CE
:106C1000206933204D4B322E3553204F4B2E004DE3
:106C20003630300053442063617264206F6B006F14
:106C300070656E526F6F74206661696C6564007672
:106C40006F6C756D652E696E6974206661696C651F
:106C50006400534420696E6974206661696C006F3A
:106C600070656E206661696C65642C2046696C6590
:106C70003A200043616E6E6F7420656E74657220F9
:106C80007375626469723A20004D3234004D3233BC
:106C9000202573005072696E7465722073746F7072
:106CA0007065642064756520746F206572726F7200
:106CB000732E205375706572766973696F6E2072DA
:106CC000657175697265642E0047312045252D2E4A
:106CD0003366204632373030004D383300312F399B
:106CE00000880020746F6F206C6F6E672065787469
:106CF000727573696F6E2070726576656E74656407
:106D00000020636F6C6420657874727573696F6EB0
:106D10002070726576656E746564004D6F766520CF
:106D200061626F7274656400084AD73B3BCE016EA6
:106D300084BCBFFDC12F3D6C74319ABD56833DDAD2
:106D40003D00C77F11BED9E4BB4C3E916BAAAABEE1
:106D5000000000803F05A84CCDB2D44EB93836A90A
:106D6000020C50B9918688083CA6AAAA2ABE000047
:106D700000803F07634236B79BD8A71A3968561878
:106D8000AEBAAB558C1D3CB7CC5763BD6DEDFD75F0
:106D90003EF6177231BF000000803F08000000BEC1
:106DA000922449123EABAAAA2ABECDCCCC4C3E00BE
:106DB000000080BEABAAAAAA3E00000000BF0000EF
:106DC00000803F0000000000084178D3BB4387D11A
:106DD000133D190E3CC3BD4282AD2B3E68EC82765A
:106DE000BED98FE1A93E4C80EFFFBE01C4FF7F3FBB
:106DF0000000000000000D94B7020C9433B30C9413
:106E00001BE30D9408300C94C3B00C94C5BA0C94D9
:106E10000CB50D94D61D0D94E0040D94D0060C9481
:106E2000CDB00C94C2C00D94842F0D9425650D94A3
:106E3000DC110C94AEB00D9491070C9411B50D9427
:106E4000E8040C94FAC30C947FBC0D94A5310D9406
:106E5000D9060D94843A0C944DB70C949DFC0C9477
:106E60008BBB0C94C7EA0D9471310C943DFE0C94CD
:106E700077B40D9494070D9405950D94FB310C9403
:106E8000EFB00C94E1FD0C948CB10D9468220C943D
:106E900064B50D940C310C9450FE0C947AFE0C9455
:106EA00007B50C9431C10C94E6C00C94356E0D946A
:106EB0001F2F0C948AE60C9468BC0C94C7B50D94F3
:106EC000BC010D94DB310D94EB310C94EDFD0D9470
:106ED000FC010C94B4B00C940AFF0C943FBA0C94CF
:106EE00089FC0C94DBB00C94EDF60C9445FC0D94ED
:106EF000A2310D94C7060C94E9B00D9474310C9432
:106F0000D4C00C94C3EA0C94A9B80C943EB30C946E
:106F100036C60C9459B40C942C6E0C942DE30C943E
:106F200090BC0C944EB50D949F6B0D944F110C9426
:106F30000F6C0C94DDF70C9416B50C9492B10D9473
:106F4000732F0C9493FC0C9488FE0C944AEF0C94D1
:106F5000C9B00C940EE80D94F3310C94F8FD0C9428
:106F6000CCC00C945EEF0C94F7B00C94A7FC0C947E
:106F7000CFBA0D94CB110D943E650D949D650C9484
:106F800050BC0C94CBEA0C94D85E0C9496FE0C94F6
:106F90001DC10C94FABA0C94C3FF0C9454E90D94DF
:106FA000AB310C94D7B00D943D6B0D9480650C946F
:106FB000F0C00C94086E0D94A4650D94E92E0D9408
:106FC000B46B0D940C010C94BFEA0D94DD300D945C
:106FD000B92F0D94E3310C94E5B00D94BB310C94B2
:106FE000DABB0D94A8310C94E7EF0C9444EA0C94AE
:106FF000BB6F0D94CE120C94C7FC0D94A66B0C9431
:10700000DBFC0C943CE30D94A52F0C94586E0D946E
:10701000092F0C94BDFC0D94230D0C94D4FE0C94FC
:107020003FEB0D9450020C94E1EA0D94ED040D94A5
:1070300051040D940C970C9458BC0C946A6E0C94EB
:10704000F3B00C9427B30D94A26B0C94CEBB0D94AB
:107050003E070D9498110D94660C0C943FFE0C9411
:10706000D8F60C94E36D0D9403320C941AFE0C9434
:1070700081FE0D9432050D94F61C0C94FDB40C9415
:1070800020B50C9493BC0D940F310C94FAC00D9460
:10709000C3310C94C5BB0C94C8BB0C94B1FC0D94CB
:1070A000D3310C940CB30D948E2F0C94D5FD0D940C
:1070B000DA0F0C94B8C00C94F2FC0D94080E0C94EA
:1070C000D3B00D9445090C94E1B00D940F030C94CA
:1070D00027E30C94B9EA0C9430E30C94BBE90C94CC
:1070E00013C10C94A1C00D949C2F0D944F000C94CF
:1070F00018B30D946E310C94BFE90D943C110C94AF
:1071000038EC0D9442310C94C0B00D946D400C9449
:10711000AEC00C94FD6D0C94D1FC0C9436FE0D9415
:10712000273A0C9477F70C94B8B00C941BB50C94D8
:10713000D6E20C9460BC0D949F0A0D9405310D9419
:10714000836B0D94C5300D94F8110C94166E0C944D
:1071500027C10C948EBC0D94A0650C94F5F70C948B
:10716000D1BB0C94CBBB0D94AF6B0C94FBB00D94C6
:10717000B3310C946FB60C94C2BB0C94E2E20C9445
:107180003BC10D94390F0C9403FD0C94A9C00C94D1
:10719000ADB30D948A2F0D94592F0C94D6F60C9400
:1071A00031FD0C94FAE20C945AB00C94BCB00C94DF
:1071B000DCC00C9408E80C94EEB00D9476010D94AC
:1071C000152F0D94CB310C948FB60C942AE30D94AB
:1071D00002310C94D6700C94E0B50C9409C10C9457
:1071E00014C60C9402B50C948FFE0C9474BC6E61A2
:1071F0006E00696E660000407A10F35A00A0724E6D
:1072000018090010A5D4E80000E87648170000E44B
:107210000B54020000CA9A3B000000E1F505000093
:1072200080969800000040420F000000A0860100F8
:107230000000102700000000E803000000006400C8
:10724000000000000A000000000001000000000033
:107250002C76D888DC674F0823DFC1DFAE59E1B157
:10726000B796E5E3E453C63AE651997696E8E6C266
:107270008426EB898C9B62ED407C6FFCEFBC9C9F6D
:1072800040F2BAA56FA5F490055A2AF75C936B6C8F
:10729000F9676DC11BFCE0E40D47FEF520E6B50083
:1072A000D0ED902E0300943577050080841E0800F1
:1072B00000204E0A000000C80C333333330F986EA1
:1072C00012831141EF8D2114893BE65516CFFEE65E
:1072D000DB18D1844B381BF77C1D901DA4BBE42424
:1072E000203284725E228100C9F124ECA1E53D27A1
:1072F0002200002045535000204E535000204F469E
:107300004600204F4E005056303100205B4D505DFE
:107310002000256920686F757273202569206D69CA
:107320006E757465730052582074696D656F75745D
:10733000004D333130004D313132004D31313000AC
:1073400046756C6C20525820427566666572005313
:10735000657474696E67732053746F72656400534B
:10736000746F7265642073657474696E67732072DC
:1073700065747269657665640048617264636F6400
:1073800065642044656661756C7420536574746926
:107390006E6773204C6F61646564005632000000B4
:1073A00000C8420000C8420000C843000005430076
:1073B00000484300004843000040410000F042E81C
:1073C000030000E8030000C800000088130000006C
:1073D000409C4400409C440000000000000000204D
:1073E0004E00000000204100002041CDCCCC3E00EA
:1073F000009040000000000000000000000000CDF0
:10740000CCCC3E3D0A8141FF08433EB099AB438F4F
:1074100042FC42E65A343F4C62B045000000000096
:107420004040000034420000000000000000000066
:107430000041000000E03F00002C4300002C43000E
:107440000040410000F042C0030000C0030000C83B
:10745000000000881300001010101000409C440031
:1074600000803F0000003F19140000002030780029
:10747000203078006572726F723A200044323320F7
:107480002D20656D657267656E637920736572691D
:10749000616C2064756D7000437573746F6D004E80
:1074A000796C6F6E504100536174696E20200054F6
:1074B000657874757200536D6F6F746800312E308B
:1074C00000312E3500554E4B4E4F574E004C41313A
:1074D00030433A204C696E65617220416476616E7A
:1074E0006365206D6F64653A20004C413130433A4A
:1074F0002041646A757374656420452D4A65726B1A
:107500003A2000CE80CEDE3E0FA8AF00480069963C
:107510000000DF6025555887680427F2E0005E34DC
:1075200003CC1960F33C0EF88F00DB080294920044
:107530003E1C079A8700E524008528527E06001B22
:10754000E4007E781270787061F812788F88417844
:107550004270787061782570787061F850788F8803
:10756000D1F02527078761F025278F88412C0D272B
:10757000AA50D1BC0707871161BE788F8811417866
:107580005270787061F852788F8841201278887034
:1075900063205278887063485278888743031117B4
:1075A000997064181278F870654412F8F8F045186C
:1075B0004278F87065182578F87065185278F87078
:1075C00065185078F870650C078F872365A20F8FB8
:1075D0008F11450012062270690012072227490008
:1075E0002506227069002507222749001206222756
:1075F0006C026236A2706C40456C44704C0362228F
:1076000022706C43888888F04C7812BC88806E7831
:1076100052BC88806E38127888706F7812788887AC
:107620004F38427888706F38257888706F3A0079C3
:10763000AC786F3D079AAC786F7850788887EF39CF
:10764000497888706F0852BC8880729852F88F9879
:107650005220127870F07348127863875320527862
:1076600070F0734852786387531007870F247312A2
:10767000786387245360699A988BE22304E444304A
:1076800074104E444324747C12888960753C508881
:107690008870557825288960757949088960753C16
:1076A00012887070790C12885222594412F124F019
:1076B0007A4452F124F07A8C52F0368F5A4420F1F9
:1076C00024F07A00401454CDCCCC3D0AD7233C178B
:1076D000B7D13877CC2B329595E6241FB14F0A00ED
:1076E0000020410000C84200401C4620BCBE4CCADD
:1076F0001B0E5AAEC59D744E414E494E4600007A4F
:10770000430000524300005243000000000000808C
:10771000C09A99193E00000000000080C09A991993
:107720003E20503A002042403A0020403A00202FAC
:10773000002054303A00202F0020423A00202F0031
:10774000543A002553457863657373697665206202
:107750006564206C6576656C696E6720636F727214
:10776000656374696F6E3A202569206D6963726F75
:107770006E730A00426564206C6576656C696E679D
:10778000206661696C65642E20546F6F206D75638F
:107790006820766172696174696F6E2066726F6DC0
:1077A00020656570726F6D206D6573680042656459
:1077B000206C6576656C696E67206661696C6564CE
:1077C0002E2053656E736F722074726967676572DD
:1077D000656420746F6F20736F6F6E002020004D02
:1077E0006561737572656420706F696E74733A00B9
:1077F0005A20736561726368206865696768743AC6
:1078000020352E3066004E756D20582C593A2037A1
:107810002C37004D65736820626564206C65766561
:107820006C696E67206E6F74206163746976652E73
:107830000020453A00205A3A0020593A0020453AA3
:1078400000205A3A0020593A00583A00202D3E2094
:107850000053706F6F6C4A6F696E3A20002C2000E5
:10786000496E6163746976697479205368757464CC
:107870006F776E004B494C4C45442E005072696E38
:107880007465722068616C7465642E206B696C6C21
:1078900028292063616C6C656421005A206C69762C
:1078A000652061646A757374206F7574206F66203B
:1078B00072616E67652E2053657474696E672074FB
:1078C0006F20302E20436C69636B20746F20636FD0
:1078D0006E74696E75652E005A206C69766520613C
:1078E000646A757374206F7574206F662072616EA0
:1078F00067652E2053657474696E6720746F20303D
:107900000020453A3020423A00543A0062757379BB
:107910003A2070617573656420666F7220696E70BD
:10792000757400627573793A2070617573656420AF
:10793000666F72207573657200627573793A207094
:10794000726F63657373696E670073657269616CEA
:107950002064756D702000496E76616C69642054F6
:1079600020636F64652E004475706C696361746593
:1079700020542D636F64652069676E6F7265642E95
:1079800000416476616E6365204B3D004B206F754E
:1079900074206F6620616C6C6F7765642072616E15
:1079A000676521004D4B322E3553004D4B322E353D
:1079B000534D4D553253001C4FFC002533642F2589
:1079C00033640025336400200A200A200A200025A1
:1079D000534172632053657474696E67733A205023
:1079E0003A4D6178206C656E677468286D6D29204A
:1079F000533A4D696E206C656E67746820286D6D12
:107A000029204E3A436F7272656374696F6E7320FA
:107A1000523A4D696E207365676D656E74732046CA
:107A20003A5365676D656E74732F7365632E0A250F
:107A30005320204D3231342050252E3266205325DC
:107A40002E3266204E256420522564204625640A85
:107A500000255346696C616D656E7420736574749E
:107A6000696E67733A2044697361626C65640A00E9
:107A7000255346696C616D656E7420736574746915
:107A80006E67733A0A25532020204D32303020444F
:107A9000252E32660A002553526574726163743A6A
:107AA00020533D4C656E67746820286D6D29204613
:107AB0003A537065656420286D6D2F6D29205A3A00
:107AC000205A4C69667420286D6D290A25532020A0
:107AD000204D3230372053252E32662046252E3257
:107AE00066205A252E32660A25535265636F7665E5
:107AF000723A20533D4578747261206C656E6774EC
:107B00006820286D6D2920463A53706565642028E9
:107B10006D6D2F6D290A25532020204D32303820DD
:107B200053252E32662046252E32660A255341758E
:107B3000746F2D526574726163743A20533D302026
:107B4000746F2064697361626C652C203120746FDE
:107B500020696E74657270726574206578747275D0
:107B600064652D6F6E6C79206D6F7665732061731F
:107B7000207265747261637473206F722072656322
:107B80006F7665726965730A25532020204D323067
:107B900039205325640A0025535049442068656103
:107BA000746265642073657474696E67733A0A253C
:107BB000532020204D3330342050252E326620496A
:107BC000252E32662044252E32660A002553504960
:107BD000442073657474696E67733A0A25532020D4
:107BE000204D3330312050252E32662049252E324B
:107BF000662044252E32660A00255353746570733F
:107C00002070657220756E69743A0A255320204DE4
:107C100039322058252E32662059252E3266205AB8
:107C2000252E32662045252E32660A25534D617871
:107C3000696D756D20666565647261746573202871
:107C40006D6D2F73293A0A255320204D3230332091
:107C500058252E32662059252E3266205A252E327E
:107C6000662045252E32660A25534D6178696D756B
:107C70006D20616363656C65726174696F6E202845
:107C80006D6D2F7332293A0A255320204D32303141
:107C90002058256C752059256C75205A256C752047
:107CA00045256C750A2553416363656C6572617483
:107CB000696F6E3A20503D7072696E742C20523D8F
:107CC000726574726163742C20543D7472617665C0
:107CD0006C0A255320204D3230342050252E326638
:107CE0002052252E32662054252E32660A25534115
:107CF0006476616E636564207661726961626C6549
:107D0000733A20533D4D696E2066656564726174F7
:107D10006520286D6D2F73292C20543D4D696E20F0
:107D200074726176656C2066656564726174652045
:107D3000286D6D2F73292C20423D6D696E696D751C
:107D40006D207365676D656E742074696D6520289C
:107D50007573292C20583D6D6178696D756D2058BB
:107D600059206A65726B20286D6D2F73292C202095
:107D70005A3D6D6178696D756D205A206A65726B28
:107D800020286D6D2F73292C2020453D6D61786969
:107D90006D756D2045206A65726B20286D6D2F739F
:107DA000290A255320204D3230352053252E3266A6
:107DB0002054252E32662042256C752058252E32FF
:107DC000662059252E3266205A252E3266204525FA
:107DD0002E32660A2553486F6D65206F666673659F
:107DE0007420286D6D293A0A255320204D323036F3
:107DF0002058252E32662059252E3266205A252EEF
:107E000032660A004361703A25533A25630A0050EE
:107E1000525553415F4D4D553200455854454E44DF
:107E200045445F4D3230004155544F5245504F52FA
:107E3000545F504F534954494F4E004155544F528F
:107E400045504F52545F46414E53004155544F5296
:107E500045504F52545F54454D50000044656C6589
:107E600074696F6E206661696C65642C2046696C6C
:107E7000653A200046696C652064656C65746564CC
:107E80003A004E6F74205344207072696E74696EAC
:107E900067005072696E74207361766564005344A4
:107EA000207072696E74207061757365640025338B
:107EB000642F253364006676007468780050524E53
:107EC0000022283229006E6F2076616C696420637D
:107ED0006F6D6D616E64007A65726F72697A656448
:107EE00000666163746F727920726573746F726576
:107EF0006400696E6465782C2074656D702C207543
:107F0000737465702C20756D0050494E4441206398
:107F1000616C207374617475733A2000503A005795
:107F200061697420666F722050494E44412074612B
:107F3000726765742074656D7065726174757265C1
:107F40003A00204100205000204200204C002052E6
:107F500000205A00204E4F5420494E495449414C6C
:107F6000495A45440053686565742000205A2056DC
:107F7000414C5545204F5554204F462052414E47C5
:107F80004500496E76616C6964207368656574208C
:107F900049442E20416C6C6F7765643A20302E2E58
:107FA000004155544F004C414E472053454C20460C
:107FB0004F524345440020643A0020693A00207043
:107FC0003A0020643A0020693A0020703A0025699E
:107FD00025250A00256925250A0022283129002F98
:107FE0002F00002045585452554445525F434F5589
:107FF0004E543A3100204D414348494E455F545953
:1080000050453A00312E3000206261736564206F64
:108010006E204D61726C696E204649524D57415237
:10802000455F55524C3A68747470733A2F2F6769E4
:10803000746875622E636F6D2F707275736133642F
:108040002F50727573612D4669726D77617265206C
:1080500050524F544F434F4C5F56455253494F4E29
:108060003A00303030303030303030005F0038325D
:108070003337002B004649524D574152455F4E4120
:108080004D453A50727573612D4669726D77617214
:108090006520004D3131332053006F6B2000206389
:1080A0006D2E00206D696E20005354415453200002
:1080B0006E2F61003F546F736869626120466C6186
:1080C0007368416972204765744950206661696C24
:1080D00065640A00000125301D0CFF24311C0BFFD4
:1080E000232F1B0A17FF0406222B1A0336353538B7
:1080F0002569206D696E2C20256920736563004910
:108100006E76616C6964204D20636F64653A20254A
:10811000730A0050494E44412070726F62652063BB
:10812000616C6962726174696F6E207374617274DC
:10813000004E6F2050494E444120746865726D694D
:1081400073746F7200736574006E6F7A7A6C650079
:108150004D424C004652004C7A004C616E67003133
:108160005F37356D6D5F4D4B3235532D52414D426A
:108170006F3133612D453344763666756C6C005231
:10818000657600332E31342E312D383233370046A8
:10819000697200534E20696E76616C696400534EBB
:1081A000005245534554004D4D5552455300757688
:1081B0006C6F0046414E0046414E50494E54535458
:1081C0000050525553410047312058313020593129
:1081D0003830204634303030004731205A3130209A
:1081E0004631333030004D313430205330004D3182
:1081F000303420533000473120452D302E30373574
:1082000020463231303000473120463430303000A3
:108210004D323034205331303030004731205A3520
:1082200020463732303000473120452D312E352061
:108230004632313030004739300047312058352040
:108240004534204631303030004731205A302E320C
:108250002046313030300047312058353520453206
:108260003520463134303000473120592D322046F8
:1082700031303030004731205832343020453235EB
:1082800020204632323030004731205A302E332001
:1082900046313030300047312058353520453820C0
:1082A00046323030300047312058352045323920B1
:1082B0004631383030004731205835352045323985
:1082C00020463130373300473932204530004732BD
:1082D00038004D313039004D313930001000C902BD
:1082E00010012C014001220170011801B0010E01A2
:1082F000F00104015002FA00B002F0003003E60081
:10830000D003DC009004D2007005C800A006BE00B7
:108310000008B400B009AA00D00BA000600E9600BF
:1083200060118C000015820020197800C01D6E00BD
:10833000A0226400B0275A00902C50000031460063
:10834000E0343C0010383200903A2800603C1E00B7
:10835000A03D1400803E0A00203F00004578706573
:1083600072696D656E74616C00302E383000302E8D
:10837000363000302E343000302E323500446973F0
:1083800061626C65206661726D206D6F646500527C
:1083900065736574204D4D55004D4D55004D343479
:1083A000004739390044697361626C652066617207
:1083B0006D206D6F64653F00473238205859004D7D
:1083C00020383400852E2E002533642F30002533CD
:1083D000642F30006C63645F73656C66636865630B
:1083E0006B5F617869732025642C2025640A00483E
:1083F0006F74656E6400426564005A00590058004D
:108400002D2D2D2D2D2D2D2D2D2D2D2D2D2D2D2D9C
:108410002D2D2D2D00537570657250494E44413AF3
:1084200000E967F681EE81E681D981C78147312075
:10843000582564205925642045252D2E3566004792
:1084400031204631303830004731205A252D2E3327
:1084500066204637323030004731205835302059B9
:1084600031353500C7823682D96C27821B82108253
:1084700007824731205825642045252D2E3366205C
:10848000463130303000B682A68296828882C7821A
:1084900075826882578249823A8254256400473146
:1084A000205A302E342046313030300047312059A8
:1084B0002D3320463130303000E967D782D282CE6A
:1084C00082C7824D3834205859004D3130392053FD
:1084D0003238300047312058313235205A3230306E
:1084E00020463130303000496E76616C696420502E
:1084F00049442063616C2E20726573756C74732E11
:10850000204E6F742073746F72656420746F204501
:108510004550524F4D2E004D3330312050252E32D4
:10852000662049252E32662044252E3266004D33C2
:1085300030332045302053253375005243004445E5
:1085400056004245544100414C5048410000002132
:1085500000240027002A002D003000330001010014
:1085600000040107010A0100002200250028002B59
:10857000002E003100340002010000050108010B4B
:1085800001000020002300260029002C002F0032CB
:1085900000000100000301060109010505050507AA
:1085A0000508080808020202020A0A08080404046E
:1085B000040101010101010101030303030303039A
:1085C00003040707070C0C0C0C0C0C0C0C02020229
:1085D0000206060606060606060B0B0B0B0B0B0B1C
:1085E0000B07070A0A0A0A0A0A0505050404040813
:1085F00008010210202008081020401020408002AE
:1086000001020108040201010204081020408080D8
:10861000402010080402018004020180402010085C
:108620000402010804020101020408102040800134
:108630000204081020408010080408801020400424
:108640004080102040048000000A0B02090C0D0E2F
:108650000807030401000000000000000000000003
:10866000000000000000000000000000000000000A
:1086700000000012111000000000000000000000C7
:1086800000000000000000000000000000000000EA
:1086900000000000000000000000000000332E3148
:1086A000342E31000A204F726967696E616C205068
:1086B000727573612069330A2020205072757361CE
:1086C0002052657365617263680A2532302E32303C
:1086D000530053706F6F6C4A6F696E20697320008E
:1086E0006164635F696E697400200A200A200A20B1
:1086F00000416C6C2044617461005365727669635B
:10870000652070726570005368697070696E6720CB
:108710007072657000537461746973746963730077
:108720004C616E67756167650045524153494E471C
:1087300020616C6C206461746100466163746F72C7
:1087400079205245534554005052555341334446C5
:10875000570003000E00010040000300020000006B
:108760000400556E6B6E6F776E00313937302D30E7
:10877000312D30312030313A30303A303000203332
:108780002E31342E312D383233375F3030303030A7
:1087900030303030007374617274004D323900250E
:1087A0002D392E39535B0033332942000058419A4A
:1087B000998D4133335340200A200A20004D4D55F6
:1087C000323A004D6561737572652063656E74653C
:1087D0007220200078797A63616C5F6D65617375D2
:1087E00072655F656E7465720A0078797A63616C90
:1087F0005F73706972616C382063783D2564206313
:10880000793D2564207A303D256420647A3D2564D5
:10881000207261646975733D25642061643D25643F
:108820000A0078797A63616C5F7365617263685A74
:10883000206E6F207369676E616C0A20783D256C2D
:108840006420793D256C64207A3D256C640A002003
:108850004F4E2D5349474E414C20617420783D25A1
:108860006420793D2564207A3D25642061643D259E
:10887000640A0078797A63616C5F7365617263681A
:108880005A20783D256C6420793D256C64207A3D22
:10889000256C640A002530327800205B256620258F
:1088A000665D206D6D207061747465726E20636505
:1088B0006E7465720A00205B25662025665D5B2567
:1088C000665D206D6D20646976657267656E6365AF
:1088D0000A000000F000F801FC03FE07FE07FE0797
:1088E000FE07FC03F801F000000000000000F000AB
:1088F000F801FC03FC03FC03FC03F801F00000009A
:10890000000078797A63616C5F6D6561737572657B
:108910005F6C656176650A00203C20005741524E2D
:10892000494E473A2046726F6E7420706F696E74BC
:10893000206E6F7420726561636861626C652E20C1
:108940005920636F6F7264696E6174653A0000004C
:108950000040410000804000005C43000080400077
:10896000005C4300004443000040410000444325B4
:10897000642F3400497465726174696F6E3A200027
:1089800043616C6962726174696F6E206661696CC3
:1089900065642120436865636B2074686520617895
:1089A000657320616E642072756E20616761696E07
:1089B0002E004D494E54454D502042454420666995
:1089C000786564004D494E54454D5020484F5445FC
:1089D0004E442066697865640024F4D43050C38E18
:1089E00020C2A24017828B7011127A910D816CD92E
:1089F0000AA861E108C7586607615143061E4B5D2E
:108A000005C145A7041A411104093D980371393184
:108A1000034036DB0265339102D4305402802E1DB0
:108A200002632CEE01752AC501B028A00110278130
:108A3000018F2564012B244B01E0223401AC211F5E
:108A4000018D200D01801FFC00841EED00971DDFAD
:108A500000B81CD200E61BC600201BBC00641AB282
:108A600000B219A8000A19A0006A189900D117913C
:108A70000040178B00B516840031167E00B31579BF
:108A8000003A157300C7146F0058146A00EE13669D
:108A9000008813630025135E00C7125B006C125739
:108AA0000015125400C111510070114F0021114BDB
:108AB00000D61049008D10470046104400021042B5
:108AC00000C00F4000800F3E00420F3C00060F3BED
:108AD00000CB0E3800930E37005C0E3500270E34A5
:108AE00000F30D3200C10D3100900D3000600D2EED
:108AF00000320D2D00050D2C00D90C2B00AE0C29D9
:108B000000850C29005C0C2700350C27000E0C2674
:108B100000E80B2400C40B2400A00B23007D0B23D2
:108B2000005A0B2100390B2100180B2000F80A1FF6
:108B300000D90A1E00BB0A1E009D0A1D00800A1DE6
:108B400000630A1C00470A1B002C0A1B00110A1AAA
:108B500000F7091A00DD091900C4091900AB091949
:108B600000920917007B091800630917004C0916C9
:108B70000036091600200916000A091500F5081527
:108B800000E0081400CC081400B8081400A408146D
:108B900000900813007D0812006B0813005808129B
:108BA00000460812003408110023081100120811B1
:108BB0000001081100F0071000E0071000D00710B6
:108BC00000C0071000B0070F00A107100091070EAA
:108BD0000083070F0074070F0065070E0057070E8C
:108BE0000049070E003B070D002E070E0020070D61
:108BF0000013070D0006070D00F9060C00ED060D29
:108C000000E0060C00D4060C00C8060C00BC060CE4
:108C100000B0060C00A4060B0099060C008D060B94
:108C20000082060B0077060B006C060B0061060A3B
:108C30000057060B004C060A0042060A0038060AD6
:108C4000002E060A0024060A001A060A0010060969
:108C50000007060A00FD050900F4050900EB0509F7
:108C600000E2050900D9050900D0050900C705097A
:108C700000BE050900B5050800AD050800A50509F9
:108C8000009C050800940508008C05080084050870
:108C9000007C050800740508006C050700650508E0
:108CA000005D050700560508004E0507004705074B
:108CB000004005080038050700310507002A0507B0
:108CC00000230507001C050600160507000F050711
:108CD000000805060002050700FB040600F504076E
:108CE00000EE040600E8040600E2040700DB0406C8
:108CF00000D5040600CF040600C9040600C304061C
:108D000000BD040600B7040600B1040500AC04066B
:108D100000A6040600A00405009B040600950405B7
:108D200000900406008A04050085040500800406FE
:108D3000007A04050075040500700405006B040545
:108D40000066040500610405005C04050057040585
:108D500000520405004D04050048040500430405C5
:108D6000003E0404003A0405003504050030040404
:108D7000002C04050027040400230405001E04043D
:108D8000001A04040016040500110404000D040474
:108D900000090405000404040000040400FC0304AA
:108DA00000F8030400F4030400F0030400EC0304DF
:108DB00000E8030400E4030400E0030400DC03040F
:108DC00000D8030400D4030400D0030400CC03043F
:108DD00000C8030300C503030024F404D9201BC406
:108DE0000C5C0E9804C4095F0265077101F405F973
:108DF00000FB04B30048048700C103690058035511
:108E00000003034500BE023A008402310053022AE7
:108E1000002902250004022000E4011C00C80119F9
:108E200000AF0117009801140084011300710110B4
:108E3000006101100051010E0043010D0036010BCD
:108E4000002B010B0020010B00150109000C01098A
:108E50000003010800FB000800F3000800EB000716
:108E600000E4000600DE000600D8000600D200067E
:108E700000CC000500C7000500C2000500BD0004CD
:108E800000B9000400B5000400B1000400AD000406
:108E900000A9000400A5000300A20003009F000435
:108EA000009B00030098000300950002009300035C
:108EB00000900003008D0002008B00030088000278
:108EC000008600020084000300810002007F00028F
:108ED000007D0002007B00020079000200770001A3
:108EE00000760002007400020072000100710002AE
:108EF000006F0002006D0001006C0002006A0001BA
:108F000000690002006700010066000100650001C1
:108F100000640002006200010061000100600001C5
:108F2000005F0002005D0001005C0001005B0001C9
:108F3000005A0001005900010058000100570001CB
:108F400000560001005500010054000100530000CC
:108F500000530001005200010051000100500001C7
:108F6000004F0001004E0000004E0001004D0001C6
:108F7000004C0001004B0000004B0001004A0001C2
:108F800000490001004800000048000100470001BE
:108F900000460000004600010045000000450001B9
:108FA00000440001004300000043000100420000B3
:108FB00000420001004100000041000100400001AA
:108FC000003F0000003F0001003E0000003E0001A5
:108FD000003D0000003D0001003C0000003C00009E
:108FE000003C0001003B0000003B0001003A000093
:108FF000003A00010039000000390001003800008B
:109000000038000000380001003700000037000180
:109010000036000000360000003600010035000078
:10902000003500000035000100340000003400006D
:109030000034000100330000003300000033000161
:109040000032000000320000003200010031000058
:10905000003100000031000100300000003000004D
:1090600000300001002F0000002F0000002F000042
:10907000002F0001002E0000002E0000002E000135
:10908000002D0000002D0000002D0000002D00012B
:10909000002C0000002C0000002C0000002C00011F
:1090A000002B0000002B0000002B0000002B000113
:1090B000002A0000002A0000002A0000002A000107
:1090C00000290000002900000029000000290000FC
:1090D00000290001002800000028000000280000EE
:1090E00000280000002800010027000000270000E1
:1090F00000270000002700000027000100260000D4
:1091000000260000002600000026000000260001C6
:1091100000250000002500000025000000250000BB
:1091200000250000002500010024000000240000AC
:10913000002400000024000000240001002300009F
:109140000023000000230000002300000023000093
:109150000023000000230001002200000022000084
:109160000022000000220000002200000022000176
:10917000002100000021000000210000002100006B
:10918000002100000021000000210001002000005B
:10919000002000000020000000200000002000004F
:1091A000002000000020000000200001001F00003F
:1091B000001F0000001F0000001F0000001F000033
:1091C000001F0000001F0001001E0000001E000024
:1091D000001E0000001E00000045303A20005A3AF0
:1091E0002000593A2000583A20004D53312C4D535D
:1091F000322050696E7300504944204175746F7479
:10920000756E652066696E697368656421205075A6
:109210007420746865206C617374204B702C204B33
:109220006920616E64204B6420636F6E7374616E9D
:1092300074732066726F6D2061626F766520696E4F
:10924000746F20436F6E66696775726174696F6EC3
:109250002E6800504944204175746F74756E652006
:109260006661696C6564212074696D656F75740051
:1092700020403A00543A00423A0050494420417597
:10928000746F74756E65206661696C656421205425
:10929000656D706572617475726520746F6F20689A
:1092A00069676800204B643A2000204B693A20002F
:1092B000204B703A200020436C6173736963205027
:1092C000494420002054753A2000204B753A200074
:1092D000206D61783A2000206D696E3A200020648C
:1092E0003A200020626961733A20005049442041CD
:1092F00075746F74756E6520737461727400504973
:1093000044204175746F74756E65206661696C6583
:10931000642E2042616420657874727564657220E1
:109320006E756D6265722E00486F74656E6420669E
:10933000616E207370656564206973206C6F77655A
:1093400072207468616E206578706563746564006E
:109350005072696E742066616E207370656564205A
:109360006973206C6F776572207468616E20657810
:10937000706563746564004D494E54454D502042FC
:109380004544004D494E54454D50004D41585445BB
:109390004D50004D415854454D50204245440070B9
:1093A000012C0190012701B0012201C0011D01F033
:1093B0000118011002130130020E01600209019030
:1093C000020401C002FF000003FA004003F5008020
:1093D00003F000D003EB002004E6007004E100E09D
:1093E00004DC004005D700C005D2004006CD00D007
:1093F00006C8008007C3003008BE00F008B900C0EE
:1094000009B400B00AAF00B00BAA00D00CA5000050
:109410000EA000500F9B00C010960050129100004B
:10942000148C00C0158700B0178200B0197D00D0E1
:109430001B7800001E730040206E0090226900F02F
:1094400024640040275F0090295A00E02B5500104B
:109450002E500020304B0010324600E03341009087
:10946000353C001037370070383200A0392D00B07D
:109470003A2800A03B2300603C1E00103D190090DC
:109480003D1400103E0F00703E0A00C03E05000073
:109490003F000020484F54454E4420544845524D0B
:1094A000414C2052554E41574159002048454154A6
:1094B00042454420544845524D414C2052554E415E
:1094C00057415900544845524D414C2052554E4148
:1094D0005741590042454420544845524D414C2083
:1094E00052554E415741590020544845524D414C28
:1094F0002052554E41574159202850524548454128
:109500005420484F54454E44290020544845524D5C
:10951000414C2052554E4157415920285052454800
:109520004541542048454154424544290050524544
:1095300048454154204552524F5200424544205024
:10954000524548454154204552524F5200207472B2
:109550006967676572656421004865617465727347
:10956000207377697463686564206F66662E2000D7
:109570003A20004572723A200000FF010201000209
:10958000FFFFFE0001FE01FF00506C656173652066
:109590007265737461727400555341525432207273
:1095A000782046756C6C212121003A2000252D3150
:1095B000322E313253252D642F36002533642F256A
:1095C0002D336400203A200025335300252D3773B6
:1095D00000252D31352E313553252D35640A252DA5
:1095E00031352E313553252D35640A0025530A2097
:1095F000252D31362E313653252D33640A20252D65
:1096000031362E313653252D33640025530A20255B
:109610002D31362E313653252D33640A20252D3138
:10962000362E313653252D33640A20252D31362E22
:10963000313653252D33640025530A20252D31362C
:109640002E313653252D33640A25530A20252D311A
:10965000362E313653252D33640A002025732533E9
:109660006481200A0025752E25752E25752E2575F9
:109670000020002000466C617368416972204950E7
:1096800020416464723A004D4D5520202020202056
:1096900020204E2F410025642E25642E25640020B5
:1096A00046573A00313937302D30312D30310045B1
:1096B0003344763666756C6C0052414D426F3133DF
:1096C0006100315F37356D6D5F4D4B323553002092
:1096D000486173683A3030303030303030300020FC
:1096E0005265706F3A556E6B6E6F776E0020332E39
:1096F00031342E312D38323337004669726D77613F
:1097000072653A00464C4558202D20203234302FC7
:10971000353000464C4558202D2020323430005042
:10972000502020202D20203235342F313030005071
:10973000502020202D20203235340048495053201D
:109740002D20203232302F31303000484950532004
:109750002D20203232300041425320202D20203253
:1097600035352F3130300041425320202D2020321A
:1097700035350050412020202D20203237352F391B
:10978000300050412020202D202032373500505607
:109790004220202D20203231352F373500505642BF
:1097A00020202D20203231350050432020202D2034
:1097B000203237352F3130350050432020202D20E6
:1097C000203237350041534120202D2020323630C1
:1097D0002F3130350041534120202D2020323630AA
:1097E0000050455420202D20203233302F383500B2
:1097F00050455420202D202032333000504C412041
:10980000202D20203231352F363000504C41202081
:109810002D2020323135006E6F7A7A6C65202D2034
:10982000203235302F30006661726D2020202D20CF
:10983000203235302F383000252D31322E31325341
:10984000252B382E31660045787472756465723A3E
:109850000025632531372E32666D6D00583A005968
:109860003A005A3A002563252D31332E31335325E2
:109870002B352E3366002533750050494E44412068
:1098800063616C6962726174696F6E206661696C94
:1098900065642E20436F6E74696E756520776974F8
:1098A00068207072657373696E6720746865206BD9
:1098B0006E6F622E0050494E44412063616C6962B4
:1098C000726174696F6E20646F6E652E20436F6ED7
:1098D00074696E756520776974682070726573733A
:1098E000696E6720746865206B6E6F622E005A3057
:1098F000005A3100593000593100583000583100B9
:10990000456E642073746F707320646961670047EB
:109910003830004D3435004D3435205A0047373645
:10992000004D3730312050300057697A6172642021
:1099300073746174653A2025640A0078797A6361EA
:109940006C5F73706972616C322063783D256420AE
:1099500063793D2564207A303D256420647A3D2575
:1099600064207261646975733D25642061643D25DE
:10997000640A000A00436F756E74646F776E3A2054
:109980002564200025640A005363616E20636F75AF
:109990006E74646F776E3A20005061747465726EF5
:1099A0002063656E746572205B25662025665D2CDC
:1099B000206D6174636820256625250A00205B25DB
:1099C000662C2025665D5B25665D2066696E616C90
:1099D00020636972636C650A000000A0400000A06B
:1099E000400000004000007A43000056439AD951DD
:1099F00043FFFFFFE02D903E8988B24111369C3E27
:109A00007777C14129CBB03EEFEEDA41BA49CC3E7F
:109A1000EFEEFC4161C3F33EEFEE16429CA2133F12
:109A2000CDCC36428AB0113FABAA56428863DD3DA9
:109A3000ABAA5642B8AF433F555572421826533F22
:109A400033B38242302A593FEF6E8642000070C124
:109A50000000C8420000C4C10000A0410000E0C0F6
:109A600000002041000060C00000C0400000A04194
:109A70002222F2400000A0C19A99A14000000CC22D
:109A800055550542436F6F6C696E672074696D654B
:109A9000722073746F7070656400486561746572DC
:109AA00020636F6F6C646F776E00436F6F6C696ECD
:109AB000672054696D656F75742073746172746585
:109AC0006400536176696E6720616E642070617214
:109AD0006B696E670048656174657220636F6F6CB7
:109AE000646F776E2070656E64696E67005265738F
:109AF000756D696E672058595A00473120582564A2
:109B00002059252D2E32662045252D2E33660057EF
:109B1000726974696E6720746F2066696C653A209B
:109B20000046696C6520616C7265616479206F70B4
:109B3000656E656400315820580C58F757E157CED0
:109B400057B857A45793577D570C58205869575A00
:109B500057465735572057C45A0A57F856E556D432
:109B600056BF56AC56985683567A56685653564D3D
:109B7000363030204155544F0046494E444120660E
:109B8000696C616D656E742072756E6F75742100FD
:109B9000436F6D6D756E69636174696F6E20746972
:109BA0006D656F75740050726F746F636F6C2045D4
:109BB00072726F720003000356657273696F6E20D4
:109BC0006D69736D6174636800436F6D6D616E6480
:109BD000204572726F7200436F6D6D616E6420720A
:109BE000656A6563746564004D4D552042757474F3
:109BF0006F6E207075736865640052657472794287
:109C00007574746F6E50726573736564008E5A79E3
:109C10005A625A4D5A385A245A145AFD59E659CFA5
:109C200059BB59A7599159915991597C597C597CE3
:109C3000596959695969595659565956593F593FA1
:109C4000593F592A592A592A59145914591459044F
:109C500059EF58D958C358B458A75890587D586BE5
:109C600058585846583658427574746F6E00436899
:109C700065636B55736572496E7075742D62746E91
:109C80004C4D52200052657365745265747279416F
:109C90007474656D7074730046493A202046533AD7
:109CA000202020203E2020822020208100486F7428
:109CB000656E642074656D7065726174757265207F
:109CC0007265616368656400526573756D696E677E
:109CD0002054656D7000436F6F6C646F776E206603
:109CE0006C616720636C65617265640020573A009F
:109CF00020453A00543A004E6F2030784646207294
:109D0000656365697665640053656E64696E672096
:109D1000307846460046696C652073656C656374EF
:109D20006564002053697A653A200046696C6520B5
:109D30006F70656E65643A20004E6F7720667265BD
:109D400073682066696C653A20004E6F7720646FF7
:109D5000696E672066696C653A20002220706F7317
:109D6000002220706172656E743A2200535542528F
:109D70004F5554494E452043414C4C207461726705
:109D800065743A2200747279696E6720746F20637B
:109D9000616C6C207375622D67636F646520666902
:109DA0006C6573207769746820746F6F206D616EC5
:109DB00079206C6576656C732E0020222573220055
:109DC0002025236C78004449525F4558495400448B
:109DD00049525F454E5445523A202573202225733F
:109DE000220A006175746F25692E6700041A4465A4
:109DF0006372656D656E74526574727941747465D1
:109E00006D70747300081B1C0B14525354436F6D18
:109E10006D54696D656F7574002C206C61737420CE
:109E200062797465733A200022206661696C65640A
:109E30003A204275666665722066756C6C21002258
:109E400000456E717565696E6720746F2074686572
:109E50002066726F6E743A2022004572726F723AF9
:109E6000004D4D5532746F6F6C3D004D4D55323A7B
:109E7000004D4D55323A006563686F3A003E5330ED
:109E80002A63362E004D4D552069732000252E3152
:109E90003053200025346400457872656D65207369
:109EA00070616E206F6620746865205A2076616C40
:109EB000756573210025642F39004D4D55323A00E8
:109EC0002533640018010419020A5462DE616461DA
:109ED000F760AE601C60A45F3C5FED5ECD5E815EAE
:109EE000CD5E6A5E6A5E6A5E6A5E6A5E6A5E6A5ECF
:109EF0006A5E6A5E6A5E6A5E6A5E6A5E6A5E6A5E22
:109F00006A5E6A5E6A5E6A5E6A5E6A5E6A5E335E48
:109F1000F25DA85D355D005DB65C6C5C0E5CD55B8A
:109F2000935B765B01010101010101027101710185
:109F30003232320303030303030303030303030364
:109F4000030303030303939324380393030102568B
:109F500003650066006700680069006A006B006CBA
:109F600000730074007D007E00C900D300DD00CACC
:109F700000D400DE002D01370141012E01380142DD
:109F8000012F013901430130013A01440131013B04
:109F9000014501320191019201F501F601F701F845
:109FA00001F901FA01FB01FC018403E1624A63D675
:109FB00062CD62C662414B503DBF62B562252E3212
:109FC00030530A70727573612E696F2F30342568B3
:109FD00075007B5B4552523A00332E31342E3100EE
:109FE0005D5B4657523A005D5B54494D3A005D5BFC
:109FF000464E4D3A005D5B46454D3A005D5B504331
:10A00000443A005B5446553A005B50524E3A005B6E
:10A0100050464E3A305D005B4449413A005D5B4139
:10A0200054423A005D5B4154303A005D5B53544208
:10A030003A005B5354303A007B5B50524E3A355DE8
:10A04000007B5B50524E3A305D007B5B50524E3A83
:10A05000395D007B5B50524E3A385D007B5B524568
:10A06000533A305D5B46494C3A007B5B5245533A6C
:10A07000315D5B46494C3A000000211042206330BC
:10A080008440A550C660E770088129914AA16BB150
:10A090008CC1ADD1CEE1EFF13112100273325222F8
:10A0A000B5529442F772D662399318837BB35AA3A0
:10A0B000BDD39CC3FFF3DEE36224433420040114C8
:10A0C000E664C774A44485546AA54BB528850995F0
:10A0D000EEE5CFF5ACC58DD5533672261116300698
:10A0E000D776F6669556B4465BB77AA71997388740
:10A0F000DFF7FEE79DD7BCC7C448E5588668A77858
:10A100004008611802282338CCC9EDD98EE9AFF98F
:10A11000488969990AA92BB9F55AD44AB77A966A37
:10A12000711A500A333A122AFDDBDCCBBFFB9EEBDF
:10A13000799B588B3BBB1AABA66C877CE44CC55C07
:10A14000222C033C600C411CAEED8FFDECCDCDDD2F
:10A150002AAD0BBD688D499D977EB66ED55EF44ED7
:10A16000133E322E511E700E9FFFBEEFDDDFFCCF7F
:10A170001BBF3AAF599F788F8891A981CAB1EBA1D3
:10A180000CD12DC14EF16FE18010A100C230E3204F
:10A190000450254046706760B9839893FBA3DAB3F7
:10A1A0003DC31CD37FE35EF3B1029012F322D2329F
:10A1B0003542145277625672EAB5CBA5A8958985C7
:10A1C0006EF54FE52CD50DC5E234C324A0148104EF
:10A1D0006674476424540544DBA7FAB79987B89797
:10A1E0005FE77EF71DC73CD7D326F2369106B0163F
:10A1F00057667676154634564CD96DC90EF92FE957
:10A20000C899E9898AB9ABA944586548067827688E
:10A21000C018E1088238A3287DCB5CDB3FEB1EFB36
:10A22000F98BD89BBBAB9ABB754A545A376A167ADE
:10A23000F10AD01AB32A923A2EFD0FED6CDD4DCD06
:10A24000AABD8BADE89DC98D267C076C645C454C2E
:10A25000A23C832CE01CC10C1FEF3EFF5DCF7CDFD6
:10A260009BAFBABFD98FF89F176E367E554E745E7E
:10A27000932EB23ED10EF01E7C3C3E3F2F2A225C34
:10A2800000008538D85E11241FBECFEFD1E2DEBFBB
:10A29000CDBF00E00CBF13E0A0E0B2E0E0E1F0E5EC
:10A2A00003E00BBF02C007900D92A430B107D9F7AD
:10A2B00027E1A4E0B3E001C01D92A430B207E1F7AA
:10A2C00011E5C2E4D1E500E006C021970109802F25
:10A2D000FE010F944CA2C134D10780E00807A9F712
:10A2E0000E9496D80D94F6A70C9443752F923F9236
:10A2F0004F925F926F927F928F929F92AF92BF9296
:10A30000CF92DF92EF92FF920F931F93CF93DF9341
:10A31000CDB7DEB72F970FB6F894DEBF0FBECDBF17
:10A320006C011B015A01FC011782168283819E0178
:10A330002F5F3F4F490181FDD2C08FEF9FEFEEC2EB
:10A34000F12C512C00E0003238F48B3209F190F4FA
:10A350008032F9F0833209F107FD34C020ED280F77
:10A360002A3020F506FF1BC0FAE0FF9E200D1124C5
:10A37000F22E05C08D3279F0803371F70160F10162
:10A3800093FD859193FF81911F018111DCCF1AC04C
:10A3900002600460F4CF0860F2CF0061F0CF3AE0D1
:10A3A000539E200D1124522E0062E9CF8E3221F4EB
:10A3B00006FDB1C20064E3CF8C3611F40068DFCF34
:10A3C0008836E9F29BEB980F933008F05FC000618C
:10A3D000805E06FD02C046E0F42E102F1F73853606
:10A3E00009F05BC0106417FF61C08F2D9BE39F15C0
:10A3F00008F48BE344244394480E27E03501F4E04D
:10A400006F0E711CF5016081718182819381042D31
:10A41000A4010F94F59D5C01F981FC87F0FF03C056
:10A420000DE2F3FF07C00BE211FD04C0012F047021
:10A4300012FD00E22C852C70E22E09F46BC0011194
:10A44000D8C2F3E0E12CF515A0F483E0E52CE81A7E
:10A4500013FD08C0B60180E290E00F94A49FEA9437
:10A46000E110F8CF002329F0B601802F90E00F947F
:10A47000A49F3C852EEEA22E21E7B22E33FD04C010
:10A4800092EFA92E91E7B92E107122C09BE9980F87
:10A49000933008F047C10F7E9CCF863611F41068C8
:10A4A000A2CFFF2009F49FCFFA949DCFE7E02F2D94
:10A4B000EF1518F427E037E0F32E412C9FCF111150
:10A4C0008052B60190E00F94A49F8FEFA81AB80AAB
:10A4D000F50184918111F3CFE11084C25301F6019B
:10A4E0009381F10193FD859193FF81911F01882351
:10A4F00009F411C2853241F493FD859193FF819156
:10A500001F01853209F01CCFB60190E00F94A49F83
:10A510003501E4CF17FF6FC04A0CFC85F4FF04C07F
:10A520008A81813309F44A9414140CF086C028E01F
:10A53000241510F488E0482E85E090E017FF06C04F
:10A54000C501B7FE02C090E080E0019601110196BE
:10A55000FF2031F02F2D30E02F5F3F4F820F931FF0
:10A560005816190619F014F0E52CE81A812F897095
:10A5700011F4E11067C0002329F0B601802F90E0AC
:10A580000F94A49F13FD02C0E11063C017FF7CC0AD
:10A590008501B7FE02C010E000E0C50184199109F1
:10A5A0002C016F2D70E0EE27FF27E61BF70BFF87CE
:10A5B000EE870F3F100729F4B6018EE290E00F946A
:10A5C000A49FA016B1060CF44BC0401651060CF027
:10A5D00047C0F501E01BF10BE80DF91D8181015029
:10A5E00011092E853F8502171307E4F1B60190E0AB
:10A5F0000F94A49FDECF16FD9FCFEF2DF0E0EA155C
:10A60000FB0534F03CEFA3163FEFB3060CF01068E7
:10A610003296E80DF91D01C0FA94FF2019F08291DD
:10A620008033D1F317FF88CF442443944F0CFA149E
:10A630001B0431F02CF0FA187FCF442443947CCFD4
:10A64000F12C7ACFB60180E290E00F94A49FEA94B7
:10A6500090CFB60180E390E00F94A49FEA9494CF4A
:10A6600080E3BDCFA016B10641F49A81963350F431
:10A67000953319F43C8534FF05C0B60190E00F9482
:10A68000A49F2ACF81E3F9CF8A81813319F09C8579
:10A690009F7E9C87B60190E00F94A49FFF20A9F0B5
:10A6A000B6018EE290E00F94A49FF394F394E2E05D
:10A6B00001E00E0FE80DF92DF11D8081B60190E04B
:10A6C0000F94A49FE02F0F11F3CF85E690E014FFC5
:10A6D00002C085E490E0B6010F94A49FB7FC06C0C9
:10A6E000A114B104C1F4EC85E4FF15C0B194A194A8
:10A6F000B1088DE2B60190E00F94A49F80E32AE0B8
:10A70000A216B10454F4B60190E00F94A49FB601D0
:10A71000C501C096B4CF8BE2EDCF8F5FFAE0AF1AE0
:10A72000B108EDCF8336C9F0833771F1833509F075
:10A730005BC03501F2E06F0E711CF501A080B180A5
:10A740006F2D70E006FD02C06FEF7FEFC5010F9423
:10A75000389F9D878C8700680DC0350132E0630EFD
:10A76000711CF5018081898321E030E03D872C87D1
:10A7700054010F7703FD06C02C853D855216130644
:10A7800009F0A8F4E52C2BC0350132E0630E711CF2
:10A79000F501A080B1806F2D70E006FD02C06FEF63
:10A7A0007FEFC5010F945D9F9D878C87E2CFB60137
:10A7B00080E290E00F94A49F5A94DECFF50107FD4C
:10A7C000859107FF81915F01B60190E00F94A49FEE
:10A7D000E110EA948C859D8501979D878C87EC8597
:10A7E000FD85EF2B59F778CE843619F0893609F0BC
:10A7F00074C0350107FF66C0F4E06F0E711CF501EF
:10A800006081718182819381102F1F7697FF08C02C
:10A8100090958095709561957F4F8F4F9F4F1068F1
:10A820002AE030E0A4010F94CBA0A82EA818BA2CDF
:10A83000012F16FF0AC00E7FAF1438F414FF04C0B6
:10A8400012FD02C0012F0E7EBF2C04FFA3C0FE012B
:10A85000EA0DF11D8081803309F095C0097EF02F4B
:10A86000F870EF2E03FDA5C000FF9FC0FA2CB514B1
:10A8700010F4F50CFB1804FFA2C0B60180E390E0D1
:10A880000F94A49F02FF09C088E790E001FF02C077
:10A8900088E590E0B6010F94A49FAF1408F49BC024
:10A8A000AA940A2D10E00F5F1F4F080D191DF80123
:10A8B00082918F01B60190E00F94A49F80169106BB
:10A8C000B1F70ACEF2E06F0E711CF5016081718163
:10A8D000072E000C880B990B97CF102F8537A9F402
:10A8E0001F7E2AE030E0350117FF44C0F4E06F0E10
:10A8F000711CF5016081718182819381A4010F94A3
:10A90000CBA0A82EA8181F7792CF197F8F3679F188
:10A91000F0F4883539F1F601868197812F960FB6CC
:10A92000F894DEBF0FBECDBFDF91CF911F910F9185
:10A93000FF90EF90DF90CF90BF90AF909F908F905F
:10A940007F906F905F904F903F902F900895803749
:10A9500039F0883701F714FD146020E130E0C3CFEF
:10A960001061F9CF04FD166020E132E0BCCF28E091
:10A9700030E0B9CFF2E06F0E711CF501608171819A
:10A9800090E080E0BBCF02FD02C0B39468CFB394E7
:10A99000B39465CF802F867809F461CFF6CFB601E6
:10A9A00080E290E00F94A49FB394B514C0F3E12C1F
:10A9B00062CFE52CEB18B51408F45DCFF8CF802FEB
:10A9C000867809F46ACF8BE201FF80E207FD8DE211
:10A9D000B60190E060CFB60180E390E00F94A49FB1
:10A9E000FA945BCFB60180E290E00F94A49FEA94C2
:10A9F00073CD24E0E12C251508F036CD84E026CD7A
:10AA000020E030E040E85FEB60917E0270917F02D1
:10AA100080918002909181020F9459A3882321F1A3
:10AA2000E091CB11F091CC11E252F04F80818B7FFD
:10AA30008230D1F480E1EEE7F2E0A5EFB1E10190E0
:10AA40000D928A95E1F780E090E0A0E8BFEB80935B
:10AA50007E0290937F02A0938002B0938102809146
:10AA6000E0119091E111089581E090E0089580E176
:10AA7000E3E9F6E0A5EFB1E101900D928A95E1F7E7
:10AA80000895E6ECF6E7833021F0E82FF0E0ED538F
:10AA9000F948849108958091AF059091B005209177
:10AAA000B1053091B205821B930B8F7799270895DA
:10AAB000982F9F7083FF0DC080917B0088608093EA
:10AAC0007B0080917C00887F9770892B80937C002D
:10AAD000089580917B00877FF2CF8091B10590919E
:10AAE000B2059093B0058093AF0585ED99E69F93ED
:10AAF0008F938091D1119091D211A091D311B091E7
:10AB0000D4110196A11DB11DBF93AF939F938F9355
:10AB10008DEF94E69F938F9384E095E69F938F93B8
:10AB20000F94FE9F8DB79EB70A960FB6F8949EBFFE
:10AB30000FBE8DBF08950F931F93CF93DF93EC014A
:10AB4000C60FD71F8C179D0779F08C010F5F1F4F21
:10AB50000F943CA18F3F31F081E0DF91CF911F91A5
:10AB60000F910895C801EECF80E0F7CF682F880FCE
:10AB7000770B8091CB119091CC118F51904F0F9406
:10AB800093A79C019093F6168093F51681E0232BF2
:10AB900009F480E008958091F5169091F6164AE048
:10ABA00050E070E060E001960F94C79C862F0895F6
:10ABB0008091F5169091F6164AE050E070E060E062
:10ABC00001960F94C79CCB0108950F931F93CF93C9
:10ABD000DF938C01862FEA010E94B655882319F174
:10ABE0000E94D8559C0197FF03C0319521953109EA
:10ABF000253631059CF09F938F938AE59EE99F93BC
:10AC00008F9383E497E79F938F930F94FE9F0F900A
:10AC10000F900F900F900F900F9080E0DF91CF91E9
:10AC20001F910F910895F80180818823B1F3CE011F
:10AC3000DF91CF911F910F910D943CA18091F5165A
:10AC40009091F6164AE050E070E060E001960D94B5
:10AC5000C79C60E086E69FE00F9460A160E088E614
:10AC60009FE00F9460A160E085E69FE00F9460A1F3
:10AC700060E084E69FE00F9460A160E082ED9EE0DA
:10AC80000F9460A160E08FEC9EE00D9460A180368F
:10AC90009105F8F44091CB115091CC112091DC0F2B
:10ACA0003091DD0F4217530739F46091CF11709145
:10ACB000D011161617066CF0B901680F791FFB0149
:10ACC000E359FF4F2417350730F481E04E175F0733
:10ACD00008F480E00895EE3EF140F8F06C5F7F4F9D
:10ACE0006E3E714018F449365105B8F483599F4FB0
:10ACF0004817590770F34DEE51E0421B530B70E0BB
:10AD000060E0C9018252904F0F946EA78FB7F894FC
:10AD10001092DD0F1092DC0F8FBF81E008952F920B
:10AD20003F924F925F926F927F928F929F92AF92DB
:10AD3000BF92CF92DF92EF92FF920F931F93CF9328
:10AD4000DF93CDB7DEB7CC58D2400FB6F894DEBF54
:10AD50000FBECDBFCB58DD4F688379838A839B8339
:10AD6000C557D240FE01E754FE4F88E2DF011D9235
:10AD70008A95E9F7E85BF1401F0180E991E0DF0186
:10AD8000FC011D923197E9F7C75ADD4F19821882ED
:10AD9000C955D2409E012F513E4FC159DD4F3983D5
:10ADA0002883CF56D2408E01075A1D4FCE018F5CAB
:10ADB0009D4FC359DD4F99838883CD56D2403C01C6
:10ADC000490140EBA42E4FE0B42E53E2C52ED12C06
:10ADD000F12CE12CB6010D2C000C880B990B0F9473
:10ADE000CA9BD4016D937D938D939D934D01F80182
:10ADF000619171918F01072E000C880B990B0F94B4
:10AE0000CA9BD3016D937D938D939D933D01BFEFBD
:10AE1000EB1AFB0AE6E0EE16F10409F038C3CB5852
:10AE2000DD4F288139814A815B81C557D240C159A4
:10AE3000DD4FA881B981CF56D2406D917D918D9122
:10AE40009C910F94EDA4412C512C320118160CF456
:10AE500002C3C359DD4F08811981CD56D2400C5E23
:10AE60001F4FC159DD4FE880F980CF56D240B4E181
:10AE7000EB0EF11C6E01EFEDCE1AEDEFDE0A9E0136
:10AE80002B553E4FCF58DD4F39832883C157D240D1
:10AE9000D8014D905D906D907C90F701608171813B
:10AEA00082819381D7015E914E913E912E917D01D9
:10AEB0000F9463A24B015C01F801529142913291CF
:10AEC00022918F01C301B2010F9463A2A5019401E5
:10AED0000F9463A3D6019E938E937E936E936D0120
:10AEE000CF58DD4FE881F981C157D240B292A2928A
:10AEF00092928292CF58DD4FF983E883C157D240B6
:10AF0000C359DD4F28813981CD56D240021713072E
:10AF100009F0BECF4E013FE6831A3EEF930A5E0171
:10AF200083EFA81A8DEFB80A61018101EE24E39442
:10AF3000F12CD4014D905D906D907D904D012D913F
:10AF40003D914D915C91C301B2010F9464A29B01AC
:10AF5000AC010F9464A2F80164A775A786A797A710
:10AF6000F1E0EF16F10461F0D80198964D925D92F0
:10AF70006D927C929B97F80144825582668277821B
:10AF8000FFEFEF1AFF0AF5012081318142815381E1
:10AF900084E0A80EB11C64817581868197810F942D
:10AFA00063A220E030E040EC50E40F94099CD6010D
:10AFB000DC966D937D938D939C93DF97045D1F4F7B
:10AFC000B8E2CB0ED11CE5E0EE16F10409F0B1CFEA
:10AFD0007E01FDE2EF0EF11C28E2A22EB12C00EB67
:10AFE0001FEF24E0220E311CD7012D913D914D9190
:10AFF0005C91139798966D917D918D919C919B9703
:10B000000F9463A32B013C016101C01AD10A88246B
:10B010008394912CF601E00FF11FEA0DFB1D2081B6
:10B02000318142815381C301B2010F94099C9B017C
:10B03000AC01F60160817181828193810F9463A2DA
:10B04000D6016D937D938D939D936D01BFEF8B1A08
:10B050009B0AE6E08E169104E9F63CE2E30EF11C51
:10B060000852110988E2A80EB11C08339FEF190796
:10B0700009F0BACF1E01F5EB2F0E311C6E0121EB4A
:10B08000C20ED11C7E0137E3E31A3EEFF30A04E05F
:10B0900010E04801B12CA12C412C512C3201F601B9
:10B0A000EA0DFB1DD701AA0DBB1D2D913D914D91C0
:10B0B0005C9160817181828193810F94099C9B01D5
:10B0C000AC01C301B2010F9464A22B013C018FEFCC
:10B0D000881A980A94E0A90EB11CA5E08A1691047A
:10B0E000F1F6A3019201F101608171818281938166
:10B0F0000F9463A2D6012D913D914D915C910F94D7
:10B1000063A3F701608371838283938301501109E4
:10B11000F8E22F1A31082CE2C21AD10834E0E31AFF
:10B12000F1080115110509F0B4CFCB50DE4F88812D
:10B130009981AA81BB81C55FD140CF57DD4F8883FC
:10B140009983AA83BB83C158D2401E0197E4291A70
:10B150009EEF390A10E000E0C159DD4FA881B981A6
:10B16000CF56D240CD90DD90ED90FD90C159DD4F8E
:10B17000B983A883CF56D240CB58DD4F288139817F
:10B180004A815B81C557D240C701B6010F9459A3CC
:10B190001816B4F0CB58DD4F288139814A815B8184
:10B1A000C557D240C159DD4FE881F981CF56D24011
:10B1B00060817181828193810F94EDA487FF18C013
:10B1C0000430110509F030C1CB58DD4F2881398199
:10B1D0004A815B81C557D240CF57DD4F6881798165
:10B1E0008A819B81C158D2400F9459A387FF1CC10B
:10B1F000D10114968D909D90AD90BC9017978D9134
:10B200009D910D90BC91A02DCF58DD4F88839983DF
:10B21000AA83BB83C157D240F801EE0FFF1FEE0F88
:10B22000FF1F21E931E02C0F3D1FE20FF31F40808B
:10B23000518062807380C359DD4FA881B981CD569A
:10B24000D2408D919D910D90BC91A02DC358DD4FA2
:10B2500088839983AA83BB83CD57D240A7019601E7
:10B26000CB58DD4F688179818A819B81C557D24057
:10B270000F9463A26B017C0120E030E040E450E4D5
:10B280000F94D4A5CB57DD4F688379838A839B8342
:10B29000C558D240C358DD4F288139814A815B812E
:10B2A000CD57D240C359DD4FE881F981CD56D24008
:10B2B00064817581868197810F9463A2A3019201B5
:10B2C0000F9463A3C758DD4F688379838A839B8378
:10B2D000C957D240A3019201C301B2010F9464A2E5
:10B2E000CF58DD4F288139814A815B81C157D240D7
:10B2F0000F94099CC757DD4F688379838A839B83AA
:10B30000C958D240A3019201C501B4010F94099C10
:10B310009B01AC01C757DD4F688179818A819B8190
:10B32000C958D2400F9464A220E030E040EC50E4D1
:10B330000F9463A39B01AC01C758DD4F68817981ED
:10B340008A819B81C957D2400F9463A2A7019601BD
:10B350000F94099CC758DD4F688379838A839B8348
:10B36000C957D240CF58DD4F288139814A815B814E
:10B37000C157D240C501B4010F9463A24B015C01D7
:10B3800020E030E040EC50E4C301B2010F94099C8E
:10B390009B01AC01C501B4010F9463A3CB57DD4FF2
:10B3A000288139814A815B81C558D2400F94099C1C
:10B3B0004B015C0120E030E040E05FE3CF58DD4F1F
:10B3C000688179818A819B81C157D2400F94099C01
:10B3D0002B013C01A7019601C701B6010F94099CFE
:10B3E0009B01AC01C301B2010F94099C9B01AC010C
:10B3F000C501B4010F9464A29B01AC01C758DD4F95
:10B40000688179818A819B81C957D2400F9464A257
:10B41000C358DD4F288139814A815B81CD57D240A5
:10B420000F9464A22B013C010F5F1F4FF4E02F0E1D
:10B43000311CC359DD4F28813981CD56D2402C5F54
:10B440003F4FC359DD4F39832883CD56D240053055
:10B45000110509F081CEC301B201C457DD4F0FB60B
:10B46000F894DEBF0FBECDBFDF91CF911F910F913A
:10B47000FF90EF90DF90CF90BF90AF909F908F9014
:10B480007F906F905F904F903F902F900895C501EF
:10B490000F944AA1D8018D939C93B5E0CB0ED11C9B
:10B4A000E2E0AE0EB11C96CC0F931F93CF93209188
:10B4B0009412213079F58C0180E50E94B6558823DD
:10B4C00049F10E94CB55C82F853020F5013C82E020
:10B4D000180749F0023C124069F08C2FCF911F9160
:10B4E0000F910D940B6C60E08C2FCF911F910F91F9
:10B4F0000D944E6C8EEC9EE00F943CA1882351F08D
:10B500000F941455882331F08C2FCF911F910F91F8
:10B510000D94CB6CCF911F910F9108958F929F92B4
:10B52000AF92BF92CF92DF92EF92FF920F931F9351
:10B53000CF93DF930091F5161091F6160F5F1F4F12
:10B5400068018FEFC81AD80AD801DC918D2F90E0DE
:10B550000F94CD9E7C01892B01F5DD3201F5680148
:10B56000B2E0CB0ED11CF801D181C1E086010150BF
:10B57000110943E050E06AEF76E7C8010F94039F9A
:10B58000892BC1F460E070E080E89FEFC111DBC05F
:10B5900060E070E080E89FE7D6C08601D1CFDB3263
:10B5A00039F46801F2E0CF0ED11CD8011196DC917C
:10B5B000C0E0DCCF43E050E067EF76E7C8010F94CE
:10B5C000039F892B09F4CCC0F60110E000E020E0D5
:10B5D00030E0A9016F01D053DA3060F5BC2E6894D9
:10B5E000B1F88C2F8870C2FF09C0811102C00F5FB3
:10B5F0001F4F3196D601DC91CB2DECCF882311F073
:10B6000001501109A5E0B0E00F94D1A19B01AC015C
:10B61000220F331F441F551F2D0F311D411D511D7A
:10B620002839B9E93B074B07B9E15B0710F3C6605E
:10B63000BC2EDFCFDE3F31F4C3FD33C0BC2E689497
:10B64000B3F8D7CFD53369F580818D3231F4C0613D
:10B65000BF016E5F7F4F818105C0BF018B32C9F38F
:10B660006F5F7F4F80538A30E0F4FB01B0E8EB1648
:10B67000BCE0FB065CF4B701660F771F660F771F0F
:10B68000E60EF71EEE0CFF1CE80EF11C81918053B4
:10B690008A3060F3C4FF03C0F194E194F1080E0D09
:10B6A0001F1DCA01B9010F94C89BC370C33009F4B0
:10B6B00090584B015C0120E030E0A9010F9459A3A0
:10B6C000882309F43EC0C3EFD6E717FF05C01195E4
:10B6D00001951109CBEDD6E76E01E8E1CE1AD1084C
:10B6E00080E2E82EF12C0DC0FE01259135914591A7
:10B6F00054910E191F09C501B4010F94099C4B0107
:10B700005C01D501C4010E151F0574F72497F5944B
:10B71000E794CC16DD06A9F78A2F880F8B2F881F98
:10B720008F3F49F020E030E0A901C501B4010F943A
:10B7300059A3811106C082E290E09093F91680939C
:10B74000F816C501B401DF91CF911F910F91FF90C1
:10B75000EF90DF90CF90BF90AF909F908F90089523
:10B7600060E070E080EC9FE7EECF2F923F924F9227
:10B770005F926F927F928F929F92AF92BF92CF9281
:10B78000DF92EF92FF920F931F93CF93DF93CDB78A
:10B79000DEB7A1970FB6F894DEBF0FBECDBF84EC25
:10B7A00092E09D8F8C8F85EF282E81E1382E03E962
:10B7B00016E091E09A8F198EEC8DFD8D8191FD8FB1
:10B7C000EC8F0E94B655E82E882309F454C1F090FE
:10B7D000EB11FA8DFF220E948E5A2B013C01F801D9
:10B7E0004082518262827382F98DF33009F045C044
:10B7F000DD24D394F11001C0D12C809010029090E0
:10B800001102A0901202B090130220E030E040E854
:10B810005FE3C501B4010F9459A3882359F1F110D6
:10B8200015C02091011230910212409103125091E3
:10B830000412C301B2010F9463A260939F06709338
:10B84000A0068093A1069093A206DE2CA501940188
:10B8500060919F067091A0068091A1069091A2062A
:10B860000F94099C60939F067093A0068093A10695
:10B870009093A206D11003C05FC0FF2089F0F101B0
:10B880002081318142815381F801608171818281FF
:10B8900093810F9464A2F801608371838283938300
:10B8A000F98DF230D9F580918903823009F0EEC02C
:10B8B0008CE0E0EAF2E0DE011D9601900D928A959F
:10B8C000E1F78CE0ECEAF2E0DE01119601900D92D6
:10B8D0008A95E1F7C0909B06D0909C06E0909D066B
:10B8E000F0909E0620E030E0A901C701B6010F9458
:10B8F00059A387FF52C0CE0101967C01D12CF701DC
:10B9000061917191819191917F010F94D5A38D2DBA
:10B910000F94ED21D394F3E0DF12F1CFF98DFF5FA7
:10B92000F98F8A8D880F8A8F94E0290E311C0C5F65
:10B930001F4FF43009F040CF86E40E94B6558823AB
:10B9400099F00E948E5A6B017C0120E030E0A90141
:10B950000F94EDA4181644F4C0927A02D0927B02A0
:10B96000E0927C02F0927D02A1960FB6F894DEBFC1
:10B970000FBECDBFDF91CF911F910F91FF90EF9040
:10B98000DF90CF90BF90AF909F908F907F906F90FF
:10B990005F904F903F902F90089520E030E048E472
:10B9A00053E4C701B6010F94EDA41816A4F4CE0118
:10B9B0000D967C01D12CF70161917191819191914A
:10B9C0007F010F94D5A38D2D0F94ED21D394F3E037
:10B9D000DF12F1CFA3CFCE01019699A388A3FE0178
:10B9E0003D96FF8FEE8F1B8EE8A1F9A1C190D190FB
:10B9F000E190F190F9A3E8A3EE8DFF8D6191719133
:10BA000081919191FF8FEE8FA70196010F9463A210
:10BA100020E030E048E453E40F9463A34B015C0161
:10BA200020919B0630919C0640919D0650919E0668
:10BA30000F94099C2B013C0120E030E0A901C501D5
:10BA4000B4010F94099C9B01AC01C701B6010F948E
:10BA500063A29B01AC01C301B2010F9464A20F94D5
:10BA6000D5A38B8D0F94ED21FB8DFF5FFB8FF33002
:10BA700009F0BACF53CFF10180819181A281B381C6
:10BA8000F80180839183A283B38348CFEA8DEE0FC0
:10BA9000EA8FF4E02F0E311C0C5F1F4F83E0898F7B
:10BAA0008BCE609100177091011790E08A3020F0E2
:10BAB000895A9F4F0D94A49FC096FCCF84FF18C055
:10BAC0005A9A85FF17C0A49A2FB786FF15C0F8941D
:10BAD000909102019068909302012FBF87FF11C0DF
:10BAE000A39A5B9A85E08A95F1F700005B98089528
:10BAF0005A98E7CFA498E8CFF894909102019F77E5
:10BB0000EACFA398EECF0F931F93CF93DF93C82F65
:10BB1000D62F8A0160FF15C05D9A8AE18A95F1F7F8
:10BB200000C08C2F0E945E5DD1FD04C08C2F8295D9
:10BB30000E945E5DC801DF91CF911F910F910C941F
:10BB4000D6BF5D98EACFCF92DF92EF92FF92CF936C
:10BB5000DF93EC016A017B010F9444A16F3F7F4F9B
:10BB60008F4F9F4F59F4B701A601CE01DF91CF91BE
:10BB7000FF90EF90DF90CF900D9492A1DF91CF9145
:10BB8000FF90EF90DF90CF9008957F928F929F92D9
:10BB9000AF92BF92CF92DF92EF92FF920F931F93DB
:10BBA000CF93DF93CDB7DEB760970FB6F894DEBFC3
:10BBB0000FBECDBF5C016B01742E81E080937802D3
:10BBC0001F930F931F922F938FE394E69F938F936E
:10BBD0000F94FE9F81E40E94B6550F900F900F9036
:10BBE0000F900F900F90882389F08091F516909117
:10BBF000F616FC012181283709F056C040E150E0DB
:10BC000070E060E002960F94C79C5B0183E40E94A1
:10BC1000B655882309F44DC00E941E564B0175018C
:10BC2000CA14DB0408F47601C4018E0D9F1DC816EA
:10BC3000D90618F08E159F0518F446018E189F0836
:10BC400088E50E94B655882309F471C02091F51645
:10BC50003091F6162F5F3F4FCE0101965C01DC015B
:10BC6000D12CC12CF90180812F5F3F4F8823B9F17E
:10BC700090E1C916D10499F18032A1F38A3079F1AB
:10BC800090ED980F9A30C8F48295807F9F012E5FC7
:10BC90003F4F918140ED490F4A30B8F4842B8D938A
:10BCA000EFEFCE1ADE0ADECF0E948E5A0F94D5A394
:10BCB000ACCF88248A94982CB2CF9FE9980F963005
:10BCC00058F48295807F8057E1CF4FE9490F463085
:10BCD00018F49755892BE3CFD194C194D108912CB6
:10BCE000812CC814D90491F0F50161915F01C40160
:10BCF0008E0D9F1DF1E07F1631F0FC016083FFEF98
:10BD00008F1A9F0AEECF0F9484A1F9CFFF92EF9282
:10BD10001F930F939F928F9285E194E69F938F9349
:10BD20000F94FE9F0FB6F894DEBF0FBECDBF472D18
:10BD3000B401C70160960FB6F894DEBF0FBECDBF49
:10BD4000DF91CF911F910F91FF90EF90DF90CF90F7
:10BD5000BF90AF909F908F907F900D94425380E161
:10BD6000E5EFF1E1A0E9B2E001900D928A95E1F7EB
:10BD700080918E0290918F029093F4118093F31131
:10BD80008091F1119091F2119093F0118093EF1145
:10BD90008091ED118093EC118091EB1183FB88274A
:10BDA00080F98093EA118091E9118093E811089558
:10BDB000CF93DF938AEF95E10E94BC7088E394E112
:10BDC000892B51F0CAE0D5E1A397CE010E94BC7047
:10BDD00084E1C833D807C1F785E194E10E94BC70C3
:10BDE00080EF93E1DF91CF910C94BC70CF93DF9300
:10BDF000C5EFD1E120E030E048EC51E46C857D8571
:10BE00008E859F850F9464A26C877D878E879F8720
:10BE100063E373E383E590E4DF91CF910D94D085E4
:10BE200060E085EA9FE00F9460A160E08FE79CE00E
:10BE30000F9460A180E090E0A0E8BFEB80937E02C9
:10BE400090937F02A0938002B093810282E080935E
:10BE500079021092E71108958091EF119091F011FD
:10BE60002091F1113091F2112817390771F0909358
:10BE7000F2118093F11181E0809399030F94CE0F1A
:10BE80000F94F54E82E08093990308958091E71115
:10BE9000882341F080918E0290918F029093F4114B
:10BEA0008093F3110895CF92DF92EF92FF92C090AA
:10BEB000CA04D090CB04E090CC04F090CD048091E3
:10BEC000C904882309F44EC020E030E0A901C7016D
:10BED000B6010F94EDA418160CF044C02BED3FE012
:10BEE00049E450E4C701B6010F94099CA7019601EB
:10BEF0000F94099C20E030E040E85EE30F94099C39
:10BF00009B01AC0160E070E080E89FE30F9463A3C5
:10BF10006B017C016091590270915A02643671057F
:10BF2000A1F0072E000C880B990B0F94CA9B2AE0F6
:10BF300037ED43E25CE30F94099C9B01AC01C70120
:10BF4000B6010F94099C6B017C01C0921002D09243
:10BF50001102E0921202F0921302FF90EF90DF9034
:10BF6000CF900895C12CD12C80E8E82E8FE3F82ED5
:10BF7000D1CF8F929F92AF92BF92CF92DF92EF92EA
:10BF8000FF9281EF9FE00F9414496B017C018DEECD
:10BF90009FE00F9414494B015C010F94C41C2CE3E7
:10BFA00030E040E050E00F94AFA1BA01A901480D84
:10BFB000591D6A1D7B1D8DEE9FE00F9472A160914B
:10BFC000840670918506809186069091870628EEFA
:10BFD00033E040E050E00F94AFA1BA01A9014C0D4D
:10BFE0005D1D6E1D7F1D81EF9FE00F9472A10F9468
:10BFF000992010928406109285061092860610925F
:10C00000870680919412813081F46091981270912A
:10C01000991290E080E00F94FC48109299121092CF
:10C02000981210929B1210929A12FF90EF90DF904C
:10C03000CF90BF90AF909F908F9008958091E9111D
:10C040001F928F93809140031F928F93E5E8F3E056
:10C05000428153812CE3249FC001259F900D112420
:10C060009F938F9340815181249FC001259F900D04
:10C0700011249F938F9386ED94E69F938F930F9453
:10C08000FE9F8DB79EB70A960FB6F8949EBF0FBE5F
:10C090008DBF08958AE493E00D94FB1120E030E019
:10C0A00040E752E40F9463A3089510927702409101
:10C0B0003B0350913C0360913D0370913E034093DC
:10C0C0007A0250937B0260937C0270937D0290937E
:10C0D0008F0280938E028AE493E00D94FB111F93EC
:10C0E000CF93DF93182F80917A0290917B02A091D9
:10C0F0007C02B0917D0280933B0390933C03A0931C
:10C100003D03B0933E03C0918E02D0918F0284E62E
:10C1100090E090938F0280938E028AE493E00F94D4
:10C12000FB1110937702CE01DF91CF911F910895FB
:10C13000CF92DF92EF92FF920F931F93CF93DF93F3
:10C1400090E0EC01CC0FDD1FCC0FDD1FFE01EB5E9C
:10C15000F8482591359145915491FE01E657FB4FE2
:10C16000C080D180E280F3808E010B501E4EC7014B
:10C17000B6010F9464A2F801608371838283938374
:10C18000FE01E75FF84825913591459154918E0164
:10C190000C5D1D4FC701B6010F9464A2F8016083C6
:10C1A000718382839383FE01E350F9482591359191
:10C1B00045915491C85EDD4FC701B6010F9464A24A
:10C1C000688379838A839B83DF91CF911F910F913D
:10C1D000FF90EF90DF90CF90089540E050E0BA01DB
:10C1E0008DEE9FE00F9472A140E050E0BA0181EF24
:10C1F0009FE00F9472A10E94295670E060E085E0F4
:10C200009FE00F947EA170E060E083E09FE00F94D8
:10C210007EA170E060E081E09FE00F947EA170E07D
:10C2200060E08FEF9EE00F947EA170E060E083ED10
:10C230009EE00F947EA170E060E080ED9EE00F94A0
:10C240007EA140E050E0BA0188EA9CE00D9472A122
:10C25000F89488E19FE00FB6F894A8958093600069
:10C260000FBE90936000FFCF85EA9FE00F943CA142
:10C2700091E0811101C090E0892F089580919B0386
:10C28000811106C081E090915903923009F080E05D
:10C29000089580916A1381110AC08091D51181118E
:10C2A00006C081E090915903913009F080E0089533
:10C2B000CF93DF93C0910512C1111FC08091061268
:10C2C00081111CC00E943E61811118C0D091C80D1F
:10C2D000D43061F48091F1119091F211892B91F495
:10C2E0008091ED119091EE11892B61F40E944961CA
:10C2F000C82F811103C0C1E0D111C0E08C2FDF91A4
:10C30000CF910895C1E0FACF0E945861882389F047
:10C3100020E030E040E050E46091FD117091FE11AA
:10C320008091FF11909100120F9459A3881F8827C4
:10C33000881F08950E944961811118C00E943E61C2
:10C34000811114C08091E711811110C08091C80D36
:10C3500081110BC080919512811107C08091051247
:10C36000811104C080910612089581E0089580E152
:10C37000E5EFF1E1A3E9B6E001900D928A95E1F7CE
:10C3800008954F925F926F927F928F929F92AF9299
:10C39000BF92CF92DF92EF92FF920F931F93CF93B2
:10C3A000DF9300D000D01F921F92CDB7DEB720914F
:10C3B000E711222309F473C120919C03223009F470
:10C3C0006EC120919C03213011F410929C032B012B
:10C3D0003C011092E9111091EC1160918A03709167
:10C3E0008B0380918C0390918D030F94DCA36117D4
:10C3F00031F0812F90E09093EE118093ED110E9427
:10C400002C5F8091E8118093E9119091EB1180915C
:10C41000EA1181958927887089278093EB11A30100
:10C42000920160919C0270919D0280919E02909178
:10C430009F020F9463A26D837E838F839887CE01C2
:10C4400005960F9428761092400220E030E040E8F4
:10C450005FEB6091900270919102809192029091B5
:10C4600093020F9459A3811120C08091F5119091EE
:10C47000F611A091F711B091F8118093900290936A
:10C480009102A0939202B09393028091F91190913E
:10C49000FA11A091FB11B091FC118093940290933A
:10C4A0009502A0939602B0939702A3019201609126
:10C4B0009C0270919D0280919E0290919F020F9428
:10C4C00063A269837A838B839C83E090FD11F09053
:10C4D000FE110091FF1110910012209194023091F1
:10C4E000950240919602509197026091900270914E
:10C4F000910280919202909193021F921F921F923B
:10C500001F92E2E68E2EE7E29E2EE6E7AE2EE2E4F2
:10C51000BE2EFE0131966F010F948276A301920127
:10C5200060919C0270919D0280919E0290919F0269
:10C530000F9463A269837A838B839C83E090980233
:10C54000F090990200919A0210919B02209194021E
:10C55000309195024091960250919702609190021D
:10C560007091910280919202909193021F921F927A
:10C570001F921F920F948276E0909802F090990299
:10C5800000919A0210919B022091940230919502A1
:10C5900040919602509197026091900270919102A1
:10C5A00080919202909193021F921F921F921F926C
:10C5B000812C912CF8EEAF2EF2E4BF2EACE9CA2EFE
:10C5C000A2E0DA2E0F9482760F94A02211E010934D
:10C5D00040026091E2117091E31190E080E00F94CD
:10C5E000C89B60937A0270937B0280937C02909345
:10C5F0007D028091F3119091F41190938F028093BA
:10C600008E0280E1E0E9F2E0A5EFB1E101900D9248
:10C610008A95E1F70E94B761809179020FB6F8948C
:10C62000DEBF0FBECDBF811151C06091D811709196
:10C63000D9118091DA119091DB1160937E1670937D
:10C640007F1680938016909381160F9453448091A7
:10C65000D8119091D911A091DA11B091DB1180938A
:10C66000DC119093DD11A093DE11B093DF111093D4
:10C670006A1360E085EA9FE00F9460A160E08FE7B5
:10C680009CE00F9460A18BE09CE60E9493E682E020
:10C69000809379021092E71181E08093AC0D289687
:10C6A0000FB6F894DEBF0FBECDBFDF91CF911F91C3
:10C6B0000F91FF90EF90DF90CF90BF90AF909F9041
:10C6C0008F907F906F905F904F900895813089F6A2
:10C6D0008091D8119091D911A091DA11B091DB110C
:10C6E0008093D1119093D211A093D311B093D41110
:10C6F0001092DB0F1092DA0F0E946D55BACF3F9265
:10C700004F925F926F927F928F929F92AF92BF9261
:10C71000CF92DF92EF92FF920F931F93CF93DF930D
:10C720003090DC16332009F480C08B01EC0131FE1F
:10C7300054C088809980AA80BB80FB01C080D180D2
:10C74000E280F3802091B1163091B2164091B31679
:10C750005091B416C501B4010F94099C2B013C0102
:10C760002091B5163091B6164091B7165091B81673
:10C77000C701B6010F94099C9B01AC01C301B20132
:10C780000F9464A22B013C012091A9163091AA16A6
:10C790004091AB165091AC16C501B4010F94099CA1
:10C7A0004B015C012091AD163091AE164091AF1651
:10C7B0005091B016C701B6010F94099C9B01AC01C2
:10C7C000C501B4010F9464A2688379838A839B8333
:10C7D000F801408251826282738230FE26C020912D
:10C7E000D4163091D5164091D6165091D71668813F
:10C7F00079818A819B810F9464A2688379838A837B
:10C800009B832091D8163091D9164091DA16509119
:10C81000DB16F80160817181828193810F9464A29B
:10C82000F8016083718382839383DF91CF911F919D
:10C830000F91FF90EF90DF90CF90BF90AF909F90BF
:10C840008F907F906F905F904F903F9008952F92C0
:10C850003F924F925F926F927F928F929F92AF9290
:10C86000BF92CF92DF92EF92FF920F931F93CF93DD
:10C87000DF9300D000D01F921F92CDB7DEB78C019E
:10C880001B01FC0180819181A281B38189839A83FC
:10C89000AB83BC83FB0180819181A281B3818D83B5
:10C8A0009E83AF83B887BE016B5F7F4FCE01019639
:10C8B0000E947F63C980DA80EB80FC8020E030E05A
:10C8C000A901C701B6010F9459A387FF35C019828A
:10C8D0001A821B821C82FF24F3948D809E80AF807D
:10C8E000B88420E030E040E850ECC501B4010F947A
:10C8F00059A387FF35C080E090E0A0E8B0EC8D83BD
:10C900009E83AF83B887CD80DE80EF80F8848980F6
:10C910009A80AB80BC807090DC1671104CC0F8011E
:10C9200080829182A282B382F101C082D182E282AE
:10C93000F382FF24F39425C020E030E04AE753E47B
:10C94000C701B6010F94EDA4F12C181634F680E05F
:10C9500090E0AAE7B3E489839A83AB83BC83BBCF1F
:10C9600020E030E042E553E4C501B4010F94EDA4AA
:10C9700018162CF480E090E0A2E5B3E4C0CFF110EB
:10C98000C2CF8F2D28960FB6F894DEBF0FBECDBF55
:10C99000DF91CF911F910F91FF90EF90DF90CF909B
:10C9A000BF90AF909F908F907F906F905F904F90CF
:10C9B0003F902F90089570FE1CC02091D4163091A6
:10C9C000D5164091D6165091D716C501B4010F94D3
:10C9D00063A24B015C012091D8163091D916409189
:10C9E000DA165091DB16C701B6010F9463A26B01F2
:10C9F0007C0171FE9ECF2091C4163091C5164091E6
:10CA0000C6165091C716C501B4010F94099C2B019D
:10CA10003C012091C8163091C9164091CA16509118
:10CA2000CB16C701B6010F94099C9B01AC01C30151
:10CA3000B2010F9464A2F8016083718382839383AF
:10CA40002091CC163091CD164091CE165091CF1634
:10CA5000C501B4010F94099C4B015C012091D016D3
:10CA60003091D1164091D2165091D316C701B6011C
:10CA70000F94099C9B01AC01C501B4010F9464A201
:10CA8000F101608371838283938353CFCF92DF92CE
:10CA9000EF92FF92CF93DF93EC01BC016C5F7F4F6D
:10CAA0000E942764C0902C02D0902D02E0902E02AC
:10CAB000F0902F02A7019601688579858A859B856C
:10CAC0000F9459A387FF04C0C886D986EA86FB86DF
:10CAD000C0902002D0902102E0902202F090230228
:10CAE000A7019601688579858A859B850F94EDA4B9
:10CAF000181624F4C886D986EA86FB86DF91CF9182
:10CB0000FF90EF90DF90CF9008952F923F924F9239
:10CB10005F926F927F928F929F92AF92BF92CF92CD
:10CB2000DF92EF92FF920F931F93CF93DF93CDB7D6
:10CB3000DEB7A2970FB6F894DEBF0FBECDBF1C01C3
:10CB400083E996E00E9446658AE493E00F94FB1126
:10CB50004090F5115090F6116090F7117090F81117
:10CB6000C0909306D0909406E0909506F0909606BB
:10CB7000A7019601C301B2010F9459A381113FC0CF
:10CB800020919706309198064091990650919A0607
:10CB90006091F9117091FA118091FB119091FC1143
:10CBA0000F9459A381112BC020E030E040E752E4FC
:10CBB00060917A0270917B0280917C0290917D025B
:10CBC0000F9463A30F949D850E943755A2960FB6CC
:10CBD000F894DEBF0FBECDBFDF91CF911F910F91B3
:10CBE000FF90EF90DF90CF90BF90AF909F908F908D
:10CBF0007F906F905F904F903F902F90089560913D
:10CC00008E0270918F02072E000C880B990B0F94E7
:10CC1000CA9B20917A0230917B0240917C02509114
:10CC20007D020F94099C2EE333EC4EE259E30F94FE
:10CC3000099C6F83788789879A8780919C128823C3
:10CC400009F40FC1A3019201C701B6010F9463A2B9
:10CC50002B013C012091F9113091FA114091FB1107
:10CC60005091FC11609197067091980680919906F9
:10CC700090919A060F9463A26B877C878D879E871D
:10CC8000C301B2019F772B853C854D855E855F771B
:10CC90000F9464A26B017C0120E030E0A9010F94A5
:10CCA000EDA418160CF0DDC020E030E040EF51E4B8
:10CCB000C701B6010F9463A30F9442A30F94DCA3A2
:10CCC0007E836D836230710508F4CBC0211431047A
:10CCD00009F4C7C02091FD113091FE114091FF1160
:10CCE0005091001260919B0670919C0680919D0668
:10CCF00090919E060F9463A26F87788B898B9A8B95
:10CD000020910112309102124091031250910412AD
:10CD100060919F067091A0068091A1069091A20655
:10CD20000F9463A26B8B7C8B8D8B9E8BAD81BE81B0
:10CD3000CD01B0E0A0E08F8F98A3A9A3BAA32D8165
:10CD40003E812216330608F08CC0B10190E080E0ED
:10CD50000F94C89B6B017C016F8D78A189A19AA16A
:10CD60000F94C89B9B01AC01C701B6010F9463A34C
:10CD70006B017C01AC019B016B897C898D899E894B
:10CD80000F94099C9B01AC016091011270910212F9
:10CD900080910312909104120F9464A269837A83A4
:10CDA0008B839C83A70196016F85788989899A89ED
:10CDB0000F94099C2091FD113091FE114091FF11BB
:10CDC000509100120F9464A26F8B788F898F9A8F85
:10CDD000A70196016B857C858D859E850F94099CA6
:10CDE0002091F9113091FA114091FB115091FC11F1
:10CDF0000F9464A26B8F7C8F8D8F9E8FA7019601FD
:10CE0000C301B2010F94099C2091F5113091F611E4
:10CE10004091F7115091F8110F9464A23F922F9214
:10CE2000A5EFB1E1BF93AF938F809884A984BA84B2
:10CE3000DE0111966D01EF88F88C098D1A8D2B8D0E
:10CE40003C8D4D8D5E8D0F9482760F900F900F90DC
:10CE50000F908091AC0D8111B7CEBFEF2B1A3B0A1A
:10CE60006ECFE0909B06F0909C0600919D0610917D
:10CE70009E06209197063091980640919906509110
:10CE80009A06609193067091940680919506909110
:10CE900096061F921F92E5EFF1E1FF93EF938F80CB
:10CEA0009884A984BA84EFE9CE2EE6E0DE2E0F94B2
:10CEB00082760F900F900F900F9086CECF92DF92D8
:10CEC000EF92FF92CF93C090FD11D090FE11E090B1
:10CED000FF11F0900012A70196010F9464A26093D5
:10CEE000FD117093FE118093FF119093001283B196
:10CEF0009091A506911102C084FF26C085EF91E1B3
:10CF00000E94466560914E0470914F0480915004D8
:10CF1000909151040F94D0850F94A022A7019601FF
:10CF20006091FD117091FE118091FF11909100129E
:10CF30000F9463A26B017C01C701B601CF91FF90F2
:10CF4000EF90DF90CF90089515980F94A02281E084
:10CF50000F94D82CC82F65E575E585E591E40F940D
:10CF6000D0850F94A02282E00F948C22A701960115
:10CF70000F9463A26B017C018C2F0F94D82CDCCF13
:10CF80008F929F92AF92BF92CF92DF92EF92FF92D9
:10CF90004B015C01C090FD11D090FE11E090FF119B
:10CFA000F0900012AC019B01C701B6010F94EDA4F3
:10CFB00087FF11C0A5019401C701B6010F9463A2B8
:10CFC0009F77FF90EF90DF90CF90BF90AF909F90B2
:10CFD0008F900C945E67FF90EF90DF90CF90BF90A2
:10CFE000AF909F908F9008952F923F924F925F92B3
:10CFF0006F927F928F929F92AF92BF92CF92DF9269
:10D00000EF92FF920F931F93CF93DF9300D01F9265
:10D010001F92CDB7DEB7D82E2A013B01322EE9820E
:10D02000FA820B831C830F94A02281E08093051267
:10D03000FC2CE32CD31010C0ED2CDC100DC060E0F4
:10D0400070E080EA90E40E94C067FF24F394EE242D
:10D05000E3942224239401C02D2C0F94BC90809142
:10D060009C128D8310929C1282E00F948C2260930C
:10D07000FD117093FE118093FF1190930012F11037
:10D080000F946B8C81E00E946F608C010E94B761ED
:10D0900010927A0210927B0210927C0210927D0212
:10D0A000222019F080E00F941C55EE2019F081E049
:10D0B0000F941C55DD20E9F0411451046104710402
:10D0C000C1F0C301B2010F94CA9B9B01AC016091F6
:10D0D0008A0470918B0480918C0490918D040F943C
:10D0E00064A26093F5117093F6118093F7119093F9
:10D0F000F811332001F189819A81AB81BC810097BD
:10D10000A105B105C1F0BC01CD010F94CA9B9B01E3
:10D11000AC0160918E0470918F0480919004909185
:10D1200091040F9464A26093F9117093FA118093A3
:10D13000FB119093FC11FF2009F499C060E070E0AE
:10D1400080EA90E40E94C0678091A306811102C02A
:10D150000F941C558091A406811103C081E00F94A7
:10D160001C550F942191E3E5F9E885919591A591DE
:10D17000B491EFE4F9E8459155916591749140932C
:10D180009306509394066093950670939606809349
:10D19000970690939806A0939906B0939A0667E92C
:10D1A00076E083E996E00E947F630F94839020E00D
:10D1B00030E040E850EC60919706709198068091BD
:10D1C000990690919A060F9459A387FF0CC080E0AE
:10D1D00090E0A0E8B0EC8093970690939806A09317
:10D1E0009906B0939A0680E090E0A6E1B3E48093BC
:10D1F0007A0290937B02A0937C02B0937D021092FE
:10D2000077020F94908460917A0270917B028091F2
:10D210007C0290917D020F949D850F94A0228091B5
:10D22000930690919406A0919506B09196068093EE
:10D23000F5119093F611A093F711B093F811809126
:10D24000970690919806A0919906B0919A068093BE
:10D25000F9119093FA11A093FB11B093FC1181E0A6
:10D26000809377020F94F42C82E00F941C55CC200D
:10D27000E9F081149104A104B104C1F0C501B40125
:10D280000F94CA9B9B01AC0160919204709193042E
:10D2900080919404909195040F9464A26093FD1181
:10D2A0007093FE118093FF11909300120F9490845D
:10D2B000C8010E9455600F94F42C0F9421910F9493
:10D2C000BF8ED11007C0311005C08B8D811102C0F7
:10D2D000CC2039F1F11025C09D81992311F181E015
:10D2E00080939C120F948C226B017C0180E00F9440
:10D2F0008C22A70196010F9468619B01AC0160919B
:10D30000FD117091FE118091FF11909100120F9408
:10D3100063A26093FD117093FE118093FF119093AF
:10D32000001284E10F945F990F94A02210920512CD
:10D330000F900F900F900F900F90DF91CF911F9152
:10D340000F91FF90EF90DF90CF90BF90AF909F90A4
:10D350008F907F906F905F904F903F902F900895A7
:10D36000E3E3F3E09FE781918F3731F0DF0111971D
:10D3700087FF07C08F778C9383E0EB33F80799F72B
:10D3800008959C93F9CF90915B02981710F48093C5
:10D390005B0280915C02882339F0E091D203F09126
:10D3A000D303309709F019940895CF93DF93CDB745
:10D3B000DEB7AE014A5F5F4FFA0161917191AF0133
:10D3C00080EC93E00F9483A0DF91CF91089560ECFF
:10D3D00073E00D94D49F60EC73E0082E000C990B61
:10D3E0000D94A49FCF93C82FC15020F080E20E94DB
:10D3F000EB69FACFCF910895CF93C82F862F643071
:10D4000008F083E0809332030E9441558C0F809393
:10D41000310344E650E060E08068CF910C94835D76
:10D42000CF93DF93EA010E94FC6960EC73E0CE01C8
:10D43000DF91CF910D94D49FCF93C42F0E94FC69AC
:10D4400060EC73E08C2FCC0F990BCF910D94A49FBF
:10D4500060E080E00E94FC6910923103089540E48E
:10D4600056E060E081E00E94835D109232031092EA
:10D47000310348E050E06FE770E083E393E00D9400
:10D480006EA790915C02981709F180935C02882343
:10D49000E9F010920705109206051092110681EB33
:10D4A00093E00F94FB110F94CE0F61507109810925
:10D4B00091096093930370939403809395039093E1
:10D4C00096030E942F6A82E00C94C3690895CF935B
:10D4D000C82F109232031092310348E050E06FE7FA
:10D4E00070E083E393E00F946EA744E951E162E0BA
:10D4F00080E30E94835D46E950E062E080E30E94A1
:10D50000835D46E950E062E080E30E94835D46E986
:10D5100050E062E080E20E94835D8091CE0344E6A9
:10D5200050E060E080620E94835D84E0809330037D
:10D5300044E650E060E08CE00E94835DC1110E94EF
:10D540002F6A44E650E060E086E0CF910C94835D62
:10D5500081E00C94676ACF92DF92FF920F931F9342
:10D56000CF93DF9300D000D01F921F92CDB7DEB7CC
:10D570008A30D9F480913203843018F08FEF809391
:10D580003203609132036F5F80E00E94FC6928964D
:10D590000FB6F894DEBF0FBECDBFDF91CF911F91C4
:10D5A0000F91FF90DF90CF90089590E8980F44E698
:10D5B00050E061E09A3408F5482F4058550B9A0125
:10D5C00096E0929FA001939F500D1124FA01E45F11
:10D5D000FA48F490E3E3F3E030E020E09FEF61915C
:10D5E000782F76277F7789F4F901ED5CFC4F8083F3
:10D5F000F22E44E650E061E08F2D0E94835D809121
:10D6000031038F5F80933103C2CF6F3709F03CC085
:10D61000F901ED5CFC4F8083922FF92EFA01E95F4E
:10D62000FA488E010F5F1F4FD801959188E0182EA0
:10D6300010FE05900294802D9795881F8D931A9463
:10D64000B9F7BF2DE8E0BE02C001112444E650E066
:10D6500060E080640E94835D6E01F9E0CF0ED11C12
:10D6600044E650E061E0D8018D918D010E94835D18
:10D67000C016D106A9F78091310344E650E060E07E
:10D6800080680E94835DB5CF67FF922F2F5F3F4F69
:10D690002830310509F0A3CF9F3F09F0BECFA9CFB5
:10D6A0008F929F92AF92BF92EF92FF920F931F9330
:10D6B000CF93DF93CDB7DEB7A0970FB6F894DEBF58
:10D6C0000FBECDBF611571058105910599F480E309
:10D6D000A0960FB6F894DEBF0FBECDBFDF91CF91FD
:10D6E0001F910F91FF90EF90BF90AF909F908F9000
:10D6F0000C94AB6A00E0842E912CB12CA12C9E01DD
:10D700002F5F3F4F7901A50194010F94AFA1F7015D
:10D71000E00FF11D6083B901CA010F5F611571054A
:10D720008105910581F70E0D1F2D111DE016F106E3
:10D7300059F0F80182918F018A3020F4805D0E94B7
:10D74000AB6AF4CF895CFBCFA0960FB6F894DEBF2E
:10D750000FBECDBFDF91CF911F910F91FF90EF9042
:10D76000BF90AF909F908F900895CF92DF92EF92ED
:10D77000FF926B017C01F7FE0BC08DE20E94AB6A49
:10D78000F094E094D094C094C11CD11CE11CF11C15
:10D790004AE0C701B601FF90EF90DF90CF900C9464
:10D7A000506B0F931F93CF938C01C62FCC2359F04E
:10D7B000F8012491222339F00F5F1F4F84910E94BA
:10D7C000AB6AC150F3CF8C2F0E94F2698C2FCF919E
:10D7D0001F910F9108950F931F93CF938C01C62F24
:10D7E000CC2349F0F80181918F01882321F00E9418
:10D7F000AB6AC150F5CF8C2F0E94F2698C2FCF916C
:10D800001F910F910895CF93DF93EC0189918823A5
:10D8100019F00E94AB6AFACFDF91CF9108950E9470
:10D82000AB6A90E080E008951092630310921406B2
:10D830000895CF9380916303C1E0811104C0C0E0DB
:10D840008C2FCF9108950E94146CFACF8EEF9FE039
:10D850000F943CA18E3F39F091E020912F032813C3
:10D8600090E0892F089580E0089510922F036EEFC5
:10D870008EEF9FE00D9460A1853728E6920709F4AA
:10D8800059C0F8F48E3625E6920709F459C050F4D1
:10D89000833723E69207B1F185369446B1F184E5EA
:10D8A00094E60895823726E6920791F1823728E6BA
:10D8B000920709F442C08337954689F78BEA94E6CC
:10D8C00008958C3620E7920731F170F48C362EE6FD
:10D8D000920721F18F362EE6920731F1843799466F
:10D8E000F1F689E994E608958B3623E79207F9F07B
:10D8F000863723E79207A9F08F36924781F687E5AE
:10D9000094E608958BEB94E6089583EB94E60895EE
:10D9100082EA94E6089582E994E6089587E894E619
:10D9200008958FE794E6089589E794E608958EE6D2
:10D9300094E6089587E694E608958EE594E60895C2
:10D9400083EC94E60895E3E0F5E785919591A59140
:10D95000B4918F3F9F4FAF4FBF4FB1F020E031E008
:10D9600081E0F9014591559165917491453A5A4587
:10D97000644B7B4409F00895F90134964591549124
:10D98000240F351F8F5FEDCF81E008950F931F9314
:10D99000811113C010922E0310922D0310922F03A9
:10D9A00090912F0398135CC0682F8EEF9FE00F9427
:10D9B00060A181E01F910F910895813089F7E0E027
:10D9C000F1E04591559165917491453A5A45644B02
:10D9D0007B4431F7E4E0F1E0A591B491E8E0F1E0B7
:10D9E0006591749150E040E030E020E0A417B50765
:10D9F00029F5261B370B3227232732276217730797
:10DA000009F0CECFECE0F1E005911591259134912C
:10DA1000E3E0F5E745915591659174910417150779
:10DA20002607370709F0BCCF20E031E030932E0302
:10DA300020932D0391E090932F03B2CFFA01E05091
:10DA4000FF4FE491F0E098E040FD90E002C0EE0F5F
:10DA5000FF1F9A95E2F72E0F3F1F4F5F5F4FC6CF14
:10DA600080E0A8CF20912F03211104C0FC01329641
:10DA7000CF01089540912D0350912E03411551057A
:10DA8000A9F3FC01259134912F3F320779F3F90175
:10DA90003896EE0FFF1FE40FF51F25913491FA0120
:10DAA000E20FF31F2491222309F3E2CFCF93DF93F8
:10DAB000EC0120E030E04CE852E4609101127091FA
:10DAC000021280910312909104120F9464A2609349
:10DAD000011270930212809303129093041260E07B
:10DAE00070E080EA91E40F94D0850E94F65E0E9477
:10DAF0002F6A84EC9AE50E94326DAC0160E080E010
:10DB00000E94106A8881882339F061E080E00E94D9
:10DB1000FC69CE010E94036C86EB99E30E94326D92
:10DB2000AC0162E080E00E94106A83E49BE20F9403
:10DB30003F0CDF91CF910D94A0220F94E8418F3FCD
:10DB400011F180E00E94416A0E942F6A80E297E50D
:10DB50000E94326DAC0161E080E00E94106A80E2B8
:10DB60000E94AB6A0F94E841682F70E06F5F7F4FAF
:10DB7000072E000C880B990B0E94B56B0F94F36B6A
:10DB800081E00C94416A08951F920F920FB60F9294
:10DB900011240BB60F922F938F939F93EF93FF93C4
:10DBA000E0912803E830E8F4F0E08827E552F249F4
:10DBB0008F4F0D944CA2E36DFD6D086E166E2C6EAA
:10DBC000356E586E6A6E8091920681110AC08091FE
:10DBD0005B06880F80932703882319F081E08093E8
:10DBE0002803FF91EF919F918F912F910F900BBE82
:10DBF0000F900FBE0F901F901895809126038F5F96
:10DC00008093260390912703981758F382E0E7CF7B
:10DC100083E0809328038FE0809325038FEF86BDF8
:10DC200081E085BD84B58F7E84BDDBCF80912503E7
:10DC30008295807F819588BD80912503882321F07E
:10DC4000815080932503CDCF84E0809328038FEF0C
:10DC500088BD8EEF86BDC5CF85E0809328038FEF0A
:10DC600088BD86BD82E085BDBCCF2FEF28BD8091E9
:10DC700092068111B6CF809126038F5F8093260391
:10DC800090912703891708F4ACCF80915B0690E050
:10DC90008F3791050CF0A5CF86E0809328038FE0A5
:10DCA0008093250326BD81E085BD84B58061BCCF0E
:10DCB000809125038295807F819588BD8091250381
:10DCC0008111BECF87E08093280380E886BD8FEF67
:10DCD00088BD87CF1092280380E886BD8FEF88BD6E
:10DCE000C1CFCF93DF93EC0187E69FE00F943CA177
:10DCF00091E0811101C090E081E02881211101C0F3
:10DD000080E08913988387E09FE00F943CA191E025
:10DD1000811101C090E0998385ED9EE00F943CA1B4
:10DD200091E0811101C090E09A8387E49DE00F9417
:10DD30003CA18F3F21F08887DF91CF91089518860D
:10DD4000FBCFCF93C82F682F87E69FE00F9460A189
:10DD5000CC2319F0CF910D949B5351985998109260
:10DD60008416CF910895109284030F94CE0F609380
:10DD70008D1670938E1680938F169093901608953B
:10DD80008093240380FD1CC0109240032091400327
:10DD90008FEF820F8E3FE8F08091A000877F809305
:10DDA000A0001092AD001092AC009FB7222361F04A
:10DDB000F894809102018062809302019FBF0895D0
:10DDC0008FEF80934003E2CFF894809102018F7D22
:10DDD000F3CFEFB7F8948091A00088608093A00003
:10DDE00030E0809172004FEF50E081FF04C040911D
:10DDF000A8005091A900249FC001259F900D349F39
:10DE0000900D11246FEF70E00F9405A27093AD0098
:10DE10006093AC00EFBF08951F93CF93DF93D09131
:10DE20002403D1FD1DC010919A03C1E020E030E031
:10DE300048E452E46091C40D7091C50D8091C60D07
:10DE40009091C70D0F94EDA418160CF0C0E0DE7F82
:10DE5000CD2B81E0111101C080E0C82BC0932403B9
:10DE600080912403DF91CF911F910C94C06EEF92AB
:10DE7000FF920F931F93CF93DF93EC018B017A01F5
:10DE80000E949B5581110BC0A801BE01C701DF9103
:10DE9000CF911F910F91FF90EF900D9450A1DF91C2
:10DEA000CF911F910F91FF90EF9008950F931F93C3
:10DEB000CF93DF938C01D62FC72F0F944AA18F3FAA
:10DEC000980739F46D2F7C2FC8010F949AA18D2FDC
:10DED0009C2FDF91CF911F910F9108950F931F9366
:10DEE000CF938C01C62F0F943CA18F3F29F46C2F48
:10DEF000C8010F9484A18C2FCF911F910F91089589
:10DF0000CF93DF93EC010F944AA1BC016F5F7F4F69
:10DF1000CE01DF91CF910D949AA1CF93DF93EC01C5
:10DF20000F943CA161E0680FCE01DF91CF910D9479
:10DF300084A12BE0829FC0011124805B924F0F943B
:10DF40004AA121E0019609F420E0822F0895CF93A1
:10DF5000DF93C82FD8E0CF5FC8300CF0C0E08C2F23
:10DF60000E94996F811103C0D150A9F7CFEF8C2F78
:10DF7000DF91CF91089581EA9DE00F943CA10E942A
:10DF8000A76F87FD05C0682F81EA9DE00D9460A111
:10DF900008950F931F93CF93C82F8B0166EB74E7FF
:10DFA000823070F06FEA74E7843050F067EA74E70B
:10DFB000843031F06FE974E7853011F068E974E777
:10DFC000C8010F94F39E8CEF8C0F823028F0C17043
:10DFD000CF5CF801C6831782CF911F910F910895EE
:10DFE00061E080EC9FE00F9460A160E08FEB9FE028
:10DFF0000F9460A160E08EEB9FE00F9460A160E061
:10E000008DEB9FE00F9460A160E08CEB9FE00D949E
:10E0100060A1CF93C82F82958F700E94515D8C2F85
:10E020008F70CF910C94515D4091CF115091D011D0
:10E0300090E080E041155105B1F12091CB11309174
:10E04000CC1190E080E0F901E252F04FA081A230C3
:10E0500021F461817281860F971F4150510919F196
:10E06000F901EF51F04FA1919F012E5D3F40A111A9
:10E07000FACFF901E252F04F2D3EA1E03A0730F419
:10E08000A191A111E0CF2F5F3F4FF6CF2D3EE1E0F0
:10E090003E07C9F6EEEDFFE09F012E5D3F40A191E6
:10E0A000AA23D1F3D0CF08958091CF119091D011B0
:10E0B000181619060CF043C001979093D011809365
:10E0C000CF11892BA1F48091DA0F9091DB0F892B6E
:10E0D00021F41092DD0F1092DC0F8091DC0F9091F3
:10E0E000DD0F9093CC118093CB1181E00895809146
:10E0F000CB119091CC110396FC01E252F04F20819C
:10E1000001962111F9CFFC01E252F04F8D3E21E042
:10E11000920740F441919C012F5F3F4F4111E1CFA5
:10E12000C901F4CFEEEDFFE08D3E21E09207C9F684
:10E13000CF018E5D9F4021912223D1F3D2CF80E089
:10E140000895FC0120E03EE2DB014D91BD0140322B
:10E1500049F0283011F430833196DB0111974C914E
:10E16000408331962F5F2B3079F71082089540E07D
:10E1700050E0BA010D949339FC01238121110D94D3
:10E18000F26F089590910405911107C09091C0001D
:10E1900095FFFCCF8093C6000895913031F49091A3
:10E1A000C80095FFFCCF8093CE0008950E94C270F6
:10E1B00090E080E00895CF93DF93EC01FE0184911D
:10E1C000882321F00E94C2702196F8CFDF91CF9171
:10E1D0000895CF92DF92EF92FF92C090C40DD0903D
:10E1E000C50DE090C60DF090C70D89E099E70E943B
:10E1F000DB7042E0C701B6010F94A99881E099E76E
:10E200000E94DB7060918A0370918B0380918C0374
:10E2100090918D0341E00F94A998FF90EF90DF90CB
:10E22000CF900D945C994F925F926F927F928F92F4
:10E230009F92AF92BF92CF92DF92EF92FF920F9395
:10E240001F93CF93DF93CC24CA94DC2C76010EEA83
:10E250001FE093E2892E912CA12CB12C412C512C42
:10E260003201D0E0C0E08FEFC81609F45DC0C801EC
:10E270000F944AA1EC01BC01990F880B990B0F94E4
:10E28000CA9B20913E0430913F044091400450913C
:10E2900041040F9463A32B013C01C701B6010F9405
:10E2A00002988DE598E70E94DB70C501B4010F94D8
:10E2B00002988DE598E70E94DB70BE010D2E000CE0
:10E2C000880B990B0F9402988DE598E70E94DB70FC
:10E2D00020E030E04AE754E4C301B2010F94099C06
:10E2E0000F94E34185E0880E911CA11CB11C0E5FC8
:10E2F0001F4F8FEFC81AD80AE80AF80A0A3B8FE0C6
:10E30000180709F0B0CFDF91CF911F910F91FF90C7
:10E31000EF90DF90CF90BF90AF909F908F907F90C5
:10E320006F905F904F9008958DED9DE30E94DB709C
:10E33000B8CF882371F181E598E70E94DB70609186
:10E34000231270E090E080E00F94029880912312F5
:10E350008430D8F0109223128CE498E70E94DB708E
:10E360008091231290E00F9400428091231220911B
:10E37000EF113091F0113093F2112093F1110E94BE
:10E3800005F70E94F65E0D94A0228F5F8093231202
:10E39000E3CF86E89EE30E94326D70E060E00E9469
:10E3A000E2BCE5CFCF93DF9389E498E70E94DB706E
:10E3B000C5EFD1E1688179818A819B8142E00F9428
:10E3C000A99885E498E70E94DB706C817D818E813D
:10E3D0009F8142E00F94A99881E498E70E94DB7046
:10E3E000688579858A859B8542E00F94A9988DE39D
:10E3F00098E70E94DB706C857D858E859F8542E065
:10E400000F94A9988BEC94E60E94DB7080E00F9447
:10E410007E220F94CA9BC2E3D4E02C813D814E81C1
:10E420005F810F9463A342E00F94A99889E398E772
:10E430000E94DB7081E00F947E220F94CA9B288596
:10E4400039854A855B850F9463A342E00F94A998B0
:10E4500085E398E70E94DB7082E00F947E220F94A0
:10E46000CA9B2C853D854E855F850F9463A342E052
:10E470000F94A99881E398E70E94DB7083E00F94E2
:10E480007E220F94CA9B288939894A895B890F9417
:10E4900063A3DF91CF910D94E34180E497E70E945D
:10E4A000DB706091C40D7091C50D8091C60D909187
:10E4B000C70D41E00F94A9988DE397E70E94DB70A8
:10E4C0006091F1117091F211072E000C880B990BDD
:10E4D0000F94CA9B41E00F94A99889E397E70E94A3
:10E4E000DB7060918A0370918B0380918C03909113
:10E4F0008D0341E00F94A99886E397E70E94DB70B3
:10E500006091ED117091EE11072E000C880B990BA4
:10E510000F94CA9B41E00F94A99881E397E70E946A
:10E52000DB706091C40D7091C50D8091C60D909106
:10E53000C70D41E00F94A9988EE297E70E94DB7027
:10E540006091F1117091F211072E000C880B990B5C
:10E550000F94CA9B41E00F94A9988AE297E70E9422
:10E56000DB706091620670E090E080E00F940298AA
:10E5700085E297E70E94DB7060915B0670E090E0B7
:10E5800080E00F94029881E297E70E94DB7060912F
:10E590008E0670918F06809190069091910641E0D1
:10E5A0000F94A9980D945C990E94DB700D945C996E
:10E5B0008F929F92AF92BF92CF92DF92EF92FF9293
:10E5C0000F94CE0F6B017C0120913202222309F1BE
:10E5D000409178024130E9F0809114029091150247
:10E5E000A0911602B091170246015701881A990AA4
:10E5F000AA0ABB0A30E0A8EEB3E00F94DCA18616AD
:10E600009706A806B9066CF0443031F19CF442300C
:10E61000D4F4C0921402D0921502E0921602F09245
:10E620001702FF90EF90DF90CF90BF90AF909F9038
:10E630008F900895453069F787E79EE90E94DB7067
:10E640008CE099E706C087E79EE90E94DB7089E3CA
:10E6500099E70E94D472DDCF87E79EE90E94DB70C4
:10E6600083E299E7F6CFCF9381EA9DE00F943CA136
:10E67000CBE08C9FC0011124805B924F0F944AA184
:10E680008156904F803A9F40C8F088ED98E70E94ED
:10E69000D47281EA9DE00F943CA18C9FC0011124AB
:10E6A00070E060E0805B924F0F949AA18BE998E74D
:10E6B0000F947B0B81E0CF910C94416ACF91089528
:10E6C000EC01F8940F94B912179A1092A306169AB7
:10E6D0001092A406149A8AE59EE90E94DB708CE7EA
:10E6E00098E70E94D472209779F0CE010E94D472EC
:10E6F000BE0185E99CE00F949AA162E484E99CE064
:10E700000F9484A10E942861C4E7D8E7F1CF8AE47E
:10E7100093E00F94FB118091CF119091D011892B30
:10E7200079F0E091CB11F091CC11E252F04F808161
:10E73000813011F0863021F485ED99E60C94D47285
:10E7400008958091CF119091D011892B29F00E94CA
:10E7500087730E945470F5CF1092CC111092CB1198
:10E760001092DD0F1092DC0F81E08093E611089586
:10E77000EF92FF920F931F93CF93DF9380919C12A0
:10E78000882389F186E098E70E94D47280EF97E7AA
:10E790000E94D4728FED97E70E94D472C7E0DCE14B
:10E7A000C15058F1CD9F7001112401E010E08CEDB3
:10E7B00097E70E94DB70F801EE0FFF1FEE0FFF1FBF
:10E7C000EE0DFF1DE756FD4E6081718182819381C0
:10E7D00045E00F94A9980F5F1F4F0830110539F7D6
:10E7E0000F945C99DDCF83E198E7DF91CF911F9182
:10E7F0000F91FF90EF900C94D472DF91CF911F9105
:10E800000F91FF90EF900895CF92DF92EF92FF92D9
:10E810006B017C01C0922903D0922A03E0922B0362
:10E82000F0922C03809145038230B1F420E030E077
:10E8300040E950E4C7010F9459A387FF14C08091A9
:10E84000620490916304A0916404B0916504803DDA
:10E850009740A105B10520F5C701B601FF90EF90E3
:10E86000DF90CF9008952AE939E949E95EE3C701CD
:10E87000B6010F9459A387FF0AC020E030E048E3B7
:10E8800051E4C701B6010F94099C6B017C018AEE2B
:10E8900094E70E94DB70C701B6010F94E341DCCF1F
:10E8A0002AE939E949E95EE3C701B6010F9459A3A2
:10E8B00087FDE3CF20E030E040E85EE3C701B6012A
:10E8C0000F94099C20E030E048E550E40F9464A2E6
:10E8D000DCCFCF92DF92EF92FF92CF9390914503DE
:10E8E0009817B9F1C82FC0902903D0902A03E0905F
:10E8F0002B03F0902C0320E030E0A901C701B60102
:10E900000F9459A3882341F0C0928604D0928704C3
:10E91000E0928804F09289048DEC94E70E94DB7009
:10E92000C13011F1E0F0C23011F1C09345036091A4
:10E9300086047091870480918804909189040E94D4
:10E940000474609386047093870480938804909382
:10E950008904CF91FF90EF90DF90CF90089585ECE0
:10E9600094E70E94D472E1CF81EC94E7FACF8DEB6B
:10E9700094E7F7CF0F94A022179AE3EAF6E010820B
:10E98000169A1182149A80E00E9469748FEF9FEFAB
:10E9900090937502809374022FEF209371029093ED
:10E9A0003E0280933D0220933F0290937302809336
:10E9B000720290933C0280933B020895182FF894C2
:10E9C000CDB7DEB700D0CF90DF90EF9088E199E22D
:10E9D0000FB6F894A895809360000FBE90936000E6
:10E9E0009FB7F894E2E0F1E08081886080839FBF68
:10E9F0000F94B9128CE794E70E94D47284E794E7ED
:10EA00000E94DB70612F70E090E080E04AE00F949C
:10EA10008C9780E794E70E94DB708E2DB60190E022
:10EA200040E10F948C978CE694E70E94DB70BE0166
:10EA300090E080E040E10F948C970F945C9940E067
:10EA400060E072E290E080E00F94425385ED99E639
:10EA50000E94D4720E942861C82F9FB7F8948091B9
:10EA600002018460809302019FBF6C2F83E09DE0D0
:10EA70000F9460A180917C06882319F08C2F0E944E
:10EA8000DE740E9428611F920F920FB60F9211241C
:10EA900083E00E942C751F920F920FB60F921124E3
:10EAA00082E00E942C7541ED50E06BE973E782E350
:10EAB00094E00F94D69E0F94F5750F94F4180E946D
:10EAC000535F87E79EE90E94DB7089E793E70C9428
:10EAD000D47244E050E064E170E082E394E00F948B
:10EAE0002CA143E050E06BE973E782E394E00F94DC
:10EAF0001B9F892B09F05DC0EFE5F4E74591559127
:10EB00006591749188ED90E00E94A35DE3E6F4E7DF
:10EB100045915591659174918CED90E00E94A35DB3
:10EB2000E7E6F4E7649180EE90E00E946E6FE8E61D
:10EB3000F4E76591749181EE90E00E94566FEAE6E9
:10EB4000F4E76591749183EE90E00E94566FEBE5D7
:10EB5000F4E7459155916591749184ED90E00E94A0
:10EB6000A35D47E354E760E170E080EB90E00E9432
:10EB7000376F47E454E760E170E080EC90E00E947A
:10EB8000376F41ED50E064E170E082E394E00F9470
:10EB90002CA10E94535F0F94F5750F94F41887E72A
:10EBA0009EE90E94DB708FE593E70E94D47281E0BA
:10EBB00008950E94537564E070E084E190E00E9443
:10EBC0009B5591E0892708956BE973E782E394E010
:10EBD0000F94F39E41ED50E064E170E082E394E035
:10EBE0000F9450A187E79EE90E94DB708FE493E7C2
:10EBF0000C94D4722F923F924F925F926F927F92B9
:10EC00008F929F92AF92BF92CF92DF92EF92FF923C
:10EC10000F931F93CF93DF93CDB7DEB7A0970FB6B7
:10EC2000F894DEBF0FBECDBF8FE590E00E9447563F
:10EC3000882309F4A1C00E944B558F37910561F4D8
:10EC40008091B1059091B2059093B0058093AF0586
:10EC500080E493E70E94D4726E014FE1C40ED11C90
:10EC6000992493940E944B55181619060CF078C0FD
:10EC70008091E711882329F00E943E61882309F4DE
:10EC80006FC08091610381116BC02091B1053091FB
:10EC9000B2058091AF059091B0058217930711F3EB
:10ECA000F901E15DFA4F80812F5F3F4F2F773327C6
:10ECB0003093B2052093B1058F3F09F079C0809160
:10ECC0001B03882309F471C090921A0310921B034E
:10ECD0001F8E18A280901E03882021F280911C03B1
:10ECE0008F8FF1E0F81518F480911D0388A310921E
:10ECF0001E031601822D8C19881508F0B3CFF1017F
:10ED000011911F0181E293E00F94301017FDF2CFB3
:10ED10008091DA0F9091DB0F1A3009F44BC11D304E
:10ED200009F448C18F3591050CF049C11B3311F42A
:10ED300090922003209120032111DCCF9C012F5FB2
:10ED40003F4F3093DB0F2093DA0F2091DC0F30918F
:10ED5000DD0F2252304F820F931FFC011383CACF65
:10ED60008091DA0F9091DB0F181619060CF451C23E
:10ED700080916A13811167C2A0960FB6F894DEBF26
:10ED80000FBECDBFDF91CF911F910F91FF90EF90FC
:10ED9000DF90CF90BF90AF909F908F907F906F90BB
:10EDA0005F904F903F902F90089590921B0390CFCB
:10EDB00090911A03992309F458C0893FE9F170F53D
:10EDC000863F09F44AC0873F09F443C08BE093E7CC
:10EDD0000E94DB7086E093E70E94DB7010911903BC
:10EDE00082E093E710FD02C08DEF92E70E94DB7096
:10EDF000012F027088EF92E711FD02C083EF92E7C6
:10EE00000E94DB7082EF92E70E94D472002349F1E6
:10EE100085E480930B0210921A035ACF8A3F41F087
:10EE20008B3FA1F680911903816080931903CECFA7
:10EE3000809119038E7FF9CF10921E0310921A034E
:10EE4000109219031092180310921B0310921703CB
:10EE5000BDCF809119038260E8CF809119038D7F27
:10EE6000E4CF90E290930B02D6CF90911B033091A8
:10EE70001903992331F1E0911E0330FF49C020911D
:10EE80001703222309F440C091E09E0F90931E03C4
:10EE9000AE2FB0E0A45EBC4FFFEFFC93409118038F
:10EEA000442351F0EE5FE0931E03E92FF0E0E45EAF
:10EEB000FC4F4083109218032150209317031092A7
:10EEC0001B03E0911E0330FF6CC090911703992340
:10EED00049F121E02E0F20931E03AE2FB0E0A45E77
:10EEE000BC4F8C9380911803882351F0EE5FE09320
:10EEF0001E03E22FF0E0E45EFC4F808310921803C3
:10EF0000915090931703E4CE42E040931703D7CF7C
:10EF100091E09E0F90931E03F0E0E45EFC4F9FEFA4
:10EF20009083CDCFA82FAF7030E021E0AF3029F033
:10EF3000B0E0A050BE4F3C9120E0482F407F403FC2
:10EF400059F4226020FF13C09092170321FF0CC0D8
:10EF5000E2E0E0931703BCCE82958F70A82FB0E05B
:10EF6000A050BE4F9C91EECF90931803B1CE81E09C
:10EF70008E0F80931E03AE2FB0E0A45EBC4F3C9377
:10EF80003A3009F4A5CE21FF03C090921703A0CE1A
:10EF9000EE5FE0931E03E82FF0E0E45EFC4F908309
:10EFA00097CE91E09E0F90931E03F0E0E45EFC4F3D
:10EFB00080838ECE009719F410922003DDCE00914D
:10EFC000DC0F1091DD0F0F51104F800F911FFC01CE
:10EFD00010821A830983809120038111FDC0F801FA
:10EFE00080818E3409F084C04AE050E0BE016F5F3A
:10EFF0007F4FC80101960F94C79C2B013C01E9800B
:10F00000FA80F7018081803231F4FFEFEF1AFF0AB6
:10F01000FA82E982F4CF8091D1119091D211A0911E
:10F02000D311B091D4110196A11DB11D8415950580
:10F03000A605B70549F044E050E06BE373E7C7016C
:10F040000F941B9F892BA1F46AE270E0C7010F9413
:10F0500093A79093F6168093F516009709F441C094
:10F06000F801F12C8E179F07F1F02191F226FACFCB
:10F070008AE59EE90E94DB7082EE93E60E94DB70D7
:10F080006091D1117091D2118091D3119091D411CE
:10F090000F9402980F945C990E946D551092DB0FAB
:10F0A0001092DA0F69CE0E94D855F816190639F079
:10F0B0008AE59EE90E94DB7083EC93E6DFCFE09166
:10F0C000F516F091F6161082E980FA8066E373E790
:10F0D000C7010F94EA9E892B39F589E296E60E94D2
:10F0E00060738AE59EE90E94DB7089E993E6C6CFEA
:10F0F00089819A81FC012081203221F401969A8332
:10F100008983F6CF6AE270E00F9493A7892B39F0D8
:10F110008AE59EE90E94DB708FE693E6AFCF442438
:10F120004A94542C3201D0CF44E050E061E373E7BD
:10F13000C7010F941B9F5C01F7018081873481F424
:10F140008091CB0D853061F085ED91E10F94301009
:10F15000F6E0F093CB0D60E085EA9FE00F9460A1AC
:10F16000AB2821F08091CE11811198CF26E077FC59
:10F1700021E08091DC0F9091DD0FFC01E252F04F15
:10F18000208349815A81F801DA0140175107A1F51E
:10F1900001900020E9F79F01201B310B0396280FF7
:10F1A000391F2D3EF1E03F0779F13093DD0F2093B9
:10F1B000DC0F8091CF119091D01101969093D011D6
:10F1C0008093CF1177FC08C04092D1115092D21198
:10F1D0006092D3117092D4111092DB0F1092DA0F5B
:10F1E0000E944B55892B09F4C7CD8FE590E00E9412
:10F1F000475681117FCDC0CD6D9161939D01241B38
:10F20000350B6111F9CFCACF1092DD0F1092DC0FD0
:10F21000D0CF8091CA0D60E273E0811102C060ED31
:10F2200077E081E293E00F940110882309F4A0CDE8
:10F23000109220031092DB0F1092DA0F86E293E710
:10F240000E94D47299CD8091FD15882309F494CD44
:10F250008091DA0F9091DB0F892B09F08DCD809191
:10F26000CF119091D011892B11F410921F0312E04D
:10F2700001E040917E1650917F166091801670914A
:10F2800081168091771690917816A0917916B09199
:10F290007A16481759076A077B0708F0C1C08091A2
:10F2A0001F038111BDC00F942B494091021650914C
:10F2B0000316609104167091051640937E165093C4
:10F2C0007F1660938016709381162091DA0F30912B
:10F2D000DB0F8A3061F08D3051F0833209F487C042
:10F2E0002F35310524F48F3F980709F087C0211589
:10F2F000310509F441CD8091FD15811103C040E035
:10F3000050E0BA018091DC119091DD11481B590B3E
:10F31000A091DC0FB091DD0FFD01E252F04F1083A0
:10F320004183528313962252304FF901EA0FFB1F9B
:10F330001082A252B04FFD0101900020E9F73197F1
:10F34000EA1BFB0BF8948091CF119091D01101969C
:10F350009093D0118093CF11EC5F8091DC0F90914E
:10F36000DD0FE80FF92FF11DF093DD0FE093DC0FB7
:10F370008091FD15882309F43DC080917E169091FF
:10F380007F16A0918016B09181168093DC11909326
:10F39000DD11A093DE11B093DF11ED3EF14021F4B9
:10F3A0001092DD0F1092DC0F7894109220031092CF
:10F3B000DB0F1092DA0F40917E1650917F1660910C
:10F3C0008016709181168091771690917816A09191
:10F3D0007916B0917A16481759076A077B0700F526
:10F3E0008FE590E00E944756811143CFC5CC009332
:10F3F0001F037DCF80E090E0DC01C7CFA9014F5F04
:10F400005F4F5093DB0F4093DA0F4091DC0F509128
:10F41000DD0F4252504F240F351FF901838329CF4E
:10F4200040917E1650917F166091801670918116E2
:10F430008091771690917816A0917916B0917A16EE
:10F44000481759076A077B0708F496CC0E94147086
:10F45000892B09F091CC0F943A428CE593E60E94F7
:10F46000D4720F94C41C6B017C010E94B95F8CE3C1
:10F47000882E912CA12CB12CC701B601A5019401B5
:10F480000F94AFA1CA01B901A50194010F94AFA1D6
:10F490007F936F93C701B60120E13EE040E050E06A
:10F4A0000F94AFA13F932F9382E193E79F938F93A4
:10F4B0008E010F5F1F4F1F930F930F9453A087E789
:10F4C0009EE90E94DB70C8010F945D9AC8010E94FA
:10F4D0008DEF0F949B4D109256020FB6F894DEBF3D
:10F4E0000FBECDBF80916B13882359F00F946E44EB
:10F4F0008091CA0D882309F43FCC86E00F945F9970
:10F500003BCC81E00F94DA4D80916B138111EECFEB
:10F51000EFCF0F931F93CF93DF93D82F8091841653
:10F52000813009F449C0823009F44DC00E949A61CB
:10F530008111ECC08091F1119091F211009739F492
:10F540002091ED113091EE11232B09F4DFC0409191
:10F5500033025091340260913502709136024115A8
:10F5600051056105710509F4D1C0892B31F48091F1
:10F57000ED119091EE11892B29F080911A068823C4
:10F5800009F42CC18091CA0D882321F040EE52E38A
:10F5900069E270E08AE196E00F943C10882309F458
:10F5A000B7C00F94B91280E696E30E94326D0F94B3
:10F5B0007B0B0E943FFEACC082E0809384160E94C9
:10F5C000F4C3809387161092881680918416823037
:10F5D00009F0ACCF8091891681113DC00E94F4C31F
:10F5E000C82F80918716C81709F4A0CFC09387163B
:10F5F00089E896E10F943010CC23B1F18091851603
:10F60000882311F18091620381111EC080919412B0
:10F610008130D1F08091A80D9091A90D891B8F7038
:10F6200099F40E94496181110FC08091C80D843006
:10F6300059F08FE59FE00F943CA1811105C061E076
:10F6400087E797E30F94899581E08093881681E09E
:10F6500080935B026BCF64E670E089E896E10F94DB
:10F6600001108111BBCF62CF80918616882379F378
:10F67000809162038111EBCF8091A80D9091A90D2B
:10F68000891B8F7021F40E944961882301F38091C6
:10F69000E7118111DCCF809194128130C1F2809109
:10F6A000C80D8430A1F28FE59FE00F943CA1811139
:10F6B000CECF8AE295E69F938F9380E195E69F9364
:10F6C0008F930F94FE9F10928616109285160F90BE
:10F6D0000F900F900F908091E711811105C060E0AD
:10F6E00070E0CB010F94474260E070E0CB010E94D4
:10F6F000C16185E69FE00E948D6F81E09FE00E94DE
:10F70000806F8FE19CE60F94B443A1CF10921A064C
:10F710008091CF119091D011039714F40E94FA7543
:10F720009091A80D8091A90D981781F08091CB0D33
:10F73000863061F468E873E185ED91E10F94011082
:10F74000882321F085ED91E10F943010409146031C
:10F750005091470360914803709149034115510549
:10F760006105710509F03FC04091370250913802A0
:10F770006091390270913A02411551056105710598
:10F78000A9F08AE493E00F943C10882379F09091DB
:10F79000A80D8091A90D981309C0D11107C0179A1F
:10F7A0001092A306169A1092A406149AC091E91119
:10F7B0009091A90D8091A80D981701F18091A90D44
:10F7C0009EE6899FF0011124E25FF84FC08190917D
:10F7D000A80D981799F08F5F8F70F9CF8AE196E0A6
:10F7E0000F94FB1195CF8AE493E00F943C1088238B
:10F7F00009F4BACF80E698E70E946073CC2309F43D
:10F80000BEC08091410390914203A0914303B09107
:10F810004403892B8A2B8B2B81F40F94CE0F605ECF
:10F820007C4F8F4F9F4F60934103709342038093AF
:10F83000430390934403CFEF0FC00F94CE0F00917A
:10F840004103109142032091430330914403601718
:10F8500071078207930778F380918403882309F462
:10F8600097C0C093670280912D04811107C081E089
:10F8700080932D040F94B26510922D04809113068D
:10F880008823C9F1109213064FB7F894809111069E
:10F89000282F082E000C330B37FF03C0319521951C
:10F8A0003109243031050CF476C0982F87FF02C04F
:10F8B00093E0980F95959595209106053091070551
:10F8C000290F311D97FD3A953093070520930605C2
:10F8D000837887FF03C081508C6F8F5F8093110600
:10F8E0004FBF86E00F94FD2C80915B02811103C015
:10F8F00081E080935B0280911406882361F00E946E
:10F90000146CE091D403F091D503309721F08091ED
:10F910005C02811119952091621330E0A8EEB3E0EA
:10F920000F94DCA1AB01BC0183E693E10F943C1082
:10F93000882399F08091611380FD0E944D7280911F
:10F94000611382FD0E94D2718091611381FD0E943A
:10F950001E6083E693E10F94FB118091CA0D811123
:10F9600002C00E94D87240E355E760E070E08AE58B
:10F9700093E0DF91CF911F910F910D943C10109265
:10F98000410310924203109243031092440364CF48
:10F99000C093050568CF109211064FBF80E0A2CF3B
:10F9A000CF93DF93EC010F94AF3281E00E94897A0C
:10F9B00080E00E94C369209799F0C233D10540F0DE
:10F9C00062E370E080E090E00F94D50DE297EBCF1A
:10F9D000BE0190E080E00F94D50DD0E0C0E0E3CF11
:10F9E000DF91CF910895CF93DF93C82FDFEF0F946E
:10F9F000AF3281E00E94897A809192128F3FD9F4D0
:10FA000080912712843021F480912A128111EFCF46
:10FA10008091651290916612019749F780918C123E
:10FA200090918D128932904811F360E089E290E85C
:10FA30000F940750DCCFD0939212853039F4CF3F2A
:10FA4000F9F261E08C2F0F944E6CD1CF8430C1F667
:10FA5000DF91CF910895CF93DF93EC0189918823B3
:10FA600019F00E94C270FACFDF91CF910895FF92F2
:10FA70000F931F93CF93DF93EC01F62E662309F4C7
:10FA80004BC00F94FA9E8C01C8010E9447568823F0
:10FA900009F453C08091DC0F9091DD0FFC01E2521C
:10FAA000F04F23E020838F51904FBE01FF20E9F1FA
:10FAB0000F94F39E87E79EE90E94DB7081E593E651
:10FAC0000E94DB708091DC0F9091DD0F8F51904F81
:10FAD0000E942B7D80EF92E70E94D4728091DC0F10
:10FAE0009091DD0F0496080F191F0D3E81E0180755
:10FAF000F9F01093DD0F0093DC0F8091CF119091FE
:10FB0000D01101969093D0118093CF11DF91CF91B6
:10FB10001F910F91FF900895FC0101900020E9F7DB
:10FB200031978F01081B190BAFCF0F94A7A7C2CF36
:10FB30001092DD0F1092DC0FE0CF8AE59EE90E9463
:10FB4000DB7081E593E60E94DB70CE01FF2059F067
:10FB50000E94DB7088E29EE9DF91CF911F910F91A7
:10FB6000FF900C94D4720E942B7DF4CF0F931F93BF
:10FB7000CF93DF93D62F8C01C0E0F801859194914B
:10FB800061E00E94377DCF5F0E5F1F4FDC13F5CF22
:10FB9000DF91CF911F910F910895CF93DF93CDB750
:10FBA000DEB76E970FB6F894DEBF0FBECDBF9E01D5
:10FBB0002C5D3F4FF901419151919F016EE170E041
:10FBC000CE0101960F9492A060E0CE0101960E94B2
:10FBD000377D6E960FB6F894DEBF0FBECDBFDF91B6
:10FBE000CF9108951F920F920FB60F9211240BB66A
:10FBF0000F922F933F934F935F936F937F938F93C6
:10FC00009F93AF93BF93EF93FF9320917800309130
:10FC10007900E0911603F0E0EE0FFF1FEA5FFC4F62
:10FC200080819181820F931F91838083809105034E
:10FC30008F5F809305038031E9F5809116038F5F14
:10FC400080931603883071F5809106039091070325
:10FC500090934A068093490680910A0390910B0382
:10FC600090934C0680934B06809108039091090372
:10FC7000909348068093470681E080936306FF9146
:10FC8000EF91BF91AF919F918F917F916F915F9114
:10FC90004F913F912F910F900BBE0F900FBE0F9081
:10FCA0001F901895809104034FE553E08F5F41F456
:10FCB0001092040380917A00806480937A00DFCFF1
:10FCC0009A01082E02C0359527950A94E2F720FF85
:10FCD000EDCF809304030E94585510920503EACF9C
:10FCE000CF93DF93CAE7D0E088818F7B888310921F
:10FCF0000503109216031092040380E00E945855E9
:10FD0000E6E0F3E080E1DF011D928A95E9F7888162
:10FD100080648883DF91CF9108952F923F924F9214
:10FD20005F926F927F928F929F92AF92BF92CF928B
:10FD3000DF92EF92FF920F931F93CF93DF93CDB794
:10FD4000DEB7A4970FB6F894DEBF0FBECDBF0F94F9
:10FD5000A0228091AC0D811117C081E08093061222
:10FD60008091A306882349F08091A406882329F076
:10FD70002091A5062F83211120C081E08093E611F8
:10FD800086EB98E60F94B443A4960FB6F894DEBFC2
:10FD90000FBECDBFDF91CF911F910F91FF90EF90DC
:10FDA000DF90CF90BF90AF909F908F907F906F909B
:10FDB0005F904F903F902F9008958BEA9DE00F94B5
:10FDC0003CA1182F8EE40E94B655082F0E94CB55F7
:10FDD0008E83002329F0873009F4C9C0833029F0CD
:10FDE000133009F0C3C063E06E8380E090E0A0E8C8
:10FDF000BFE38A839B83AC83BD838AEA9DE00F9433
:10FE00003CA1888F83E40E94B655182F0E94CB55E1
:10FE1000112329F0882319F08B3008F4888F88E5A6
:10FE20000E94B655882309F4ABC00E948E5A20E088
:10FE300030E048E052E40F9463A220E030E048EB69
:10FE400051E40F9463A26A877B878C879D8789E53D
:10FE50000E94B655882309F49CC00E948E5A20E067
:10FE600030E048E052E40F9463A220E030E040EA42
:10FE700050E40F9463A26C8B7D8B8E8B9F8B87E5F8
:10FE80000E94B655882309F489C00E948E5A2A859B
:10FE90003B854C855D850F9464A220E030E048E806
:10FEA00052E40F9464A2698F7A8F8B8F9C8F88E4C1
:10FEB0000E94B655882309F47AC00E948E5A2C8974
:10FEC0003D894E895F890F9464A220E030E048E8C4
:10FED00052E40F9464A26D8F7E8F8F8F98A30F943E
:10FEE000515780912C0290912D02A0912E02B09139
:10FEF0002F0280939D1290939E12A0939F12B09315
:10FF0000A0120F946B8C05EC1FE0C8010F944AA15E
:10FF1000019609F051C00E5F1F4F053D8FE0180795
:10FF2000A1F7212CACE9B2E1BAA3A9A3B987A887AC
:10FF3000512C412C312C042D842D63E00F94EBA126
:10FF4000988B6884798410E0F889F11137C0812F8B
:10FF500063E00F94EBA1911131C021103FC17E816C
:10FF6000733009F470C08F818E8737C01E836AE9B1
:10FF700079E989E19FE36A837B838C839D833DCF0D
:10FF800080E090E0A0E8BFEF8A879B87AC87BD87C1
:10FF90005ECF60E070E080E89FEF6DCF80E090E0A2
:10FFA000A0E8BFE7898F9A8FAB8FBC8F80CF60E0CE
:10FFB00070E080E89FE78FCF2F80B4CF60E070E0E3
:10FFC00080EC9FE7D30111966D937D938D939C9365
:10FFD0001497BE81B330C1F11E86812F0F94C58C5A
:10FFE0004B015C01802F0F94C58C6B017C01A50136
:10FFF00094016A857B858C859D850F94EDA41816E8
:020000021000EC
:100000000CF41CC1298D3A8D4B8D5C8DC501B4015A
:100010000F94EDA418160CF411C1A70196016C8978
:100020007D898E899F890F94EDA418160CF406C162
:100030002D8D3E8D4F8D58A1C701B6010F94EDA4B3
:1000400018160CF4FBC033941F5F24E0620E711C81
:10005000173009F079CF6FEF461A560A88859985CF
:100060004C969987888797E04916510409F063CF29
:100070000E9408F1A091C706AF83B091AC03B88786
:1000800081E08093C7068AE0830D8093AC0381E012
:100090000E94C36980E090E0A0EAB0E48093FD1183
:1000A0009093FE11A093FF11B093001265E575E5E2
:1000B00085E591E40F94D08580E00E946F609CA359
:1000C0008BA3312C832D67E00F94EBA1F82E092F21
:1000D000682F70E07F876E8780FF03C076E0791B12
:1000E000072F802F63E00F94EBA1911105C08F2D96
:1000F0000F94EBA111E0911110E0802F0F94C58CAB
:10010000688B798B8A8B9B8B8F2D0F94C58C4B01C1
:100110005C018E81833009F099C01111C8C027E0BD
:10012000AE85BF852A9FF0012B9FF00D1124E00FB3
:10013000F11DEE0FFF1FEE0FFF1FE456FD4E60E0B6
:1001400070E080EC9FE761837283838394833394B0
:10015000E1E33E12B7CF80E090E0A0EAB0E4809304
:10016000FD119093FE11A093FF11B093001265E56D
:1001700075E585E591E40F94D0850F94A022B1E355
:100180003B1609F43CC280913F0391E0980F909395
:100190003F03882309F4D3C160E080E00E949EEF12
:1001A00084E396E30E94326D0F947B0B80E00F9402
:1001B000F72F81E0809378028BE09CE60E9493E623
:1001C0002F812093C70668856093AC0382E00E946C
:1001D000C3690F94A02210920612D6CD011103C05C
:1001E000112309F4BCCE812F63E00F94F7A1840D95
:1001F000952D911D880F991F8D53904F0F944AA1F3
:10020000BC01990F880B990B0F94CA9B2AE037ED1C
:1002100043E25CE30F94099C9B01AC0160919D1249
:1002200070919E1280919F129091A0120F9464A2DF
:10023000F301618372838383948391CEFE85FF23D0
:1002400009F402CF222009F4FECEFECE2889398996
:100250004A895B896A857B858C859D850F94EDA491
:10026000181604F1288939894A895B89698D7A8D44
:100270008B8D9C8D0F9459A387FD14C0A50194010B
:100280006C897D898E899F890F94EDA4181654F08E
:10029000A50194016D8D7E8D8F8D98A10F9459A32A
:1002A00087FF05C0112309F452CF211050CF10E071
:1002B000A7E08E859F85A89FF001A99FF00D1124CE
:1002C000E00FF11FEE0FFF1FEE0FFF1FE456FD4E74
:1002D0004180528063807480C12CD12CE0EAEE2EE4
:1002E000E0E4FE2E222051F023E333E343EB5EE310
:1002F000C301B2010F9464A26B017C01A7019601B6
:100300006091FD117091FE118091FF11909100128A
:100310000F9459A387FF10C0C092FD11D092FE1117
:10032000E092FF11F092001265E575E585E591E434
:100330000F94D0850F94A022688979898A899B8936
:100340006093F5117093F6118093F7119093F81163
:100350008092F9119092FA11A092FB11B092FC11C7
:1003600069EF71E185EF91E10E94276460E070E040
:1003700086E193E40F94D0850F94A0228091AC0D78
:10038000882339F07F817093C70688858093AC03FA
:10039000FBCC812C912C70E2A72E71ECB72E222081
:1003A00051F02A813B814C815D81C301B2010F94E0
:1003B00063A24B015C01488DC501B4010F945B57EA
:1003C00081110BC089EE92E60E94326D9F938F934C
:1003D0000F94FE9F0F900F90BECE2091FD11309193
:1003E000FE114091FF1150910012C701B6010F9408
:1003F00063A220E030E0A9010F9459A387FF36C023
:1004000060E070E080EA90E46093FD117093FE116B
:100410008093FF119093001265E575E585E591E401
:100420000F94D0850F94A022488DC501B4010F947C
:100430005B57882339F22091FD113091FE114091D4
:10044000FF115091001260E070E080EA90E40F9498
:1004500063A22DEC3CEC4CEC5DE30F9459A387FFB9
:1004600005C08DEA97E70F9425A075CEC090FD11C9
:10047000D090FE11E090FF11F09000122220A1F028
:10048000A7019601C301B2010F9463A29B01AC01C5
:100490005F776A817B818C819D810F9459A387FF4F
:1004A00003C084E797E7DFCF8FEA9FE00F943CA17A
:1004B000882309F440C086EA9FE00F943CA188237A
:1004C000D1F160918E0670918F0680919006909187
:1004D00091060E948F5620913E0430913F04409136
:1004E0004004509141040F9463A39B01AC01E7E0E9
:1004F000AE85BF85EA9FC001EB9F900D1124080FC8
:10050000191F000F111F000F111F04561D4EC701A8
:10051000B6010F9463A2D80111966D937D938D93CC
:100520009C9314978091AC0381508093AC0381E03D
:100530000E94C3690CCE20E030E0A901D8CF85E04D
:100540000F94FD2CC12CD12C90EAE92E90E4F92EC9
:1005500080E096E30E94326D0F94F40A90E080E010
:100560000F94F53481E00F94513580E00F94D82C2E
:10057000182F60E070E080E89FEB0E945E6781E0EA
:100580000F94D82CC092FD11D092FE11E092FF1171
:10059000F092001265E575E585E591E40F94D0854C
:1005A0000F94A022812F0F94D82C82E00F948C22DC
:1005B00020E030E040EA50E40F94EDA4181644F235
:1005C000EF81E093C706F885F093AC0381E00E94C9
:1005D000416ADD24D394DF92812C912C5401CC24E8
:1005E000C394E12CF12C870121E040E050E0BA01F6
:1005F00081E00E94F467D092E6110F90C5CB109273
:100600003F038BA19CA10E94556010922A05109275
:10061000290580E10E944CD8882391F00E94337311
:1006200081EA9DE00F943CA12BE0829FC001112440
:10063000805B924F0F944AA190932A0580932905DD
:100640006091290570912A05072E000C880B990BE3
:100650000F94CA9B905820913E0430913F044091E2
:100660004004509141040F9463A30F94318C80ECAB
:100670009FE00F943CA191E0813009F090E09983D4
:100680004FEB5FE06CE4CE0101960E94E555F82E39
:100690004EEB5FE062E5CE0101960E94E555082F22
:1006A0004DEB5FE066E4CE0101960E94E555182F00
:1006B0004CEB5FE062E4CE0101960E94E555212FEC
:1006C000110F330B082E000C990B5C01A21AB30A10
:1006D0008F2DFF0C990B280F391F46E0429F6001B8
:1006E000439FD00C1124F12CE12C002E000C110B97
:1006F000081B190BB70163567D4E3B01460177E09D
:100700007A83D3012D903D904D905D903D01FD0188
:100710003497FB87EA87B401092C000C880B990BEE
:100720000F94CA9B2FE333EC4EE259E30F94099CDC
:10073000A20191010F9464A2AA85BB856D937D935C
:100740008D939C931397BA81B150BA83800E911EFA
:10075000B111D7CFCA0CDB1CECE1EE0EF11CF4ECAE
:10076000EF16F10439F60E9408F18DE40E94B655A7
:10077000882309F484C00E94CB552E81273009F0CC
:1007800094C0882309F491C0BB24B394AA24AA94EA
:10079000AB0C09A11AA1612C8EEF882E8B0C6A2D4F
:1007A000862D0F94FC8B99249394960C81116EC026
:1007B0006B2D862D0F94FC8BC12CD12C7601712CC6
:1007C000882381F020E030E0A901D8015D966D9189
:1007D0007D918D919C9190970F9464A26B017C0107
:1007E00077247394682D862D0F94FC8B882369F0F1
:1007F000F8017B972081318142815381C701B60185
:100800000F9464A26B017C0173946A2D892D0F945F
:10081000FC8B882361F0F801258136814781508562
:10082000C701B6010F9464A26B017C0173946A2D19
:100830008FEF860D0F94FC8B882331F1F8013397ED
:100840002081318142815381C701B6010F9464A296
:100850006B017C017394672D70E090E080E00F9451
:10086000CA9B9B01AC01C701B6010F9463A3D801D9
:1008700011966D937D938D939C93149707C08CEA8A
:100880009DE00F943CA179CF7110E5CF692C0C5FEE
:100890001F4FB7E09B1283CFB394E9A1FAA17C96D6
:1008A000FAA3E9A3F8E0BF1271CF81E080939C1214
:1008B0008FE40E94B655811103C00F94868C79CCC9
:1008C0000E94CB558111F9CF0E944A6072CC2F92C1
:1008D0003F924F925F926F927F928F929F92AF92D0
:1008E000BF92CF92DF92EF92FF920F931F93CF931D
:1008F000DF93CDB7DEB7C356D1090FB6F894DEBF8C
:100900000FBECDBF82E0809378020091CB11109191
:10091000CC110F51104F45E050E061EC71E8C80177
:100920000F941B9F892B09F09BC18091CA0D8823CE
:1009300009F44DC08DEB9EE70F94B175882379F0D3
:100940008091F7161F928F9384EB95E69F938F9378
:100950000F94FE9F0F900F900F900F9008C089EB9F
:100960009EE70F94B175882341F01092D60381E081
:10097000809378020E9487733AC286EB9EE70F94B9
:10098000B175882321F18091F5169091F61661E0FA
:1009900003960F94634C0F942B498C01809102169F
:1009A00090910316A0910416B091051680937E16BF
:1009B00090937F16A0938016B0938116802F0E948B
:1009C000C2700A30110539F70F943A42D0CF87EB45
:1009D00091E80F94B1758111CACF83EB91E80F9420
:1009E000B175882321F140918703509188032CE34E
:1009F000249FC001259F900D11249F938F934091B8
:100A0000850350918603249FC001259F900D1124DA
:100A10009F938F9382ED97E69F938F930F94FE9F02
:100A20000F900F900F900F900F900F90A0CF8EEA25
:100A300091E80F94B175882311F18CE89FE00F9431
:100A40003CA1811110C061E089E89CE60E94377DDD
:100A500060E085EA9FE00F9460A160E08FE79CE092
:100A60000F9460A184CF813009F081CF0F94B4201E
:100A700085ED91E10F9430100F94DA0F78CF87EA6B
:100A800091E80F94B175882321F080E00F94BD6345
:100A90006ECF81EA91E80F94B17581110E942861AF
:100AA0008EE991E80F94B1758823A9F044E150E0F4
:100AB00065E17DE0CE0101960F942CA18C898823FD
:100AC00029F083E991E80F9425A051CFCE0101963A
:100AD0000F94CBA74CCF8FE891E80F94B175882382
:100AE00029F083E891E80E94D47241CF8FE791E822
:100AF0000F94B175882319F08FE591E8F4CF8AE55A
:100B000091E80F94B175882319F00E94356C2FCFAE
:100B100087E591E80F94B175882379F081EA9DE02B
:100B20000F943CA12BE0829FC001112470E060E093
:100B3000805B924F0F947EA11ACF84E591E80F94C9
:100B4000B175882351F00E942F6A40E070E060E0A8
:100B500084E690E00F940B32D8CF80E591E80F94B3
:100B6000B1758823E1F086E50E94B655882309F423
:100B7000FECE0E94D85511E0892B09F410E00F94A5
:100B8000A02280919C1290E01817190609F4EFCE6C
:100B900010939C128DEF91E10F945B76E8CE89E47F
:100BA00091E80F94B175882309F4E1CE84E40E94A2
:100BB000B6558823A1F00E948E5A20E030E04AE723
:100BC00054E40F94099C20E030E040E05FE30F9490
:100BD00064A20F94DCA3CB010E942AF0C8CE85E466
:100BE00091E80F94B175882349F18091CA0D88234B
:100BF00029F18091F5169091F61602969093F616CB
:100C00008093F5160E948E5A6B017C016FEF87EA84
:100C10009DE00F9460A120E030E04AE754E4C70172
:100C2000B6010F94099C20E030E040E05FE30F94B0
:100C300064A20F94DCA385EA9DE07CCF85EA9DE069
:100C40000F944AA1BC0190E080E00F94C89B20E083
:100C500030E04AE754E40F9463A30F94E34187CE56
:100C6000D8018C91873411F00C945B911093F61697
:100C70000093F5160E94D85590935803809357031C
:100C80008B34910509F445C60CF04BC184309105B5
:100C900009F4AAC50CF0C5C097FDCFC002970CF0AF
:100CA000A2C10E9400558C010E94B55B6091840630
:100CB0007091850680918606909187060F94C89B57
:100CC0006B017C014090011250900212609003125F
:100CD0007090041280909F069090A006A090A106AC
:100CE000B090A206A5019401C301B2010F9463A2C2
:100CF00020E030E048EC52E40F94099C9B01AC01E9
:100D0000C701B6010F94EDA41816D4F4A301920103
:100D1000C501B4010F9463A220E030E048EC52E436
:100D20000F94099CA70196010F9464A20F94DCA371
:100D30006093840670938506809386069093870659
:100D40008091B404882309F446C188E50E94B65511
:100D5000811141C189E50E94B65581113CC18AE5E6
:100D60000E94B655811137C185E40E94B65588238B
:100D700009F431C120910112309102124091031205
:100D80005091041260919F067091A0068091A10677
:100D90009091A2060F9463A26B017C012DEC3CECB8
:100DA0004CEC5DEB0F9459A387FF07C180910305BD
:100DB00081110C9416B00F94A02280919F069091FF
:100DC000A006A091A106B091A20680930112909373
:100DD0000212A0930312B093041281E092E10F94E7
:100DE00028769091030581E089270E944BBECD595A
:100DF000DF4F0FB6F894DEBF0FBECDBFDF91CF91AE
:100E00001F910F91FF90EF90DF90CF90BF90AF9028
:100E10009F908F907F906F905F904F903F902F901A
:100E200008958531910509F4D9C0FCF48A30910503
:100E300009F423C50B9709F424C58091CB11909137
:100E4000CC118F51904F9F938F931F9287E48F9374
:100E500084EF96E69F938F930F94FE9F0F900F90D1
:100E60000F900F900F900F90B9C08C31910509F43D
:100E70000AC54E9711F70F94A02281E080930512C6
:100E80000E946F608C0180E090E0A8E4B4E480935D
:100E90007A0290937B02A0937C02B0937D0243E0A0
:100EA00060E070E080E291EC0F945B577090FD1170
:100EB0006090FE115090FF1140900012B090F91117
:100EC000A090FA119090FB118090FC11F090F51118
:100ED000E090F611D090F711C090F8118FE296E5EE
:100EE0000E94326D4F925F926F927F928F929F928B
:100EF000AF92BF92CF92DF92EF92FF929F938F9328
:100F00008DEA97E69F938F930F94FE9FC8010E94EE
:100F10005560109205120FB6F894DEBF0FBECDBF1C
:100F20005DC08835910509F459C0F4F48135910507
:100F300011F40C94A1905CF48C34910509F40CC567
:100F40008035910509F079CF0E948D7E47C08635A6
:100F5000910511F40C94A5908735910509F06DCF9A
:100F600080E10E947DC63AC08C35910511F40C9445
:100F7000B19074F48A35910511F40C94AA908B35D4
:100F8000910509F05ACF8091EB1187600C94AD90D8
:100F90008236910511F40C9448918336910509F03D
:100FA0004CCF1092CA0D60E084EC9FE00F9460A1DA
:100FB00082E00E94C3690C9457912DEC3CEC4CEC00
:100FC0005DE3C701B6010F94EDA4181624F48091D7
:100FD00003058111F0CEC8010E9485651092580367
:100FE00010925703C4CC0E9400552E969FAF8EAF2F
:100FF0002E970E94B55B89E40E94B655882309F4B8
:10100000A0C30E948E5A60934F0370935003809345
:101010005103909352038AE40E94B655C12CD12CFF
:101020007601882321F00E948E5A6B017C01C092C8
:101030005303D0925403E0925503F0925603E0918B
:101040005703F0915803A496FFAFEEAFA49780909A
:101050004F0390905003A0905103B0905203A7010A
:101060009601C501B4010F9400A524966CAF7DAF25
:101070008EAF9FAF249760918E0270918F02072EE2
:10108000000C880B990B0F94CA9B20917A02309127
:101090007B0240917C0250917D020F94099C2EE3CB
:1010A00033EC4EE259E30F94099C68AF79AF8AAFF5
:1010B0009BAF80E1E5EFF1E1DE01119601900D9229
:1010C0008A95E1F7A5019401505828A739A74AA7A6
:1010D0005BA7D701C601B0588CA79DA7AEA7BFA735
:1010E00029813A814B815C8128962CAF3DAF4EAF70
:1010F0005FAF2897C501B4010F9464A262966CAFEC
:101100007DAF8EAF9FAF62978D819E81AF81B88595
:101110002C968CAF9DAFAEAFBFAF2C979C01AD01AD
:10112000C701B6010F9464A266966CAF7DAF8EAF17
:101130009FAF669729853A854B855C8560919B06B4
:1011400070919C0680919D0690919E060F9463A2DB
:101150006A966CAF7DAF8EAF9FAF6A972091930672
:101160003091940640919506509196066E962CAF5C
:101170003DAF4EAF5FAF6E9762962CAD3DAD4EADBD
:101180005FAD62976E966CAD7DAD8EAD9FAD6E9787
:101190000F9463A26B017C01809197069091980651
:1011A000A0919906B0919A06A2968CAF9DAFAEAF72
:1011B000BFAFA29766962CAD3DAD4EAD5FAD6697C5
:1011C000BC01CD010F9463A24B015C013090F60489
:1011D0002090F7049091F8049CABA091F904ACAF77
:1011E000B091FE04B8ABA701960168A579A58AA5C0
:1011F0009BA50F94099C2B013C01A50194016CA5B2
:101200007DA58EA59FA50F94099C9B01AC01C301F0
:10121000B2010F9464A22B013C01A501940168A5C1
:1012200079A58AA59BA50F94099C4B015C01A70198
:1012300096016CA57DA58EA59FA50F94099C9B0189
:10124000AC01C501B4010F9463A2A30192010F94F4
:10125000E3A26B017C0120E030E0A9010F9459A3C7
:1012600087FF0AC02BED3FE049EC50E4C701B6010F
:101270000F9464A26B017C016091FF0470910005E2
:101280006115710509F461C290E080E00F94C89B7C
:101290009B01AC016BED7FE089EC90E40F9463A3BC
:1012A00024962CAD3DAD4EAD5FAD24970F94099CB7
:1012B0005B018C016091010570910205611571055A
:1012C000E1F090E080E00F94C89B20E030E040E740
:1012D00052E40F94099C9B01AC0168AD79AD8AADD5
:1012E0009BAD0F9463A33B014C019501A8010F94A2
:1012F00059A387FF02C0530184014090FA04509023
:10130000FB046090FC047090FD049501A801B201FB
:10131000C3010F94EDA4181684F09501A801632D64
:10132000722D8CA99CAD0F9459A32501380187FF1C
:1013300004C0432C522C6CA87CACA496EEADFFAD3F
:10134000A497329751F42BED3FE049EC50E4C701EC
:10135000B6010F9463A26B017C016E962CAD3DAD7E
:101360004EAD5FAD6E9728966CAD7DAD8EAD9FADE9
:1013700028970F9459A3811123C0A2962CAD3DAD9F
:101380004EAD5FADA2972C966CAD7DAD8EAD9FAD91
:101390002C970F9459A3811113C020E030E0A901CC
:1013A000C701B6010F9459A381110AC02BED3FE08C
:1013B00049EC50E4C701B6010F9464A26B017C01B3
:1013C000A701960124966CAD7DAD8EAD9FAD24979F
:1013D0000F94099C6A962CAD3DAD4EAD5FAD6A97FA
:1013E0000F9400A54B015C012FE632E143E85AE37C
:1013F0000F9459A387FD9EC19201A301C501B401B9
:101400000F9463A30F9442A30F94DCA37DAB6CAB4A
:101410006230710508F45EC12E964EAD5FAD2E9719
:10142000452B09F457C190E080E00F94C89B4B0115
:101430005C01AC019B01C701B6010F9463A32B01B2
:101440003C01A50194016A966CAD7DAD8EAD9FAD5A
:101450006A970F9463A328966CAF7DAF8EAF9FAF52
:1014600028972D853E854F85588960919F067091FC
:10147000A0068091A1069091A2060F9463A2A501F7
:1014800094010F9463A32C966CAF7DAF8EAF9FAF8A
:101490002C97A3019201C301B2010F94099C6B0127
:1014A0007C01AC019B01C301B2010F94099C20E0B7
:1014B00030E040EC50E40F9463A39B01AC01C30106
:1014C000B2010F9463A26CAF7DAF8EAF9FAF20E0EF
:1014D00030E040E05FE3C701B6010F94099C9B0137
:1014E000AC0160E070E080E89FE30F9463A2249673
:1014F0006CAF7DAF8EAF9FAF249722242394312C05
:10150000D8A8DA9458A9511125C1B10190E080E022
:101510000F94C89BA30192010F94099C6B017C015D
:101520000F945EA36CA77DA78EA79FA7C701B601E6
:101530000F9424A64B015C01C0904F03D090500340
:10154000E0905103F0905203F7FAF094F7F8F0941A
:101550008091530390915403A0915503B091560389
:1015600088AB99ABAAABBBABA70196016CA57DA5D7
:101570008EA59FA50F94099C68A779A78AA79BA70A
:1015800028A939A94AA95BA9C501B4010F94099CEE
:101590009B01AC0168A579A58AA59BA50F9464A2BF
:1015A00068A779A78AA79BA7A7019601C501B401DF
:1015B0000F94099C6B017C0128A939A94AA95BA950
:1015C0006CA57DA58EA59FA50F94099C9B01AC01E0
:1015D000C701B6010F9463A26CA77DA78EA79FA732
:1015E0009091FE0498AB28A539A54AA55BA5629603
:1015F0006CAD7DAD8EAD9FAD62970F9464A2698393
:101600007A838B839C832CA53DA54EA55FA566960A
:101610006CAD7DAD8EAD9FAD66970F9464A26D836A
:101620007E838F83988728962CAD3DAD4EAD5FAD00
:10163000289769857A858B859C850F9464A2698734
:101640007A878B879C872C962CAD3DAD4EAD5FADD8
:101650002C976D857E858F8598890F9464A26D8700
:101660007E878F87988BCE0101960E9446652E96C5
:10167000AEADBFAD2E972A163B06F8F0E984FA848A
:101680000B851C852D813E814F81588569817A812A
:101690008B819C813F922F92E5EFF1E1FF93EF93D5
:1016A00088AC99ACAAACBBACFE013D966F010F941F
:1016B00082760F900F900F900F908091AC0D81115A
:1016C00039C0FFEF2F1A3F0A2CA93DA92215330577
:1016D00009F016CF83E996E00E944665E0909B06EC
:1016E000F0909C0600919D0610919E062091970611
:1016F000309198064091990650919A066091930610
:101700007091940680919506909196061F921F9273
:10171000E5EFF1E1FF93EF9388AC99ACAAACBBACD9
:10172000EFE9CE2EE6E0DE2E0F9482760F900F903A
:101730000F900F900E9437558AE493E00F94FB11AD
:101740004DCC60E070E0CB015ECCA32CB22C0CA998
:101750001CADB0CD28A539A54AA55BA56CAD7DAD66
:101760008EAD9FAD0F94099C4B015C012CA53DA54E
:101770004EA55FA524966CAD7DAD8EAD9FAD249733
:101780000F94099C9B01AC01C501B4010F9464A2A4
:101790007B018C0128A539A54AA55BA524966CADD3
:1017A0007DAD8EAD9FAD24970F94099C4B015C01DC
:1017B0002CA53DA54EA55FA56CAD7DAD8EAD9FADB5
:1017C0000F94099C9B01AC01C501B4010F9463A265
:1017D00068A779A78AA79BA7D8AAC701D8018CA711
:1017E0009DA7AEA7BFA7FFCE80E50E94B655C12C2E
:1017F000D12C7601882331F00E948E5A0F94DCA3FD
:101800006B017C0183E50E94B655882361F00E943C
:101810008E5A20E030E04AE754E40F94099C0F947C
:10182000DCA36B017C01C114D104E104F10441F09B
:101830008091C706873021F089EC97E60E9493E6F5
:101840000F94A0220F94CE0FC60ED71EE81EF91ECD
:101850008AE493E00F94FB110F94CE0F6C157D0575
:101860008E059F0508F0BACB0F94AF3280E00E943E
:10187000897A80E00E94C369EFCF81E00E944BBE6D
:10188000ADCB80E0FBCF88E50E94B655382E412CC9
:10189000512C3201882321F00E941E562B013C015D
:1018A00089E50E94B655282E882371F10E941E56A4
:1018B0006CA77DA78EA79FA78AE50E94B655D82E54
:1018C000812C912C5401882321F00E941E564B013B
:1018D0005C0187E50E94B65588A78F93CD2CECA4B8
:1018E000FDA40EA51FA5222DB301A201832D0E94E8
:1018F000F4670F90311072CB211070CB38A53111E5
:101900006DCBD1106BCB20CB1CA61DA61EA61FA68F
:10191000D3CF08E210E094EAE92E97E6F92E602F83
:1019200070E090E080E00F94C89B0E948F569F93D8
:101930008F937F936F931F930F93FF92EF920F9468
:10194000FE9F0F5F1F4F0FB6F894DEBF0FBECDBFD7
:101950000F36110521F742CB0F940C15811105C0EC
:1019600081E391E80E94D47239CB82E00E944CD886
:10197000811107C08BE29AE30E94326D0F947B0BBA
:101980002DCB8091A306882341F08091A406882363
:1019900021F0D090A506D11008C081E08093E61117
:1019A00086EB98E60F94B44319CB82EE99E30E943C
:1019B000326D0F947B0B8BE991E50E94326D41E013
:1019C00060E00F94332E81116EC080E090E0A0EAB9
:1019D000B0E48093FD119093FE11A093FF11B0939A
:1019E000001260E070E088E492E40F94D08580E01B
:1019F00090E0A8E4B2E48093FD119093FE11A093CF
:101A0000FF11B093001280E090E0A4E3B3E4809370
:101A1000F9119093FA11A093FB11B093FC1160E0BF
:101A200070E088E492E40F94D0850F94A02281E7BF
:101A300091E50E94326D0F947B0BE3E5F9E8859107
:101A40009591A591B4918093F9119093FA11A09377
:101A5000FB11B093FC11EFE4F9E885919591A59104
:101A6000B4918093F5119093F611A093F711B09370
:101A7000F81160E070E088E492E40F94D0850F9450
:101A8000A02281E08F93812C912C5401CC24C3940B
:101A9000E12CF12C870120E040E050E0BA0180E029
:101AA0000E94F4670F9020E030E04CE052E4609137
:101AB0008E0670918F0680919006909191060F94FA
:101AC000EDA418160CF076C08091CA0D811172C079
:101AD00080E090E0A8ECB2E48093FD119093FE11B9
:101AE000A093FF11B093001260E070E088E492E4EC
:101AF0000F94D0850F94B91219821A821B821C820E
:101B00001D82CE0101960F94FB1183E2F82E0EEA9E
:101B10001EE720E030E04CE052E460918E067091C8
:101B20008F0680919006909191060F94EDA418165F
:101B3000C4F584E999E30E94326D0F94F40A42E8F7
:101B400064E080E00E941C6A1F92FF9260918E0602
:101B500070918F0680919006909191060F94D5A375
:101B60007F936F931F930F930E94D56981E80E9422
:101B7000EB6988EE93E00E94D07C0E94E97040E01F
:101B800053E567E070E0CE0101960F943C100F9092
:101B90000F900F900F900F900F90882309F4B9CFFA
:101BA000D12C81E00E94416AD11004C080E00F94E2
:101BB0000C0C14CA0F94A02281E0809305120E949D
:101BC000416A83E191E80E94D47280908E069090E1
:101BD0008F06A0909006B090910620E030E040EA99
:101BE00050E4C501B4010F9463A30F94D5A325E07D
:101BF000269FA001279F500D1124BA01550F880B75
:101C0000990B0F94CA9B1B017C0120E030E04CE053
:101C100052E40F9459A387FF06C0212C312C1CE0FD
:101C2000E12E02E4F02E222D332D4E2D5F2DC50125
:101C3000B4010F94EDA4181664F420E030E040EAFB
:101C400050E4622D732D8E2D9F2D0F9464A21B01E5
:101C50007C01FF92EF923F922F928BE897E69F9341
:101C60008F930F94FE9F20E030E040EF51E4622D0F
:101C7000732D8E2D9F2D0F9463A220E030E04CE851
:101C800052E40F9464A20F94D5A37093EE11609365
:101C9000ED1184E08093C70681E08093AC0386E376
:101CA0009BE30E94326D0E9493E680E090E0A0EA00
:101CB000B0E48093FD119093FE11A093FF11B093B7
:101CC000001260E070E088E492E40F94D08580E038
:101CD00090E0A0EAB1E48093F5119093F611A093FF
:101CE000F711B093F81180E090E0A0E7B2E48093A0
:101CF000F9119093FA11A093FB11B093FC1160E0DD
:101D000070E088E492E40F94D0858AE999E9A9E12A
:101D1000BEE38093FD119093FE11A093FF11B09349
:101D2000001260E070E088E492E40F94D0850F9494
:101D3000A0220F900F900F900F900F900F90209176
:101D40008E0630918F064091900650919106622D3B
:101D5000732D8E2D9F2D0F94EDA418163CF488EE54
:101D600093E00E94D07C0E94E970E9CF60E086EAAF
:101D70009FE00F9460A180E090E0A0EAB0E480933F
:101D8000FD119093FE11A093FF11B093001260E03B
:101D900070E088E492E40F94D085EFE4F9E885914F
:101DA0009591A591B4918093F5119093F611A0931C
:101DB000F711B093F811E3E5F9E885919591A591B4
:101DC000B4918093F9119093FA11A093FB11B09301
:101DD000FC1160E070E088E492E40F94D0850F94E9
:101DE000A02243E060E070E080E89FEB0F945B5737
:101DF000811105C00F940C0C10920512EFC8909140
:101E0000FD1198A7A091FE11ACA7B091FF11B8AB3E
:101E1000E0910012E8AFEF93BF93AF939F938EE7EB
:101E200097E69F938F930F94FE9F0F900F900F90C4
:101E30000F900F900F90AEEA8A2EAFE09A2EB3E289
:101E4000CB2ED12C0FEF1FEFB6010D2C000C880B01
:101E5000990B0F94CA9B2B013C01DF92CF92C801D2
:101E600002969F938F9322E437E63F932F930F942C
:101E7000FE9F58015FEFA51AB50A0F900F900F90C3
:101E80000F900F900F9011F40C9424B070E060E06C
:101E9000C4010F947EA1A3019201622D732D8E2D9A
:101EA0009F2D0F9459A3181644F485E0A816B10489
:101EB00011F00C9430B005E010E0580197E2A91A37
:101EC00098EFB90AAA0CBB1C85E0809F1001819F86
:101ED000300C11240D5F1F4FEAE94E2EE9E95E2E0A
:101EE000E9E16E2EEEE37E2EF9E08F2EF7E69F2ECF
:101EF000C801029705970CF0D4C0B101635D7F4F14
:101F0000072E000C880B990B0F94CA9B6B017C0168
:101F10001F930F93A5E3B7E6BF93AF930F94FE9F74
:101F20000093AC0320E030E040EF51E4C701B6017C
:101F30000F9463A220E030E040E251E40F94099C4A
:101F400020E030E040EA50E40F9463A320E030E06A
:101F500048E452E40F9464A20F94D5A37093EE1159
:101F60006093ED1180E090E0A0EAB0E48093FD1171
:101F70009093FE11A093FF11B093001260E070E007
:101F800088E492E40F94D08520E030E040EA51E408
:101F90002093F5113093F6114093F7115093F811F7
:101FA00080E090E0A0E7B2E48093F9119093FA11F9
:101FB000A093FB11B093FC1160E070E088E492E420
:101FC0000F94D0854092FD115092FE116092FF1146
:101FD0007092001260E070E088E492E40F94D08583
:101FE0000F94A0220F900F900F900F9020918E06CB
:101FF00030918F064091900650919106C701B6012D
:102000000F94EDA418163CF488EE93E00E94D07C67
:102010000E94E970EBCF80E090E0A0EAB0E480930A
:10202000FD119093FE11A093FF11B093001260E098
:1020300070E088E492E40F94D085EFE4F9E88591AC
:102040009591A591B4918093F5119093F611A09379
:10205000F711B093F811E3E5F9E885919591A59111
:10206000B4918093F9119093FA11A093FB11B0935E
:10207000FC1160E070E088E492E40F94D0850F9446
:10208000A02243E060E070E080E89FEB0F945B5794
:1020900095E0290E311C0F5F1F4F811104C00F9472
:1020A0000C0C81E0A7CE78A56CA598A988AD272F48
:1020B000362F492F582F6091FD117091FE1180919C
:1020C000FF11909100120F9463A2F62EE72ED82EE6
:1020D000C92E20913E0430913F044091400450911C
:1020E0004104D701F6016B2F7A2F8F2F9E2F0F946B
:1020F000099C0F94D5A36CAB7DAB8EAB9FABCF92FD
:10210000DF92EF92FF92809191068F9380919006DB
:102110008F9380918F068F9380918E068F939F92DD
:102120008F920F94FE9F6CA97DA9C5010F947EA18B
:10213000A2E0AA0EB11C0FB6F894DEBF0FBECDBF51
:10214000D7CE0E94B8730C94EE8780E10E9428C617
:102150000C94EE878091EB11887F8093EB110C94A7
:10216000EE8754ECC52E52E0D52E8E010C5D1F4F2C
:102170005801EE24E394F12CD6018D916D010E945B
:10218000B655F50181935F01882391F00E948E5A24
:10219000F701EE0FFF1FEE0FFF1F349721E030E035
:1021A0002C0F3D1FE20FF31F6083718382839383A3
:1021B0003FEFE31AF30A45E0E416F104E9F69FA0C5
:1021C000FCA0992001F120E030E0A9016D857E8519
:1021D0008F8598890F9459A3811115C0F11013C0F0
:1021E0008DA1811110C08EA181110DC0109201121C
:1021F00010920212109203121092041281E0809346
:10220000EF030C94EE870F94A022CE0101965C019F
:102210002AE8C22E24E0D22E35EFE32E31E1F32E50
:10222000380193E0690E711CD8018D918D018823CE
:1022300089F0F6012081318142815381D5016D9170
:102240007D918D919C910F9464A2F70160837183BD
:1022500082839383F4E0AF0EB11C24E0C20ED11C44
:1022600034E0E30EF11C60167106F1F6992061F07E
:102270008D859E85AF85B889809301129093021257
:10228000A0930312B09304120F9490840C94EE87E1
:1022900081E08093CA0D61E084EC9FE00F9460A11F
:1022A0001092890360E08FEF9FE00F9460A10E947D
:1022B00059D80C94EE878D3411F00C9426AF1093FE
:1022C000F6160093F516F801319681918032E9F304
:1022D0008930D9F380538A3030F01F930F938FEFFA
:1022E00090E80C94A6840E94D8559093AB0D8093EF
:1022F000AA0D8E3B910511F40C94339C0CF007C38E
:102300008C34910511F40C944C9B0CF0DEC18C3193
:10231000910511F40C9483990CF0F4C0853191056A
:1023200009F40AC70CF05AC08131910509F4F9C6C5
:10233000DCF4029708F45DC68091CB119091CC112A
:102340008F51904F9F938F931F928DE48F9384EFC3
:1023500096E69F938F930F94FE9F0F900F900F9090
:102360000F900F900F90A8C68231910511F40C9434
:10237000DE9C449709F781E08093780284EE96E62C
:102380000E94D47284E50E94B655182F8CE40E94F6
:10239000B65500E080FB00F910FB01F980EF93E1F6
:1023A0000E94B77083E2E0EFF3E1DE011196019045
:1023B0000D928A95E1F720E050E040E0BE016F5FAA
:1023C0007F4F8AED92E00F94C645CE0101960E94A0
:1023D000BC7086ED96E60E94D4726EC68831910577
:1023E00009F4BBC684F48631910509F4A9C6479760
:1023F00009F0A2CF8091F5169091F61661E004964F
:102400000F94634C59C68A31910509F4ECC60CF05F
:102410000CC704EC12E0F2E4AF2EF2E0BF2EA4E20F
:10242000CA2EA2E0DA2EB8E1EB2EB2E0FB2E87EC4A
:10243000882E82E0982EF80181918F010E94B65576
:10244000882321F10E948E5AD6014D905D906D90A7
:102450007C90A30192010F9459A387FD11C00E94A3
:102460008E5AF7014080518062807380A3019201EF
:102470000F94EDA4181624F00E948E5A2B013C01F3
:10248000D5014D925D926D927C921397B4E0AB0EA4
:10249000B11CE4E0CE0ED11CF4E0EF0EF11C80166E
